:100000000C94FD0F0C942E100C942E100C942E10AA
:100010000C942E100C942E100C942E100C942E1068
:100020000C942E100C942E100C942E100C942E1058
:100030000C942E100C942E100C942E100C942E1048
:100040000C942E100C942E100C942E100C942E1038
:100050000C942E100C942E100C942E100C94F5A7CA
:100060000C942E100C9422870C94F8860C942E106D
:100070000C942E100C942E100C942E100C942E1008
:100080000C942E100C942E100C942E100C942E10F8
:100090000C94CE860C94A4860C942E100C941429E7
:1000A0000C942E100C942E100C942E100C942E10D8
:1000B0000C942E100C942E100C942E100C942E10C8
:1000C0000C942E100C942E100C942E100C947A86F6
:1000D0000C9450860C942E100C9426860C94FC855F
:1000E0000C942E1007634236B79BD8A71A3968566E
:1000F00018AEBAAB558C1D3CB7CC5763BD6DEDFD4A
:10010000753EF6177231BF000000803F0800000006
:10011000BE922449123EABAAAA2ABECDCCCC4C3EFC
:1001200000000080BEABAAAAAA3E00000000BF00EB
:100130000000803F0000000000084178D3BB4387E7
:10014000D1133D190E3CC3BD4282AD2B3E68EC82FB
:1001500076BED98FE1A93E4C80EFFFBE01C4FF7F80
:100160003F00000000000C94FA2D0C9487A10C9421
:10017000B2A10C9423140C94364A0C94803A0C943B
:10018000E0A10C941D470C942D150C9496380C94FA
:10019000EDBD0C9499370C940DA20C948C230C9407
:1001A00071150C94D9160C94DB110C94E1880C9405
:1001B000DC5A0C94C8130C9494A10C94F8880C94F9
:1001C000F8340C946D190C94571E0C94D9B30C94FC
:1001D000C5130C94A8A10C94EE790C940A120C94FB
:1001E0006B7A0C94CC5B0C946C350C948E890C94CB
:1001F00010190C94BAA00C944B280C947D5F0C94AD
:1002000086250C94805F0C9432370C94C33A0C947E
:1002100007140C94BD390C944D380C94EFA10C9438
:1002200028140C9494BE0C94B7160C94BA650C94D4
:10023000EB3A0C949D5B0C94A5250C941F140C9424
:10024000913E0C940EBE0C94915B0C94F0370C9480
:10025000BE680C94E1770C945C3B0C94841E0C9467
:10026000DAA00C94E7130C94D6A10C94A1510C9431
:10027000AC120C94F4140C9483120C9457C00C948C
:1002800035C00C94F65D0C94D5130C949F5A0C94C5
:10029000A75D0C94611F0C94A6280C9423370C9432
:1002A00003A20C9452160C94FB110C94134A0C9458
:1002B000A6230C94BAA10C94962A0C9414370C948F
:1002C000173C0C94FE110C94A23B0C94C2A00C940D
:1002D000EB490C94D8140C944F4A0C9458740C9419
:1002E000BEA00C94B5110C941A210C94A51F0C946B
:1002F00025140C94705E0C940B3A0C94D8880C94D2
:10030000883B0C945B130C948FA10C9463140C9495
:10031000F1810C94E03B0C9414280C945D5B0C94DC
:10032000B25E0C94BF3A0C9466BD0C94957A0C9412
:1003300036370C941A370C947F650C94BE110C94CC
:100340007A4A0C94C41B0C94D5370C94313B0C9412
:100350007E6F0C94BE460C94A17C0C940A190C94EC
:1003600028780C945C790C94417B0C94D8390C94CB
:10037000DB460C9411140C94F3380C94407A0C94D2
:100380003B790C94D18A0C945F790C94F9680C94A5
:100390007A380C9463130C94A3500C94575E0C940D
:1003A00070160C94564A0C948C110C940D1A0C94E3
:1003B0000E150C949D210C94835B0C9424130C94C7
:1003C000E2770C94971E0C94D9BD0C94E5140C9410
:1003D0000D370C94F6780C9497140C945C7A0C946A
:1003E000E2110C94B62F0C94763B0C9458320C947A
:1003F000217B0C947A5F0C946B100C94616D0C94BF
:10040000A9490C946A130C94597B0C9406120C9411
:10041000DA170C947A170C94E3270C94DA110C94E5
:10042000BA210C94C4110C943F140C940D340C9408
:1004300045200C94A57B0C944C780C94B4200C941F
:10044000B33B0C94D3B30C94D6A00C94805B0C9467
:10045000B8250C94E7110C94A6A00C94E1A00C9480
:100460000C190C94BA110C94B0A00C9412190C94A1
:1004700057150C949EA10C94CB1E0C94E6380C944A
:10048000CCA00C94C3370C94AF780C94CCA10C94F2
:10049000C4170C949A110C94D0A00C9490B80C949E
:1004A000DD5D0C94D45E0C941C570C94745B0C941E
:1004B000DD3B0C94CF770C94B4A00C94DA380C94F8
:1004C0004C130C949D3B0C94CF7B0C9431210C94D9
:1004D00042470C94F9110C94711E0C94715D0C94AC
:1004E000EB110C9421380C94A2A00C946BBE0C94CC
:1004F000A15F0C9443890C94C3110C948CB10C949F
:10050000C8A00C94811D0C94C9110C942A5E0C9403
:100510007B120C94841D0C9438780C948F170C94D7
:10052000DEA00C9466350C946E6F0C9443130C94FF
:1005300069200C94EE3F0C94963B0C940E120C9494
:10054000365B0C9498170C94B33A0C9430100C94BE
:10055000DF150C9464380C94F2390C9485380C94A3
:10056000A9270C9402390C9402130C94A0120C9439
:1005700075200C94DFBD0C9455890C9446100C9496
:100580006F380C94D5790C94753A0C94FB3A0C9412
:100590001E120C94F9460C94E2A00C94CB130C940C
:1005A00086BE0C9421A20C94F21D0C94AE7A0C948D
:1005B000EF110C941B3B0C94813E0C944A100C944C
:1005C0000E190C94ED5E0C945B310C94BB110C94E1
:1005D0007B280C9455790C9481210C94C7880C9439
:1005E000225F0C943CB90C94AAA00C94CC110C94EE
:1005F00065790C94F9A10C94BDB60C944A5B0C94EB
:1006000005390C94963A0C9463350C949B110C9418
:100610008E5B0C9417A20C9481200C94CE130C9436
:100620000E740C942B270C94D3380C94523B0C94DE
:10063000F5390C94C2A10C94A9170C9460100C9479
:100640005A780C94373C0C94EA380C94A77A0C94A2
:10065000A0700C947A150C9440380C94A2790C94E8
:1006600008190C949CA00C948B160C9483150C9474
:10067000B23B6364696E6F70737578585B00556E3A
:100680006B6E6F776E207375666669782000556EA5
:100690006B6E6F776E20636D642000636C724374C1
:1006A000723A20002F00496E3A20003D00494E3A30
:1006B000003D004C454741435920494E3A00000057
:1006C00020002300260029002C002F00320000010A
:1006D00000000301060109012D3E00200023002D2A
:1006E0003E00200050656E6465643A20230072610C
:1006F000770076616C0074656D70007361740068DA
:1007000075650066616E0052474200485356006DA1
:100710006F646500536574436D643A0053746F727F
:100720006564204558543A00737566666978436F6E
:1007300064653A004452590046414E5F4F4E4C5951
:1007400000584F4E0048414C54002074696D653A82
:10075000004374726C205265733A002054533A007F
:1007600020543A003D0050696E3A004F4E3A416CB9
:100770007265616479204163746976650A00484155
:100780004C543A416C726561647920496E616374BE
:100790006976650A00584F4E3A416C72656164791A
:1007A000204163746976650A00584F464620736B92
:1007B00069707065642E205072657620636D643AAE
:1007C000005475726E6564206F66662066726F6D88
:1007D0003A00526573746F7265642066726F6D3A89
:1007E0000049676E6F7265642C206368616E6E6588
:1007F0006C20636D643D0020457865633A00416379
:10080000746976653A0048414C543A416C726561AE
:10081000647920496E6163746976650A00584F4EA9
:100820003A416C7265616479204163746976650A46
:1008300000584F464620736B69707065642E2050D7
:1008400072657620636D643A005475726E6564203B
:100850006F66662066726F6D3A00526573746F72D0
:1008600065642066726F6D3A00206D73203A004116
:10087000726D656420666F72200020446973617236
:100880006D656400536B697070656420686F6D6995
:1008900065207374756666004F75744F664D656D9F
:1008A0006F7279210A0020436D643A00205375620B
:1008B0003D00204974656D3D0052414D3D00282D9D
:1008C000292000282B2920002076616C756520697D
:1008D00073200020756E6B6E6F776E0A005D3D00B1
:1008E0005B0020696E76616C6964002000206F6B8C
:1008F000003A00206661696C6564003A00526574D4
:100900007279696E67206D6F6462757320434D4420
:100910000A00207365632072656D61696E696E6798
:1009200000537461747573206465666665726564EE
:100930000A002D3E005075623A2000636D6400434A
:100940004F4F4C0048454154004155544F002D3EF7
:10095000005075623A20007365740064656C002D68
:100960003E005075623A20002D3E005075623A20DC
:1009700000556E6B6E6F776E20636D64200A004FBA
:100980004646004F4E0020002D3E00436F6E7665B8
:100990007274696E6720002D3E0057726F6E67207B
:1009A00041737369676E6D656E74200052474278BB
:1009B0003A200020764C6576656C3A0020436F6ED5
:1009C00076563A0020436F6E76533A0020486F7493
:1009D0003A00436F6C643A0020436F6E7665727420
:1009E000656420563A00436F6E76657274656420C4
:1009F000533A002D3E0057726F6E67204173736942
:100A0000676E6D656E7420002D3E0057726F6E67C5
:100A10002041737369676E6D656E74200053617653
:100A200065643A0020537566663A002041543A00E6
:100A3000436F6E666967206368616E676564206CEA
:100A40006F63616C6C792C20706F7274616C2064C0
:100A5000697361626C6564002F636F6E6669672EEF
:100A60006A736F6E007265626F6F742000436D640D
:100A70003A20002F636F6D6D616E642F002F7261DD
:100A80006D2F002F6974656D2F002F6974656D2FB0
:100A9000004C6F636174696F6E3A20687474703AC9
:100AA0002F2F6C617A79686F6D652E72752F707754
:100AB00061003F6D61633D002669703D0026706FE7
:100AC00072743D00266E616D653D002F002000535D
:100AD0006B697070696E672E2E004F75744F664D8E
:100AE000656D6F727921005D20003A5B000A003A63
:100AF000004D41433A00554450205379736C6F6761
:100B000020696E697469616C697A65642E0A0053A4
:100B100079736C6F6720706172616D733A00437511
:100B20007272656E74204C414E20636F6E66696709
:100B30002869702C646E732C67772C7375626E65F0
:100B400074293A000A5573652074686573652063DB
:100B50006F6D6D616E64733A202768656C70272035
:100B60002D207468697320746578740A276D616339
:100B70002064653A61643A62653A65663A66653A48
:100B80003030272073657420616E642073746F7237
:100B900065204D41432D6164647265737320696EF5
:100BA00020454550524F4D0A276970205B69705BA4
:100BB0002C646E735B2C67775B2C7375626E657447
:100BC0005D5D5D5D27202D207365742073746174F5
:100BD00069632049500A277361766527202D2073A9
:100BE0006176652063757272656E7420636F6E66E0
:100BF000696720696E204E5652414D3B204F4E7C16
:100C00004F4646202D20656E61626C652F646973C6
:100C100061626C65206175746F736176650A276720
:100C2000657427205B636F6E666967206164647218
:100C30005D27202D2067657420636F6E66696720CD
:100C400066726F6D207072652D636F6E6669677571
:100C50007265642055524C20616E642073746F720B
:100C60006520616464722C204F4E7C4F4646202DD7
:100C700020656E61626C652F64697361626C6520CA
:100C8000646F776E6C6F6164206F6E207374617235
:100C90007475700A276C6F616427202D206C6F615A
:100CA0006420636F6E6669672066726F6D204E56B2
:100CB00052414D0A2770776427202D2064656669AC
:100CC0006E6520616E642073746F7265204D51549F
:100CD000542070617373776F72640A276F74617048
:100CE000776427202D20646566696E6520616E64D7
:100CF0002073746F7265204854545020415049202D
:100D000070617373776F72640A276C6F67205B730F
:100D1000657269616C5F6C6F676C6576656C5D2090
:100D20005B7564705F6C6F676C6576656C5D2720C2
:100D30002D20646566696E65206C6F67206C657632
:100D4000656C2028302E2E37290A276B696C6C279A
:100D5000202D2074657374207761746368646F67F5
:100D60000A27636C65617227202D20636C656172B0
:100D700020454550524F4D0A277265626F6F7427A8
:100D8000202D207265626F6F7420636F6E74726FB6
:100D90006C6C657200536F6674207265626F6F745D
:100DA000696E672E2E2E0052414D3D000A4D515462
:100DB0005420000A5379736C6F6720000A6D7174B8
:100DC0007420000A696E7075747320000A69746576
:100DD0006D7320000A436F6E666967757265643AC9
:100DE000003B003D0050696E3A003B003D4C4F57C0
:100DF00000546865726D6F3A004170706C79696E6D
:100E00006720636F6E666967004C6F61646564207C
:100E1000455441473A004E6F2073746F72656420E9
:100E2000636F6E666967004C6F616465642066720B
:100E30006F6D20454550524F4D006C6F61642066C8
:100E400061696C6564004C6F6164696E6720436F13
:100E50006E6669672066726F6D20454550524F4D32
:100E600000436F6E666967206175746F73617665A4
:100E70003A000A5379736C6F672064656275672066
:100E80006C6576656C3A0053657269616C206465C7
:100E9000627567206C6576656C3A005361766564AF
:100EA0000A005365742064796E616D69632049504E
:100EB0000A00454550524F4D20636C656172656470
:100EC0000A004D5154542050617373776F7264203F
:100ED000757064617465640A004F544120506173F9
:100EE00073776F726420757064617465640A00635F
:100EF0006F756C64206E6F742070617273653A2038
:100F000000557064617465640A004E6F204950207A
:100F10006164726573730052656C656173696E67B5
:100F200020736F636B657420616E642072657472E8
:100F30007900205361766564004C6F6164696E6767
:100F4000204854545020636F6E666967206F6E208E
:100F5000737461727475703A004F4646004F4E00CC
:100F60002B002D00455461673A20004765742045E9
:100F70005441473A2000485454502F312E312025F7
:100F8000690025733A2025730D0A002048545450F7
:100F90002F312E310D0A486F73743A2025730D0AD4
:100FA0004163636570743A202A2F2A0D0A436F6EDD
:100FB0006E656374696F6E3A20636C6F73650D0ABA
:100FC0000025730020000D0A004745540066616942
:100FD0006C656420746F20636F6E6E6563740A00C5
:100FE0004552524F523A20536572766572207265AF
:100FF0007475726E65642000436F6E666967206E5B
:101000006F74206368616E6765640A00446F6E6583
:101010002E0A00436F6E6669672070617273696E95
:1010200067206661696C65640A00676F7420436FAE
:101030006E6669670A00667265652000436F6E66BA
:101040006967205552493A20687474703A2F2F000E
:101050002044656661756C7420636F6E66696720F5
:1010600073657276657220757365643A20006C61F1
:101070007A79686F6D652E7275000A282B294D5597
:101080004C544956454E54000A282B2950574D5F61
:1010900052454C4159000A282D294D444E53000A0F
:1010A000282D2955415254425249444745000A28A7
:1010B0002B295359534C4F47000A282D2950494496
:1010C000000A282D294D43503233303137000A2889
:1010D0002D294152544E4554000A282B294F544182
:1010E000000A282D29535049204C4544000A282D38
:1010F000294D4F544F5220435452000A282B294166
:1011000043204841494552000A282D29434353387A
:10111000313120262048444331303830000A282B12
:1011200029524553544152545F4C414E5F4F4E5FDC
:101130004D5154545F4552524F5253000A282D29A5
:101140004841524452455345542C207573696E678B
:1011500020736F6674000A282D29434F554E54455D
:1011600052000A282D29444854000A282D294F5797
:10117000495245000A282D294D4F44425553000A33
:10118000282D29444D58000A282B2957697A6E6565
:101190007435783030000A282B29445332343832E1
:1011A0002D313030000A282B294672656552616D59
:1011B000207072696E74696E670064653A30313A06
:1011C00032333A30303A30303A3031000A466972C0
:1011D0006D77617265204D4143204164647265738F
:1011E0007320006C617A79686F6D652E7275000AE4
:1011F000436F6E666967207365727665723A000A9E
:10120000282B295741544348444F47003230313747
:1012100030334C0020432B2B2076657273696F6E40
:101220003A00353232373138325F323032322D3097
:10123000312D3035000A4C617A79686F6D652E72F8
:1012400075204C6967687448756220636F6E7472AC
:101250006F6C6C65722000204F464600204F4E0098
:101260002042595041535300757074696D65006692
:1012700072656568656170002054696D65723A0039
:10128000204C6F636B733A002000204C6F636B73CC
:101290003A000A52414D3D002045787069726564FC
:1012A0000A00202D746172676574207A6F6E652D57
:1012B0000020416C61726D20457870697265640A26
:1012C0000020636D643A00204375723A0020536534
:1012D000743A00536176656420746F20454550521E
:1012E0004F4D00536176696E6720636F6E66696764
:1012F00020746F20454550524F4D2E2E00206973AB
:10130000200044656C6574696E6720636F6E662E9D
:101310002052414D207761733A0053746F707065AD
:10132000640053746F7070696E67206368616E6EDD
:10133000656C73202E2E2E004E6F7420756E6C6FB0
:10134000636B656420696E20313073202D20636FDC
:101350006E74696E7565202E2E2E00556E6C6F634F
:101360006B696E6720636F6E666967202E2E2E0094
:10137000414320496E69740041432044652D496E04
:1013800069740045525200506F6C6C696E67004C76
:101390004F57004D454449554D0048494748004680
:1013A000414E5F4F4E4C59004452590048454154FC
:1013B00000434F4F4C004155544F0072617700710C
:1013C00075656974007377696E67006C6F636B0095
:1013D00044656661756C742073657269616C206D1B
:1013E0006F6465204E38312075736564003845316F
:1013F000002600384E31000600384532002E0038F5
:101400004E32000E00384F31003600384F32003E69
:1014100000374531002400374532002C00374F316A
:10142000003400374F32003C00374E3100040037A3
:101430004E32000C00203D3E002C002C002C002CD5
:1014400000456C657661746F723A20636F6E6669F1
:1014500067206661696C65643A00456C6576617405
:101460006F7220636F6E666967206572726F7200BB
:10147000456C657661746F7220636F6E6669672074
:101480006C6F616465642000456C657661746F7291
:101490003A204F7574206F66206D656D6F7279000C
:1014A000456C657661746F722044652D496E697470
:1014B00000403030525230303030303130303346EE
:1014C000303034313043303034322A004030305202
:1014D00052303030303032303037463030303231C8
:1014E00030303033302A00403030525230303030DB
:1014F00030343030334630303834313430303338B3
:101500002A003C003E00556E6B6E6F776E2073753F
:10151000666669782000556E6B6E6F776E20636D1E
:10152000642000536574206E6F7420696D706C6563
:101530006D656E74656400466F72636564206578DE
:1015400065637574696F6E00454C45563A20004DD1
:10155000756C746956656E7420636F6E666967207A
:101560006661696C6564004D756C746956656E746E
:1015700020696E6974004D756C746976656E7420AF
:1015800044652D496E697400204F75743A00206DD2
:1015900033002066726F6D2000204D6178207265E7
:1015A00071756573743A002066616E253A0020619A
:1015B000637469766520563A00546F74616C2056E6
:1015C0003A0020696E69740050574D2D4F75742094
:1015D00023002073746F700050574D2D4F75742089
:1015E00023002300524742575700524742570052A8
:1015F00047420050574D204368616E2074797065F2
:1016000020003D0050696E3A0020696E69740052F6
:10161000656C61792D4F75742023002073746F7091
:101620000052656C61792D4F75742023003D3E009A
:101630003A0070756220616374696F6E200069649E
:101640006C65006F66660068656174696E67006648
:10165000616E00647279696E6700636F6F6C696EAA
:10166000670020697320004F75742000556E6B6E03
:101670006F776E207375666669782000556E6B6EA5
:101680006F776E20636D642000616374696F6E0014
:1016900072656C61794374723A20005B305D3A2068
:1016A00000202D202D202D20EFBBBF003E003E311D
:1016B000202D200020002E00696E00735F6F75746E
:1016C000006D79686F6D6500202D3E2000456D69C5
:1016D000743A2000202D3E20004974656D436D64EE
:1016E0003A2000202D3E20004974656D3A20003ECE
:1016F0003E2000496E76616C696420636F6D6D6198
:101700006E64003E3E3E004E6F204D414320636FAD
:101710006E666967757265643A20736574206669E0
:10172000726D776172652773204D41430A004E6FD9
:101730002076616C696420454550524F4D206461AC
:1017400074612E20496E697469616C697A696E678B
:101750002E00476F74204950206164647265737372
:101760003A00276970205B69705B2C646E735B2C98
:1017700067775B2C7375626E65745D5D5D5D2720B8
:101780002D20736574207374617469632049500A55
:10179000004661696C656420746F20636F6E6669D2
:1017A000677572652045746865726E65742075731F
:1017B000696E6720444843502E20596F752063613D
:1017C0006E20736574206970206D616E75616C6C3C
:1017D0007921000A7573657320444843500A00203C
:1017E0004D41534B3A002047573A0020444E533A5C
:1017F000004C6F616465642066726F6D20666C6179
:1018000073682049503A005374617274696E67209E
:101810006C616E004142434445464748494A4B4C3F
:101820004D4E4F505152535455565758595A616264
:10183000636465666768696A6B6C6D6E6F70717200
:10184000737475767778797A303132333435363748
:1018500038392B2F3D004261736963200061726447
:1018600075696E6F3A004F544120696E6974696101
:101870006C697A65640A0044454641554C542070B1
:10188000617373776F726420666F72204F544120CA
:101890004150492E20557365206F74617077642024
:1018A000636F6D6D616E6420746F2073657400707A
:1018B000617373776F726400757074696D652C66FF
:1018C00072656568656170002473746174730035B6
:1018D0003232373138325F323032322D30312D30C2
:1018E00035004C696768744875622000246E616D2C
:1018F0006500726561647900546F6F206D616E7967
:10190000204D51545420636F6E6E656374696F6E21
:10191000206572726F72732E2052657374617274D7
:10192000204C414E002074727920616761696E20FD
:10193000696E2035207365636F6E6473006661693C
:101940006C65642C2072633D004177616974696E37
:101950006720666F722072657461696E65642074B9
:101960006F7069637300636F6E6E65637465642086
:1019700061732000202E2E2E0020757365723A00B0
:101980003A000A417474656D7074696E67204D5138
:10199000545420636F6E6E656374696F6E20746F4C
:1019A000200024737461746500646973636F6E6EE4
:1019B0006563746564005573696E67204D515454B6
:1019C0002070617373776F72642066726F6D20632D
:1019D0006F6E66696700446576696365204E616D68
:1019E000653A004174206C656173742064657669A2
:1019F0006365206E616D6520616E642062726F6B3D
:101A00006572204950206D75737420626520636F84
:101A10006E6669677572656400526562696E6420FE
:101A2000737563636573732E20495020616464721B
:101A30006573733A004572726F723A20726562691B
:101A40006E64206661696C0052656E65776564201E
:101A5000737563636573732E2049502061646472EB
:101A60006573733A004572726F723A2072656E65E3
:101A7000776564206661696C000A4E6F206C696E40
:101A80006B00526573746F72696E6720636F6E6668
:101A900069672066726F6D20454550524F4D004179
:101AA0006363657074696E6720636F6D6D616E64EA
:101AB000732E2E2E0A004E6F204D51545420636F0A
:101AC0006E66696775726564004C6F6164696E6704
:101AD00020636F6E6669672066726F6D20706F722B
:101AE00074616C2064697361626C65642E20757327
:101AF0006520676574204F4E20746F20656E6162AB
:101B00006C6500436F6E6669672069732076616C4F
:101B1000696400436F6E74696E75652077697468D7
:101B20002070726576696F75736C79206C6F616473
:101B3000656420636F6E6669670000002100240001
:101B400027002A002D0030003300010100000401AD
:101B500007010A0100002200250028002B002E00AA
:101B60003100340002010000050108010B010505E8
:101B70000505070508080808020202020A0A080803
:101B80000404040401010101010101010303030331
:101B900003030303040707070C0C0C0C0C0C0C0CC0
:101BA0000202020206060606060606060B0B0B0BD1
:101BB0000B0B0B0B050505080807070404040A0AAC
:101BC0000A0A0A0A010210202008081020401020EA
:101BD00040800201020108040201010204081020F1
:101BE00040808040201008040201800402018040EF
:101BF0002010080402010804020101020408102058
:101C000040800102040810204080044080048008C5
:101C10001010204004081020408000000B0C030A24
:101C20000D0E0F090804050200000000000000006E
:101C300000000000000000000000000000000000A4
:101C4000000000000000131211000000000000005E
:101C50000000000000000000000000000000000084
:101C60000000000000000000000000000000000074
:101C70002F64617461002F736B6574636800416346
:101C8000636573732D436F6E74726F6C2D52657143
:101C9000756573742D507269766174652D4E657427
:101CA000776F726B3A207472756500416363657378
:101CB000732D436F6E74726F6C2D416C6C6F772D4A
:101CC000486561646572733A202A004163636573F5
:101CD000732D436F6E74726F6C2D416C6C6F772D2A
:101CE0004D6574686F64733A20504F53542C4745C8
:101CF000542C4F5054494F4E5300416363657373E6
:101D00002D436F6E74726F6C2D416C6C6F772D4329
:101D1000726564656E7469616C733A20747275657E
:101D2000004F5054494F4E530044454C45544500D4
:101D30005055540047455400504F5354006175743A
:101D4000686F72697A6174696F6E3A2000417574C8
:101D5000686F72697A6174696F6E3A2000436F6EC2
:101D600074656E742D4C656E6774683A20006F63FD
:101D70007465742F73747265616D00696D61676558
:101D80002F6A70656700696D6167652F6769660016
:101D9000746578742F68746D6C006170706C696321
:101DA0006174696F6E2F6A736F6E00746578742F3B
:101DB000706C61696E00436F6E74656E742D54793A
:101DC00070653A2000436F6E6E656374696F6E3A9A
:101DD00020636C6F7365004163636573732D436F9C
:101DE0006E74726F6C2D416C6C6F772D4F726967DA
:101DF000696E3A20687474703A2F2F6C617A796832
:101E00006F6D652E727500556E6B6E6F776E004E3E
:101E10006F74204D6F646966696564004F4B004DB7
:101E20006F766564207065726D616E656E746C7935
:101E300000496E7465726E616C20536572766572CE
:101E4000204572726F72005061796C6F616420542A
:101E50006F6F204C61726765004E6F7420666F75FE
:101E60006E64005757572D41757468656E746963C9
:101E70006174653A204261736963207265616C6DBB
:101E80003D22416363657373207265737472696385
:101E90007465642200556E617574686F72697A6545
:101EA00064005061796C6F61642073697A65207792
:101EB000726F6E670042616420726571756573743C
:101EC00000485454502F312E3120002000000000D3
:101ED0000000000000004F4E000000000000004F16
:101EE0004646000000000000524553540000000028
:101EF00000544F47474C4500000048414C540000F7
:101F0000000000584F4E000000000000584F4646A9
:101F10000000000000494E435245415345004445EE
:101F200043524541534500484541540000000000DC
:101F3000434F4F4C00000000004155544F0000003B
:101F4000000046414E5F4F4E4C590044525900002C
:101F50000000000053544F50000000000048494763
:101F60004800000000004D454449554D0000004C1C
:101F70004F5700000000000054525545000000007B
:101F80000046414C534500000000454E41424C453F
:101F900044000044495341424C45440052474200EA
:101FA0000000000000485356000000000000202DF3
:101FB0003E2041543A004368616E20747970653A5E
:101FC000004E6F2073746F7265642076616C756566
:101FD00073202D2064656661756C743A200053612E
:101FE00076656420455441473A0053657420455452
:101FF00041473A20000057C035C011241FBECFEF23
:10200000D1E2DEBFCDBF00E00CBF16E0A0E0B2E041
:10201000E0E0FBEA01E00BBF02C007900D92A23D99
:10202000B107D9F720E1A2EDB6E001C01D92A635B7
:10203000B207E1F71FE0CCEFDFE000E006C0219738
:102040000109802FFE010E9436D0CB3FD10780E0EE
:102050000807A9F70E94E7AF0C946ED50C94000016
:10206000CF93DF931F92CDB7DEB76983DC01ED918B
:10207000FC910280F381E02D41E050E0BE016F5FF2
:102080007F4F19950F90DF91CF910895FC01818DBD
:10209000928D0895CF93DF931F92CDB7DEB76983FA
:1020A000DC01ED91FC910280F381E02D41E050E0F4
:1020B000BE016F5F7F4F19950F90DF91CF9108950B
:1020C000FC019485FB018485981303C081E098305E
:1020D00008F080E00895CF93DF931F92CDB7DEB76D
:1020E0006983DC01ED91FC910280F381E02D41E0F8
:1020F00050E0BE016F5F7F4F19950F90DF91CF9138
:10210000089585ED8093BC008091BC0084FDFCCFD8
:1021100010925A08089520913608260F3327331F4E
:1021200021323105ECF420915A08FC0190E080E066
:10213000243069F082E00895A09136082191AC0125
:102140004A5E574FA40FB52FB11D2C9301968617E9
:1021500098F380913608680F6093360880E0089500
:1021600081E008958FEF9FEF08958FEF9FEF08951F
:102170008091150890E09195819591090895CF93EC
:10218000DF93CB01EA01642F0E948B10CE01DF9117
:10219000CF910895CF93DF931F92CDB7DEB76983B8
:1021A00061E0CE0101960E948B1081E090E00F90DB
:1021B000DF91CF9108958F929F92AF92BF92CF926D
:1021C000DF92EF92FF920F931F93CF93DF9300D094
:1021D00000D000D01F921F92CDB7DEB77C018E01D8
:1021E0000F5F1F4F68018AE0882E912CA12CB12C23
:1021F000C601801B910B411551056105710581F0E8
:10220000CB01BA01A50194010E94ABCF942F852F79
:10221000605DF60161936F01A901692F782FE8CF06
:10222000F801E80FF91FD7010150110922912D93F0
:10223000E017F107D9F7E80EF91EF70110822B9687
:102240000FB6F894DEBF0FBECDBFDF91CF911F91C7
:102250000F91FF90EF90DF90CF90BF90AF909F9045
:102260008F900895FC01DC018D918111FDCF30E04C
:1022700020E050E040E08AE09191992301F1443060
:1022800051055CF59E3271F42F3F310509F02CF5B4
:10229000DB01A40FB51F12962C934F5F5F4F30E008
:1022A00020E0EACF829FD001839FB00D1124292F17
:1022B000990F330B205331092A0F3B1FDDCF2F3FDE
:1022C000310509F054F4443051053CF4640F751F96
:1022D000FB01228381E090E0089590E080E0089582
:1022E000CF93DF931F921F92CDB7DEB780914A1034
:1022F00090914B10009711F486E590E1BE016F5F5D
:102300007F4F681B790B072E000C880B990B0F90E1
:102310000F90DF91CF910895DC0115968D919C91DE
:10232000009739F0DC01ED91FC910680F781E02DFA
:1023300019940895089583E090E0089590E0FC01D9
:10234000E259F44EE491F0E0EE0FFF1FEC5AF44E28
:10235000A591B4912C918C53944EFC0184918223CD
:1023600091E009F490E0892F08958091BD07909144
:10237000BE070895089590E080E008958091BB071E
:102380009091BC07089508958091B9079091BA077C
:10239000089584E090E00895DC011496ED91FC919D
:1023A000309729F08081082E000C990B089590E059
:1023B00080E008950895809102079091030781704D
:1023C000992708958091F1069091F2060895FC01F5
:1023D000848195810895FC01768765870895DC01E5
:1023E000ED91FC91068CF78DE02D199591E08927F0
:1023F0000895862F089581E08627089521E0FC0145
:102400008485883008F020E0822F0895FC018485BF
:1024100095850895FC0184899589089529E234E021
:10242000FC0131832083FB014089518962897389D2
:10243000FC0142835383648375830895DC01ED912D
:10244000FC91048CF58DE02D1994CF93DF9300D08F
:1024500000D01F921F92CDB7DEB7FC016F3F710510
:1024600019F014F06FEF70E077FD60E09181892F33
:1024700082958F7081508230C8F4648388E0DE01D9
:10248000119601900D928A95E1F729813A814B814D
:102490005C816D817E818F81988528960FB6F89436
:1024A000DEBF0FBECDBFDF91CF9108959F709061C9
:1024B0009183E3CF0F931F93CF93DF93DC01C62F5C
:1024C0001196EC911197E295EF70EC3008F0BCC0DA
:1024D000F0E08827E159FD4E8F4F0C9436D07B12E7
:1024E000A012A0122413241324130213AC122413D9
:1024F00024138312831270E060E0CB01DF91CF914F
:102500001F910F91089514968D919D910D90BC91FE
:10251000A02D8F3F9105A105B10529F024F08FEF83
:1025200090E0A0E0B0E0B7FF03C080E090E0DC0105
:102530006FEF70E0681B790BC111DFCFBC01DDCFFD
:1025400014966C9170E0CC23C1F28FEF90E09C0167
:10255000261B370BB901D1CF862F14960C911497F7
:1025600015961C9115971696DC9116971796CC9197
:1025700020E030E0A901B801882331F18D2F9C2F94
:102580000E9461CE87FD1BC020E030E04FE753E49E
:10259000B8018D2F9C2F0E9469D1181624F400E0F9
:1025A00010E0DFE7C3E498014D2F5C2F60E070E09E
:1025B0008FE793E40E9454D00E9433D19ECF00E075
:1025C00010E0D0E0C0E0EFCF8D2F9C2F0E9461CEB5
:1025D00087FD13C020E030E04FE753E4B8018D2FB2
:1025E0009C2F0E9469D1181624F400E010E0DFE768
:1025F000C3E4B8018D2F9C2FDFCF00E010E0D0E0C6
:10260000C0E0F7CF14966D917D918D919C911797B5
:102610002AE030E040E050E00E94CDCF2F3F31056E
:102620004105510529F024F02FEF30E040E050E063
:1026300057FF03C020E030E0A9016FEF70E0621B9C
:10264000730BC1115ACF86CF6FEF7FEF56CFDC01EE
:102650001196EC911197E295EF70E150EB3008F094
:1026600039C0F0E08827E85CFC4E8F4F0C9436D0E0
:102670005B135B136A13431343134C13631363130A
:1026800063134313431314966D917D918D919C9127
:1026900017970E9468CE089514966D917D918D9143
:1026A0009C9117972AE030E040E050E00E94CDCFA7
:1026B000CA01B901EECF14966C9170E090E080E011
:1026C0000E9466CE089514966D917D918D919C9196
:1026D0001797089560E070E0CB010895FC01A78191
:1026E0002A2F2E7FD1F0818182958F708150833087
:1026F000A0F4A695A150BB0B2BE531E00E944DD074
:1027000024E630E040E050E00E94CDCFDA01C9017C
:1027100087569F4FAF4FBF4F08958FEF9FEF08959C
:10272000DC01ED91FC91309729F090859F7081E05C
:10273000953009F080E00895DC011496ED91FC914C
:102740001597309799F090859F708EEF890F8230A2
:1027500010F091110BC041875287638774871496DC
:10276000ED91FC918085807F826080870895DC01F7
:1027700019968D919C91009739F0DC01ED91FC91B7
:102780000280F381E02D199408958AE090E0089585
:1027900081E090E0089588E090E00895DC01ED91FB
:1027A000FC91008CF18DE02D1994CF93DF93EC0117
:1027B000E881F9810484F585E02D199529893A8904
:1027C0002F5F3F4F3A8B298BDF91CF910895CF93A5
:1027D000DF93EC018E8581110DC081E090E0498985
:1027E0005A892C853D854217530708F080E0DF9118
:1027F000CF910895E881F9810484F585E02DCE011B
:1028000019958F3F910549F780E090E0F0CFFC01EA
:10281000848595856817790708F4CB01928B818BA5
:102820000895DC011E962C911E97222339F0ED911C
:10283000FC910190F081E02D6FEF19940895FC0157
:1028400087859089089581E0089590E080E008955B
:10285000FC0122813381232B49F0868197818130CD
:10286000910539F01CF00397039730F090E080E079
:10287000089581E090E0089582E090E00895CF937C
:10288000DF93CDB7DEB760970FB6F894DEBF0FBE0B
:10289000CDBF19821A821B821C821D821E821F825A
:1028A00018868A818F708A836FEF70E0CE0101965F
:1028B0000E94251260960FB6F894DEBF0FBECDBF02
:1028C000DF91CF910895CF92DF92EF92FF920F9315
:1028D0001F93CF93DF93CDB7DEB760970FB6F89411
:1028E000DEBF0FBECDBF7C016B01BA01A901CE01D5
:1028F00001960E94DB10D701ED91FC910288F389CB
:10290000E02D9801AE014F5F5F4FB601C7011995E9
:1029100060960FB6F894DEBF0FBECDBFDF91CF91AA
:102920001F910F91FF90EF90DF90CF900895CF927D
:10293000DF92EF92FF920F931F93CF93DF9300D01C
:1029400000D0CDB7DEB78C016B017A01FC01808D20
:10295000883010F40E945D9089E294E09A83898324
:10296000F60182819381A481B5818B839C83AD83A1
:10297000BE83B701CE0101960E949A9FF801808F15
:102980008830A0F4F586E486128E118E81E02696BA
:102990000FB6F894DEBF0FBECDBFDF91CF911F9170
:1029A0000F91FF90EF90DF90CF90089580E0EFCFF0
:1029B000CF93DF93EC01888D883020F40E945D90E6
:1029C00088E0888FDF91CF910895FC01808D883059
:1029D00040F4218D328D232B21F00E942F8F90E027
:1029E00008958FEF9FEF0895CF93DF93FC01248527
:1029F000283028F08FEF9FEFDF91CF910895EC0101
:102A00000190F081E02D0084F185E02D1995892B4E
:102A100089F38C850E942F8F90E0EECFCF93DF93C8
:102A2000FC01218D328D2115310529F48FEF9FEFA7
:102A3000DF91CF910895EC01808D4217530708F084
:102A4000A9010E947E8F1816190684F7298D3A8DE8
:102A5000281B390B3A8F298FEBCF0F931F93CF93FE
:102A6000DF931F92CDB7DEB7FC01218D328D232B72
:102A700041F48FEF9FEF0F90DF91CF911F910F9156
:102A800008958C0141E050E0BE016F5F7F4FFC0173
:102A9000808D0E947E8F181619065CF7F801818DD3
:102AA000928D0197928F818F898190E0E4CFCF93AF
:102AB000DF931F92CDB7DEB741E050E0BE016F5FFC
:102AC0007F4FFC0184850E947E8F1816190634F40E
:102AD000898190E00F90DF91CF9108958FEF9FEF64
:102AE000F9CFFC018485883010F40C947E8F90E03F
:102AF00080E00895FC018485883010F40C94578F91
:102B000090E080E008950F931F93CF93DF9300D060
:102B100000D01F921F92CDB7DEB78C01D801599615
:102B20004D915C915A974115510551F0ED91FC91F1
:102B3000048CF58DE02D70E060E0C8011995EECFB2
:102B4000F801808D0E94578F892BB1F148E050E049
:102B5000BE016F5F7F4FD80158968C910E947E8F87
:102B600018161906F4F4D801509684E0FE01319647
:102B700001900D928A95E1F78D8190E0982F88273A
:102B80002E81820F911DF801958B848B8F81282FC8
:102B900030E0322F22278885820F932F911D928F4C
:102BA000818F28960FB6F894DEBF0FBECDBFDF91A0
:102BB000CF911F910F91089590E080E0F2CFCF92D6
:102BC000DF92EF92FF920F931F93CF93DF93CDB7D6
:102BD000DEB7AF970FB6F894DEBF0FBECDBF7C0156
:102BE0006A0109E214E01A8309831C861B8688EEB9
:102BF00093E0A0E0B0E08D879E87AF87B88B8FEF22
:102C000093E09A878987188F0F8B198E1A8E1B8EE7
:102C10001C8E88E089A31BA70AA71CA61DA61EA6BA
:102C20001FA680915A0D90915B0DA0915C0DB09103
:102C30005D0D8EA39FA3A8A7B9A78B839C83AD83AB
:102C4000BE8318861F82AE01465D5F4FCE0101969E
:102C50000E9490A581309105B1F4D701ED91FC91CE
:102C60000488F589E02D1DA30CA38CA59DA5AEA518
:102C7000BFA58EA39FA3A8A7B9A7A601BE016C5D9F
:102C80007F4FC7011995AF960FB6F894DEBF0FBE00
:102C9000CDBFDF91CF911F910F91FF90EF90DF900B
:102CA000CF9008950F931F93CF93DF93EC018B0187
:102CB000888D883010F40E945D90B80182E00E94F7
:102CC000A690888F883050F41D870C871A8E198E35
:102CD00081E0DF91CF911F910F91089580E0F9CFAE
:102CE0000F931F93CF93DF938C01EA01FC0184853E
:102CF000883048F40E94CD8E892B39F481E090E031
:102D0000F80193838283D0E0C0E0CE01DF91CF91C0
:102D10001F910F910895EF92FF920F931F93CF93FE
:102D2000DF937C018091C909D4E0833309F0D8E0B6
:102D300009EB19E0C0E0F801219131918F01F70111
:102D4000848195812817390729F0CF5FDC13F3CFF1
:102D500080E006C08C2F0E946B908431B1F781E037
:102D6000DF91CF911F910F91FF90EF900895CF9336
:102D7000DF93EC018C858830D0F40E946B90843115
:102D800089F0882379F0883169F021E08C3159F499
:102D9000E881F9810084F185E02DCE01199521E0CB
:102DA000892B09F420E0822FDF91CF91089580E0F4
:102DB000FBCFCF92DF92EF92FF920F931F93CF93AF
:102DC000DF93CDB7DEB7AF970FB6F894DEBF0FBE77
:102DD000CDBF8C016B017A0189E294E09A838983EB
:102DE0001B821C821D821E821C861B8648EE53E0BD
:102DF00060E070E04D875E876F87788B2FEF33E060
:102E00003A872987988F8F8B198E1A8E1B8E1C8E6E
:102E100028E029A39BA78AA71CA61DA61EA61FA65D
:102E2000D8011C968C91883060F40E946B908823A6
:102E300021F0F80184850E944F9088E0D8011C960B
:102E40008C9380915A0D90915B0DA0915C0DB09187
:102E50005D0D8EA39FA3A8A7B9A78B839C83AD8389
:102E6000BE8318861F82AE01465D5F4FB601CE015C
:102E700001960E9490A50097C1F0D801ED91FC91B8
:102E80000684F785E02D89E294E09DA38CA38CA5B0
:102E90009DA5AEA5BFA58EA39FA3A8A7B9A7A7016F
:102EA000BE016C5D7F4FC8011995AF960FB6F894BF
:102EB000DEBF0FBECDBFDF91CF911F910F91FF906D
:102EC000EF90DF90CF900895CF93C82F0E949DA2DE
:102ED00004C09695879577956795CA95D2F7611541
:102EE00071058105910521F461E070E080E090E0DA
:102EF000CF910895CF93DF93EC018C85883060F4F7
:102F00000E946B90873111F08C3131F48C850E94D6
:102F1000B08E8115984088F3DF91CF910895FC0120
:102F20008485883010F40C94B08E90E080E0089591
:102F300066E775E185E19FE00E94958285E19FE06B
:102F40000E949E811092BA071092B90781E090E02A
:102F5000089568E773E185E19FE00E94958285E12D
:102F60009FE00E949E811092F2061092F10681E08D
:102F700090E0089560E67FE0811102C062E67FE0A4
:102F800084EE9DE00C94958265E97DE084EE9DE001
:102F90000E949582F0E0E0E0199584EF91E00895B9
:102FA00063EC78E0811102C06EEB78E085E19FE090
:102FB0000C9495824F925F926F927F92AF92BF92E4
:102FC000DF92EF92FF920F931F93CF93DF9300D086
:102FD00000D0CDB7DEB77C01D62E809111088823B2
:102FE00009F4BEC0D70114969C9180912A028917DA
:102FF00008F4B6C080910F0890911008BAE06B13E6
:10300000F0C08154984FFC011082D70118960D91A1
:103010001C910115110509F49FC0F80161857285A5
:103020006115710591F445805680678070848091A8
:10303000540D9091550DA091560DB091570D481615
:1030400059066A067B0609F487C0D8011B964D9184
:103050005C911C974115510509F47EC0F70124814C
:1030600053968C91539790E0322F377002C095950C
:1030700087953A95E2F780FF6FC0A22EB12CC5016B
:10308000887F9370892B39F451968D919C91887F1C
:103090009370A82AB92AD8018D919C91DC01ED91F9
:1030A000FC916115710509F486C00688F789E02D49
:1030B0001995019709F050C06CE3F8018081918166
:1030C0000E94A281A50170E060E02AE0D8018D9104
:1030D0009C910E945281F8012281808191816EEA47
:1030E00076E1222311F06CEA76E10E949582D80104
:1030F0001D966D917C911E978D919C910E942F82BF
:1031000060E2F801808191810E94A281D8011F961E
:103110006D917C9150978D919C910E942F82F80126
:1031200022818081918161EA76E1222311F06BE9AD
:1031300076E10E9495826FEB77E0D8018D919C91AA
:103140000E942F82F80180819181DC01ED91FC9138
:10315000008CF18DE02D19951092100810920F0837
:10316000D70115968D919C911697009709F44DC043
:1031700014963C9120912B02231708F446C0DC01E1
:10318000ED91FC910190F081E02D6D2D1995269621
:103190000FB6F894DEBF0FBECDBFDF91CF911F9168
:1031A0000F91FF90EF90DF90BF90AF907F906F9066
:1031B0005F904F9008950488F589E02D29E234E06E
:1031C0003A832983D80115964D905D906D907C903F
:1031D00018974B825C826D827E82BE016F5F7F4F4B
:1031E00067CF8F3491050CF0BBCFBDE06B1709F4AE
:1031F000B7CF9C012F5F3F4F3093100820930F08EB
:103200008154984FFC016083ABCF81E090E0BFCF49
:103210000C9465C40C9465C40C9465C40C9465C48A
:103220000C9465C4CF93DF93FC0122813381232B5F
:1032300009F450C0EC0163EF75E185E19FE00E9465
:1032400095828E819F8184309105A1F08530910512
:10325000F1F0039749F56FEE75E185E19FE00E947B
:10326000958285E19FE00E949E8182E090E0DF915F
:10327000CF9108956AEE75E185E19FE00E94958205
:1032800085E19FE00E949E8181E090E0F0CF64EEB6
:1032900075E185E19FE00E94958285E19FE00E94B3
:1032A0009E8181E190E0E3CF62EE75E185E19FE0F0
:1032B0000E949582EA81FB81608585E19FE00E9402
:1032C000579585E19FE00E949E81EA81FB81808580
:1032D00090E0CDCF90E080E0CACFCF93C1E068EE20
:1032E00073E080E090E00E946BA26C2F84EE9DE082
:1032F0000E945795CF5FC43191F784EF91E0CF9151
:103300000895CF93DF93009709F484C0FC012081D6
:10331000222309F47FC0EC0167E579E00E9401C730
:10332000892B09F456C06BE379E0CE010E9401C7F6
:10333000892B09F451C06FE077E0CE010E9401C7EC
:10334000892B09F44CC06BE077E0CE010E9401C7E5
:10335000892B09F447C067E077E0CE010E9401C7DE
:10336000892B09F442C063E077E0CE010E9401C7D7
:10337000892BF1F16FEF76E0CE010E9401C7892B16
:10338000D1F16BEF76E0CE010E9401C7892BB1F13C
:1033900066EF76E0CE010E9401C7892B91F162EFC2
:1033A00076E0CE010E9401C7892B71F16BE579E0CF
:1033B000CE010E9401C7892B51F16EEE76E0CE015D
:1033C0000E9401C7892B31F58EE090E0DF91CF910B
:1033D000089582E090E0FACF81E090E0F7CF88E0B6
:1033E00090E0F4CF85E090E0F1CF86E090E0EECF82
:1033F00087E090E0EBCF89E090E0E8CF8AE090E0D2
:10340000E5CF8BE090E0E2CF8CE090E0DFCF8DE085
:1034100090E0DCCF90E080E0D9CFCF93DF93EC0158
:1034200061E276E185E19FE00E9495826C817D8179
:1034300085E19FE00E945E956BE176E185E19FE08A
:103440000E94958285E19FE00E949E8160E08C81D0
:103450000E9413A11092BE071092BD0781E090E078
:10346000DF91CF910895EF92FF921F93CF93DF9357
:10347000192F7B01C82FD92FD7FF03C0D195C19534
:10348000D10961E08C2F0E9413A182E0E816F104BB
:1034900099F460E08C2F0E94E5A060E672E185E17E
:1034A0009FE00E94958285E19FE0DF91CF911F917F
:1034B000FF90EF900C949E81612FEF2851F460955E
:1034C000661F6627661F8C2F0E94E5A06CE572E1DF
:1034D000E6CF661F6627661F8C2F0E94E5A067E572
:1034E00072E1DDCFCF93DF93EC01FB0124813581C5
:1034F00040815181628173810E94A981CE01DF9157
:10350000CF910895EF92FF920F931F93CF93DF9384
:10351000EC018B011D821C821A821B82E880F980DB
:10352000E114F10409F459C08091EC069091ED0684
:10353000892B09F452C0672B09F48701F8018085B3
:103540008F708630A9F467E374E0C8010E94D594B7
:10355000009719F0FC0181858A8363EC76E0C8014D
:103560000E94D594009709F43FC0FC0181858B83AC
:1035700069E374E0C7010E94D594009759F566EAA3
:1035800076E085E19FE00E9495826B8185E19FE076
:103590000E94579564EA76E085E19FE00E9495825B
:1035A0006A8185E19FE00E94579585E19FE00E9436
:1035B0009E8120E030E0A90169E374E0888199816F
:1035C0000E94919969E374E0888199810E94D59461
:1035D000009719F009969D838C83DF91CF911F91FD
:1035E0000F91FF90EF900895F801808191810E94E2
:1035F00095C6BDCF0F931F93CF93DF938C01EB0143
:103600002197AE01BC018CED99E00E94E277F801B0
:10361000329660E0CF01801B910B8C179D0718F448
:103620008191680FF7CF8CED99E0DF91CF911F91D9
:103630000F910C94AF78CF93DF9300D000D01F92FE
:103640001F92CDB7DEB7EFECFDE0128A118A80E061
:1036500090E19587848784E890E0948B838B81E068
:10366000868780E090E2908B87871C821B8282E2B3
:1036700093E09A838983FE83ED838FEF9FEF988792
:103680008F8363EE72E184EE9DE00E9495826091EB
:10369000EC067091ED06CE0101960E9499888FECA0
:1036A0009DE00E94CE1363ED72E184EE9DE00E94E6
:1036B000958284EE9DE00E949E810E943FA82896FC
:1036C0000FB6F894DEBF0FBECDBFDF91CF91089546
:1036D000FC0186819781009799F0FC0120852F706D
:1036E000223029F46185728583859485089525307B
:1036F00039F460E00E944A95009711F0FC01F2CF86
:1037000060E070E0CB0108950F931F93CF93DF9398
:10371000FC01C281D3812097F9F088858F708230B7
:1037200049F4672BC9F489859A85DF91CF911F9160
:103730000F910895853081F48B01CE010E9466952A
:103740008017110649F044F0602FCE010E944A957F
:10375000FC0181859285E9CF90E080E0E6CFFC0115
:103760006115710519F48481958108958681978189
:10377000681779072CF084819581860F971F08952B
:10378000828193810C94841BCF93DF93EC0168EDCD
:1037900075E185E19FE00E9495826C817D8185E1E4
:1037A0009FE00E945E9562ED75E185E19FE00E94D9
:1037B000958285E19FE00E949E81E881F981028CDB
:1037C000F38DE02DCE0119958130910529F00297F6
:1037D00059F060E08C811AC063E070E0CE010E9475
:1037E000AF1B60E00E9413A160E08C810E9413A1D6
:1037F00061E070E0CE010E94AF1B60E00E9413A167
:1038000062E070E0CE010E94AF1B60E00E9413A155
:103810001092BC071092BB0781E090E0DF91CF913E
:103820000895CF93DF93EB0163E0FC0180819181E8
:103830000E944A95FC01892BA9F080858D7091F436
:10384000C095D095CF6FAE0170E060E08185928524
:10385000A385B4858C239523A623B72381879287DC
:10386000A387B487DF91CF910895CF93DF93EB01C6
:1038700063E0FC01808191810E944A95FC01892BC3
:10388000B9F09085892F8D7099F4907F9260908720
:10389000CC27CE01B0E0A0E04185528563857485D8
:1038A000842B952BA62BB72B81879287A387B48770
:1038B000DF91CF910895CF93DF93EB0163E0FC019B
:1038C000808191810E944A95009761F0FC012085DA
:1038D0002F70223039F4818592858C239D23DF91CE
:1038E000CF91089590E080E0FACFCF93C62F63E0A8
:1038F000FC01808191810E944A95FC01892B19F17C
:103900009085892F8D70F9F4907F926090878185E2
:103910009285A385B4858827AA27BB278C2B81870E
:103920009287A387B48764E177E085E19FE00E94F6
:1039300095826C2F85E19FE00E94579585E19FE07D
:10394000CF910C949E81CF91089563E0FC0180811A
:1039500091810E944A95009719F0FC018185089594
:103960008FEF0895FF920F931F93CF93DF93CDB7FF
:10397000DEB764970FB6F894DEBF0FBECDBF8C01E3
:10398000F62E8FE290E09A838983FE01339688E0D9
:10399000DF011D928A95E9F7F8016681FF2011F099
:1039A00081E06827D80114968C910E94E5A0F80167
:1039B00087819085A185B285883E9340A105B10598
:1039C00008F48BC067E676E185E19FE00E9495826E
:1039D000D80114966D917C9185E19FE00E945E95DF
:1039E00062E676E185E19FE00E9495826F2D70E0AE
:1039F00085E19FE00E945E9585E19FE00E949E81A7
:103A000069E876E1CE0101960E94F6C6F80182814E
:103A100093810E94A51CFF2009F46BC06FE476E13E
:103A20008D3051F063E576E18E3031F06AE576E174
:103A30008B3011F067E476E1CE010B960E940AC745
:103A400062E376E185E19FE00E949582D8011296BB
:103A5000ED91FC9113970190F081E02D60817181CF
:103A6000ED91FC910288F389E02D9E012F5F3F4F7D
:103A7000AE01455F5F4FC8011995BC0185E19FE02C
:103A80000E945E9560E376E185E19FE00E94958269
:103A9000D8011296ED91FC910190F081E02D6081AA
:103AA000718185E19FE00E942F82BE016F5F7F4F91
:103AB00085E19FE00E942F826DE276E185E19FE043
:103AC0000E949582BE01655F7F4F85E19FE00E9465
:103AD0002F8285E19FE00E949E8164960FB6F89444
:103AE000DEBF0FBECDBFDF91CF911F910F91FF9031
:103AF000089563E476E1823009F49ECF6EE376E1C7
:103B00009BCF81E090E00895CF93DF93EC0168ECC8
:103B100075E185E19FE00E9495826C817D8185E160
:103B20009FE00E945E9562EC75E185E19FE00E9456
:103B3000958285E19FE00E949E818A819B81892BED
:103B400009F44DC08C819D81892B09F048C0E88122
:103B5000F981028CF38DE02DCE011995813091050C
:103B600029F0029759F061E08C811AC063E070E09F
:103B7000CE010E94AF1B61E00E9413A161E08C8125
:103B80000E9413A161E070E0CE010E94AF1B61E0D2
:103B90000E9413A162E070E0CE010E94AF1B61E0C1
:103BA0000E9413A18091A100887F8093A100809141
:103BB0009100887F809391008091A1008260809322
:103BC000A1008091910082608093910081E090E05B
:103BD0009093BC078093BB07DF91CF91089590E04D
:103BE00080E0FACFCF93DF93DC011496ED91FC9146
:103BF000309709F44FC0C681D7812097C1F1E88181
:103C0000F981309781F18081882369F165EC74E056
:103C1000CE010E94D594892B41F42FEF3FEFA901EB
:103C200065EC74E0CE010E94919966ED74E0CE01DE
:103C30000E94D594892B41F42FEF3FEFA90166ED47
:103C400074E0CE010E9491996CE374E0CE010E9471
:103C5000D594892B41F42FEF3FEFA9016CE374E079
:103C6000CE010E9491990A80DB81C02DC6CF67E604
:103C700075E185E19FE00E94958285E19FE00E94C9
:103C80009E8181E090E09093BA078093B907DF911D
:103C9000CF9108956FE475E185E19FE00E949582E0
:103CA00085E19FE00E949E8190E080E0F0CF60E798
:103CB00073E185E19FE00E94958285E19FE00E948B
:103CC0009E8126E040E855E260E070E08CED99E0EE
:103CD0000E944C8781E090E09093F2068093F10679
:103CE0000895892B71F0FB01828193810E94839654
:103CF00069ED7EE084EE9DE00E94958288EC90E084
:103D0000089590E080E0F2CF892B71F0FB01828171
:103D100093810E94209662EC7EE084EE9DE00E94FA
:103D2000958288EC90E0089590E080E0F2CF809159
:103D3000C10D9091C20D892B51F00E9469A9882371
:103D400031F062EB7EE084EE9DE00E94958210925D
:103D5000E10D1092E00D80E090E19093DC0D8093F6
:103D6000DB0D84E890E09093E30D8093E20D81E019
:103D70008093DD0D80E090E29093DF0D8093DE0D67
:103D80008FEC9DE00E9411148FEC9DE00E94CE13F9
:103D900088EC90E00895EF92FF920F931F93CF93DA
:103DA000DF93CDB7DEB72C970FB6F894DEBF0FBE0A
:103DB000CDBF8C017B0189E294E09A8389831B82C9
:103DC0001C821D821E8298878F8319861A861B8605
:103DD0001C8605301105ECF0BE01695F7F4FF701CD
:103DE000808591850E943211892B99F0CE0107962A
:103DF0000E945197BE01695F7F4FF70186819781CD
:103E00000E943211892B61F0CE0107960E942798FB
:103E10000EC0CE0101960E9451970430110554F74F
:103E2000CE0101960E942798033011058CF1BE0146
:103E3000695F7F4FF701848195810E943211892B40
:103E400039F1CE0107960E94BC97BE01695F7F4F92
:103E5000F701828193810E943211892B01F1CE01F9
:103E600007960E94E6966BE97EE084EE9DE00E9454
:103E7000958288EC90E02C960FB6F894DEBF0FBECA
:103E8000CDBFDF91CF911F910F91FF90EF900895DB
:103E9000CE0101960E94BC9702301105B4F6CE0106
:103EA00001960E94E69601301105E9F6CE010196D1
:103EB0000E94E69662EA7EE084EE9DE00E94958292
:103EC000D2CF0F931F93CF93DF938C01EB01029717
:103ED000C4F08A819B810E9495C680932B0299270A
:103EE0000E945F990230110549F08C819D810E94EA
:103EF00095C680932A0299270E946999C8ECD0E060
:103F000002C0C0E9D1E067E87EE084EE9DE00E9457
:103F1000958260912B0284EE9DE00E94579562E7A6
:103F20007EE084EE9DE00E94958260912A0284EEFC
:103F30009DE00E94579584EE9DE00E949E81CE01F7
:103F4000DF91CF911F910F910895CF93DF93EB01F4
:103F50000297A4F16DE57FE08A819B810E94E3C610
:103F6000892B29F40E9492986F770E94EF9869E557
:103F70007FE08A819B810E94E3C6892B29F40E94FD
:103F8000929860680E94EF9861E67EE084EE9DE082
:103F90000E9495820E9492986095661F6627661F10
:103FA00070E084EE9DE00E945E9584EE9DE00E94AC
:103FB0009E8188EC90E0DF91CF9108950E941B1BB9
:103FC000F8CF2F923F924F925F926F927F928F9293
:103FD0009F92AF92BF92CF92DF92EF92FF920F9398
:103FE000CF93DF9300D01F92CDB7DEB77C017A83E9
:103FF00069835C834B83DB011C92FC016081662337
:1040000009F4C2C130FFC0C1F9E06F9FB0011124B3
:104010006353714ECD010E9438C74B815C8160E4CF
:1040200074E089819A810E94A7D4E981FA81019084
:104030000020E9F7319789819A81E81BF90B1C016F
:104040002E0E3F1EAB81BC81AE1BBF0B1197BC83F4
:10405000AB83D7011196EC91E295EF70E150EC3013
:1040600008F0B3C0F0E08827E75CFF4D8F4F0C9459
:1040700036D04520B4201A2181219D218120312173
:104080003121312175206920BA21F7018481282F3F
:1040900030E050E040E0002359F030E0A4E6B0E02A
:1040A0000E94FFCF2FEF30E040E050E00E94CDCFE4
:1040B0005F934F933F932F9382E494E09F938F936A
:1040C000FC81FF938B818F933F922F920E94DFD4CC
:1040D00077C0F70187818F9386818F9385818F9336
:1040E00084818F9385E494E0E9CFF70187818F93F2
:1040F00086818F9385818F9384818F9389E494E067
:10410000DDCFF701C480D580E680F780C701B60116
:104110002AE030E040E050E00E94CDCF97FF07C09A
:1041200090958095709561957F4F8F4F9F4F9F938E
:104130008F937F936F93C701B6012AE030E040E090
:1041400050E00E94CDCF5F934F933F932F938DE428
:1041500094E09F938F93FC81FF938B818F933F9289
:104160002F920E94DFD42CC0C7010E946E13BC01A5
:10417000F701C680D780D0FADD24D0F89481F5808D
:10418000EB80BC80292F30E050E040E077FD35C067
:10419000011135C07F936F931F921F921F929F93BF
:1041A0001F92FF92DF92CF9284E594E09F938F93CA
:1041B0009C819F93AB81AF933F922F920E94DFD45B
:1041C0000FB6F894DEBF0FBECDBF89819A810F90E4
:1041D0000F900F900F90DF91CF910F91FF90EF9084
:1041E000DF90CF90BF90AF909F908F907F906F9017
:1041F0005F904F903F902F900895002361F0292FFA
:1042000030E0A4E6B0E00E94FFCF2FEF30E040E0C6
:1042100050E00E94CDCF5F934F933F932F931F9217
:10422000FF92DF92CF9287E594E09F938F93BF92A6
:10423000EF9295CFD70115968C9115971F928F937A
:1042400016969C91169717968C9181708F939F93D9
:104250008AE594E09F938F93BC81BF93EB81EF93AA
:1042600033CFD70114968D909D90AD90BC90179749
:1042700020E030E0A901C501B4010E9461CE240113
:10428000350187FF04C077FA709477F87094C30102
:10429000B2010E9433D16B01072E000C880B990BE1
:1042A0000E9468CE9B01AC01C301B2010E9454D0B0
:1042B00020E030E048EC52E40E94C7CE0E94BED11C
:1042C0000E9433D1062F772E20E030E0A901C501EE
:1042D000B4010E9461CE87FF07C07F920F93DF92E7
:1042E000CF9280E694E0B6CF7F920F93DF92CF9289
:1042F00081E694E09F938F939C819F93AB81AF93D2
:10430000E3CED70114968C9114971F928F93159634
:104310008C9115971F928F9316968C911F928F9365
:1043200087E594E09F938F93BC81BF93EB81EF93DC
:104330003F922F920E94DFD443CFD70117968C91E2
:1043400017971F928F9314968C9114971F928F93A7
:1043500015968C9115971F928F9316968C911F929C
:104360008F9384E594E09F938F93BC81BF93EB81FF
:10437000EF93F5CED70114966D917C914B815C81C2
:10438000C1010E94C5D421CF29803A8062CECF924C
:10439000DF92EF92FF920F931F93CF93DF93EC0185
:1043A000888199810E946695082F10E004301105DC
:1043B0009CF40E949E8A009739F0DC0118962C919B
:1043C0001897207F18962C93BC01888199810E94B0
:1043D00075990F5F1F4FEACFC880D98060E0C60192
:1043E0000E944A95FC01F184F88661E0C6010E94B2
:1043F0004A958C019B838A8362E0C6010E944A959C
:104400009D838C8364E0C6010E944A956C019F8362
:104410008E83F0E1FF1609F485C0FF1580F083E07C
:10442000F81689F1AAE0FA1609F46EC0DF91CF916F
:104430001F910F91FF90EF90DF90CF900895B2E120
:10444000FB1609F4ECC0E3E1FE12F0CF86E090E049
:104450000E94C9C3FC01D383C2838CE392E09183A1
:104460008083C114D10409F4F5C0D60118968C914B
:1044700018978F70823009F0EDC016968D919C913F
:1044800095838483E4C08AE090E00E94C9C37C01E4
:10449000DC011396DC93CE9312978EE592E08D9318
:1044A0009C9370E060E0CE010E94841B97FD1DC0CC
:1044B000F701958384830115110519F1F8018085B1
:1044C0008F708230D9F08530E1F4C8010E94669582
:1044D00090E0D70117969C938E93169782E892E00E
:1044E0008D939C93FA86E986A1CF91958195910948
:1044F000D70115969C938E931497DDCF81E090E0C1
:10450000E8CF90E080E0E5CF84E090E00E94C9C36E
:10451000FC01D383C2832AEE32E0318320839A8761
:10452000898784CF8BE090E00E94C9C37C01DC01C5
:104530001396DC93CE93129788EC92E011969C939D
:104540008E9316961C9270E060E0CE010E94841B50
:1045500097FD44C0F70195838483F7018481958199
:10456000009719F0863591053CF080E290E0D70184
:1045700015969C938E9314970115110509F441C06B
:10458000F80180858F708530E1F5C8010E9466953D
:104590008230B8F161E0C8010E944A95FC01908523
:1045A0009F70923039F561857285838594850E946C
:1045B00068CE20E030E04AE754E40E94C7CE0E9473
:1045C0003AD16115710581059105F9F0D70117966A
:1045D0006D937D938D939C931A9784CF919581953C
:1045E0009109D70115969C938E93149781E01696A6
:1045F0008C93B3CF933029F461857285838594853C
:10460000D8CF60E070E0CB01D4CF88E893E1A0E0A0
:10461000B0E0F70187839087A187B28763CF86E0F8
:1046200090E00E94C9C3FC01D383C28386EA92E072
:1046300091838083158214820115110541F0D80100
:1046400018968C918F70863011F415830483FA8745
:10465000E987ECCE90E080E013CFCF93DF93EC01BD
:10466000798368831A8619861B861E8A1D8A0E9492
:104670009013882329F0CE01DF91CF910C94C721AC
:10468000DF91CF910895EF92FF920F931F93CF93F5
:10469000DF93EC017B018E819F81892BD9F4888186
:1046A00099810E946695082F10E00530110594F459
:1046B0000E949E8A009721F0FC012085207F2087A0
:1046C0009F838E83BC01888199810E9475990F5FB9
:1046D0001F4FEBCFEE81FF813097D9F08085982F67
:1046E0009F70A9F4807F82608087EE81FF811186B0
:1046F000128613861486EE81FF81F782E682C70157
:10470000DF91CF911F910F91FF90EF90089592301C
:1047100061F3F12CE12CF3CFCF93DF93EC0160EA4E
:1047200074E185E19FE00E94B9828C819D810E94A5
:1047300065C470E060E08A819B810E9443231D82F2
:104740001C8281E090E0DF91CF910895CF92DF92BB
:10475000EF92FF920F931F93CF93DF93EC018C8125
:104760009D81892B61F40A811B8185E090E00E9484
:10477000C9C3BC01C8010E9443239D838C83EC8084
:10478000FD80E114F104A9F468E874E18EEE9DE087
:104790000E9495828EEE9DE00E949E8190E080E0D6
:1047A000DF91CF911F910F91FF90EF90DF90CF900D
:1047B00008951092B4071092B3071092AE071092AA
:1047C000AD071092B5071092B6071092B707109276
:1047D000B8071092AF071092B0071092B10710926D
:1047E000B20710922B0710926D07EA81FB81309778
:1047F00059F082819381009739F0DC0118962C9151
:104800002F70263009F468C061E474E18EEE9DE0FB
:104810000E94958261E070E08C819D81892B11F46A
:1048200070E060E08EEE9DE00E945E956FE374E1C3
:104830008EEE9DE00E94958261E070E08A819B810E
:10484000892B11F470E060E08EEE9DE00E945E9591
:104850006DE374E18EEE9DE00E949582EA81FB811A
:1048600061E070E082819381892B11F470E060E057
:104870008EEE9DE00E945E956BE374E18EEE9DE00E
:104880000E949582EA81FB810280F381E02D808580
:104890008F7061E070E0863011F470E060E08EEEC1
:1048A0009DE00E945E9569E374E18EEE9DE00E94BA
:1048B00095828EEE9DE00E949E816AE574E18EEE07
:1048C0009DE00E9495828EEE9DE00E949E81EC818B
:1048D000FD8182E0808362CF69E674E00E94D59416
:1048E000009709F4A8C0FC0120852F70243009F03E
:1048F000A2C0C184D284B60185E19FE00E942F82CC
:1049000065E374E185E19FE00E94958210E000E09C
:10491000C114D10409F486C0B80163517C4EC601AC
:104920000E9401C7892B09F077C0F801EF50FC4EB7
:1049300025913491922F832FD70113969C9313972F
:1049400014968C93EA81FB8160E774E08281938105
:104950000E94D594EC81FD81009709F472C0DC01BE
:1049600018962C9118972F70223009F06AC019966A
:104970004D915D916D917C911C974115510561059B
:10498000710509F45EC05283418341815281052E35
:10499000000C660B770B238186E19CE00E944C871C
:1049A000EC81FD8141815281052E000C660B770B55
:1049B000238189EF9AE00E944C87EA81FB816BEEAC
:1049C00074E0828193810E94D594009739F0FC01B4
:1049D0008185928590936C0780936B0760E774E103
:1049E00084EE9DE00E949582EA81FB810190F08136
:1049F000E02D6081718184EE9DE00E942F8284EE23
:104A00009DE00E949E81EC81FD8181E08083809306
:104A1000290281E090E0C4CE0A5F1F4F08341105DF
:104A200009F076CF60ED73E185E19FE00E94958209
:104A300096E080E081CF86E090E0F7019483838365
:104A400081CF80E09BE4928381839FCFCF92DF92DE
:104A5000EF92FF920F931F93CF93DF93EC016A01C4
:104A60007B018E819F81892BD9F4888199810E9455
:104A70006695082F10E00530110594F40E949E8A77
:104A8000009721F0FC012085207F20879F838E8363
:104A9000BC01888199810E9475990F5F1F4FEBCFF0
:104AA000EE81FF81309749F18085982F9F7019F52D
:104AB000807F82608087EE81FF81C186D286E38617
:104AC000F4866CE177E085E19FE00E9495822AE020
:104AD00030E0B701A60185E19FE00E94A98185E150
:104AE0009FE0DF91CF911F910F91FF90EF90DF90AA
:104AF000CF900C949E819230F1F2DF91CF911F9173
:104B00000F91FF90EF90DF90CF9008951F93CF9378
:104B1000DF93FC01162FC389D489818992899C0176
:104B20002F5F3F4F328B218BC80FD91FCE010E94C0
:104B300085CF181721F0612FCE010E948DCF81E023
:104B400090E0DF91CF911F910895FC0181899289B6
:104B5000248535858217930740F423893489820F91
:104B6000931F0E9485CF90E008958FEF9FEF0895E7
:104B70002F923F924F925F926F927F928F929F926D
:104B8000AF92BF92CF92DF92EF92FF920F931F935B
:104B9000CF93DF93CDB7DEB762970FB6F894DEBF41
:104BA0000FBECDBF5C014B0129013A01CA01B90119
:104BB0000E9433D11B013F926F938DE594E09F9348
:104BC0008F93CE0101967C019F938F930E941CD5F9
:104BD0000F900F900F900F900F900F9020E030E00B
:104BE000A901C301B2010E9469D1181624F077FA15
:104BF000709477F87094F70101900020E9F73197ED
:104C00006F01CE18DF088EE28083A2E0B0E0AC0F27
:104C1000BD1FAC0DBD1DBA8BA98BB10137FE03C002
:104C2000719561957109072E000C880B990B0E94F4
:104C300068CE9B01AC01C301B2010E9454D020E0B8
:104C400030E040E251E40E94C7CE0E9433D1605D63
:104C5000E989FA896083FE01EC0DFD1D1382D501FF
:104C6000ED91FC910288F389E02D9801A701B40130
:104C7000C501199562960FB6F894DEBF0FBECDBF81
:104C8000DF91CF911F910F91FF90EF90DF90CF9028
:104C9000BF90AF909F908F907F906F905F904F905C
:104CA0003F902F900895DA01E0918008F0E0FE2F08
:104CB000EE27E60FF71F90E0982F8827A901BD0186
:104CC0008E0F9F1F0C94228CCF93DF931F92CDB732
:104CD000DEB72091800830E0322F2227260F371FC1
:104CE00090E0982F8827498341E050E0BE016F5F34
:104CF0007F4F820F931F0E94228C0F90DF91CF91E4
:104D00000895CF93DF931F92CDB7DEB741E050E017
:104D1000BE016F5F7F4F0E94978B89810F90DF915B
:104D2000CF9108952091800830E0322F2227620F22
:104D3000731F90E0982F8827860F971F0C94812669
:104D400063E070E00C9492269F92AF92BF92CF9254
:104D5000DF92EF92FF920F931F93CF93DF93EC01BB
:104D60007B018091C909811121C01B821A8288EEC2
:104D700093E0A0E0B0E08C839D83AE83BF8383EBA0
:104D800093E09983888388E08C8788EE93E09E8700
:104D90008D87CE01DF91CF911F910F91FF90EF9002
:104DA000DF90CF90BF90AF909F90089534E0932E06
:104DB000833311F028E0922E89EBC82E89E0D82E9B
:104DC00010E098E0B92EA12CD6012D913D916D01F6
:104DD000F701848195812817390791F4812F0E946A
:104DE0006B90082F873111F08C3139F5812F0E949B
:104DF000578F892B59F50C3119F4812F0E944F9050
:104E00001F5F9112E1CFA11008C0D701ED91FC9175
:104E10000084F185E02DC70119951B821A8288EE66
:104E200093E0A0E0B0E08C839D83AE83BF8383EBEF
:104E300093E099838883BC86A8CF843149F081119F
:104E4000DFCFF601329711821082DACFB12ED8CFA0
:104E5000AA24A394D5CF8F929F92AF92BF92CF9264
:104E6000DF92EF92FF920F931F93CF93DF93CDB713
:104E7000DEB72F970FB6F894DEBF0FBECDBF5C0133
:104E80004B017A018091C9098823C9F104E0833379
:104E900009F008E0B501CE0101960E94A42689EB35
:104EA000C82E89E0D82E10E0F601219131916F01D2
:104EB000F501848195812817390751F4812F0E94CB
:104EC0006B90873129F4A701B401812F0E94CD8E08
:104ED0001F5F0113E9CFC7012F960FB6F894DEBF0D
:104EE0000FBECDBFDF91CF911F910F91FF90EF903B
:104EF000DF90CF90BF90AF909F908F900895F12C4E
:104F0000E12CE9CFDA01E0918008F0E0FE2FEE27F6
:104F1000E60FF71F90E0982F8827A901BD018E0F9B
:104F20009F1F0C94978B44E050E0BC018FE090E011
:104F30000C94228C44E050E0BC0185E090E00C949D
:104F4000228C44E050E0BC0181E090E00C94228C83
:104F500008959F92AF92BF92CF92DF92EF92FF920D
:104F60000F931F93CF93DF938C015B01942EE52E5B
:104F7000FC01C688D788F08C80E591E00E94209ED5
:104F80008F2D0E94738EC92DDE2D8C179D0708F47E
:104F9000EC019E01A501B6018F2D0E94F08DF80154
:104FA000868997898C0F9D1F978B868BCE01DF9109
:104FB000CF911F910F91FF90EF90DF90CF90BF9016
:104FC000AF909F900895CF93FC01C08D80E591E054
:104FD0000E94209E60E270E08C2F0E94878B62E02E
:104FE00070E08C2F0E94922684FD16C062E070E073
:104FF0008C2F0E94922683FF0AC048E162E070E095
:105000008C2F0E94642680E090E0CF91089580E587
:1050100091E00E94209EE3CF40E162E070E08C2F9F
:105020000E94642681E0F0CFFF920F931F93CF93ED
:10503000DF93EB01FC01178A168A2A81211109C02E
:105040002B81211106C02C81211103C02D81222327
:1050500001F141155105E9F08A01FC01F08C80E570
:1050600091E00E94209EAE014E5F5F4F24E030E051
:105070006CE070E08F2D0E945326B8018F2D0E94A6
:105080007A9081E090E0DF91CF911F910F91FF9096
:10509000089580E0F7CF0F931F93CF938C01FC010D
:1050A0006481758181E20E94A690C82F8830F8F44F
:1050B00080E591E00E94209E8C2F0E94A0268331E3
:1050C00031F08C2FCF911F910F910C944F9062E093
:1050D00070E08C2F0E94878BF80184819581EC2FE2
:1050E000F0E0EE0FFF1FE754F64F91838083CF91DE
:1050F0001F910F9108950F931F93CF93DF931F92EA
:105100001F92CDB7DEB7FC0124852830E0F48C0176
:1051100080E591E00E94209E22E030E0AE014F5FEA
:105120005F4F60E170E0F80184850E9482278981E9
:105130009A819827892798270F900F90DF91CF9118
:105140001F910F91089590E080E0F6CF0F931F9389
:10515000CF93DF931F921F92CDB7DEB7FC0124855A
:105160002830E0F48C0180E591E00E94209E22E04E
:1051700030E0AE014F5F5F4F64E070E0F80184857E
:105180000E94822789819A819827892798270F90E2
:105190000F90DF91CF911F910F91089590E080E0E3
:1051A000F6CFCF93DF93EC0189E294E09983888373
:1051B0001A821B821C821D8280E591E00E94209E43
:1051C000BE016E5F7F4F44E050E08FE090E00E94B0
:1051D000978BCE01DF91CF9108950E94E38C8823B5
:1051E00031F08091C909843329F0873381F090E050
:1051F00080E0089580E591E00E94209E85E390E0A4
:105200000E94812685FD0DC082E090E0089580E532
:1052100091E00E94209E8EE290E00E94812680FF15
:10522000F3CF81E090E008951F920F920FB60F9296
:1052300011240BB60F922F933F934F935F936F936D
:105240007F938F939F93AF93BF93EF93FF9380913F
:10525000B900887F803609F44DC008F040C088321C
:1052600009F4A7C028F5803109F49BC0C8F488234D
:1052700009F4F7C0883009F494C0FF91EF91BF9111
:10528000AF919F918F917F916F915F914F913F91DE
:105290002F910F900BBE0F900FBE0F901F9018957F
:1052A000883109F486C0803241F78093590814C0D0
:1052B000803409F49BC040F48033B9F38833E9F6B5
:1052C0008093590885ECAEC0803509F483C08835D9
:1052D00009F494C0883489F60E948110CECF8839B1
:1052E00009F48AC038F5883729F050F4883611F06F
:1052F000803719F683E080935A081092580855C0F9
:10530000883809F479C0803919F0803809F0B5CFB0
:1053100080915808803208F06FC0E091580881E011
:105320008E0F809358088091BB00F0E0E85CF74F47
:1053300080833BC0803B39F0D0F4803A09F477C0D9
:10534000883A09F09ACF84E080935A08109237087F
:1053500010923608F0E0E0E019958091360881114E
:105360000FC081E0809336081092160809C0803C77
:1053700009F4A8CF883C09F4A5CF883B09F07DCF7C
:10538000E091370881E08E0F80933708F0E0EA5E05
:10539000F74F80818093BB00909137088091360849
:1053A00029C080917F088093BB0085EC8093BC006E
:1053B00064CF90917E0880917D08981758F5E09110
:1053C0007E0881E08E0F80937E08F0E0E35AF74F6D
:1053D0008081E9CFE0917E0881E08E0F80937E0886
:1053E0008091BB00F0E0E35AF74F808390917E08F4
:1053F00080917D089817C8F285E8D8CFE0917E08A3
:1054000081E08E0F80937E088091BB00F0E0E35A2C
:10541000F74F808380915C0881115ECF81E080939B
:105420005B0884EA8093BC0010925A0826CF85EC72
:105430008093BC0010925A0880915808803230F452
:10544000E0915808F0E0E85CF74F1082609158084E
:1054500070E088E398E0F0E0E0E0199510925808D9
:105460000CCF1092590838CF4F925F926F927F9273
:10547000AF92BF92CF92DF92EF92FF920F931F9362
:10548000CF93DF9300D01F92CDB7DEB72B013C0145
:1054900029833A834B835C83A6019501C801B70138
:1054A000640D751D861D971D21153105410551059A
:1054B00011F00E94ABCF29813A814B815C81621748
:1054C000730784079507D0F424153505460557055D
:1054D00030F521E0822F0F900F900F900F90DF9109
:1054E000CF911F910F91FF90EF90DF90CF90BF90E1
:1054F000AF907F906F905F904F900895461657063B
:105500006806790650F421E089819A81AB81BC81DB
:1055100084159505A605B705E8F220E0DBCF21E06C
:105520004616570668067906A8F2F7CF8F929F9223
:10553000AF92BF92CF92DF92EF92FF920F931F93A1
:10554000CF93DF9300D000D000D01F92CDB7DEB74D
:105550006130710509F07AC24C010E949DA29B0145
:10556000AC016091FE067091FF068091000790915A
:105570000107A12CB12C650118E8E12E13E1F12EF1
:1055800000E010E00E94342A8823B9F080E00E94F5
:1055900064176093FE067093FF0680930007909354
:1055A000010767E873E185E19FE00E94B9826DE041
:1055B00070E082E092E00E94FA1A8CED99E00E947D
:1055C0005A788597ACF488EE93E02A960FB6F89453
:1055D000DEBF0FBECDBFDF91CF911F910F91FF9026
:1055E000EF90DF90CF90BF90AF909F908F900895F5
:1055F00045E250E064E077E08CED99E00E94208184
:105600008CED99E00E945A78892B59F062E070E0A5
:1056100080E090E00E946BA28CED99E00E943878C7
:10562000EFCF809128079091FD06891761F2809352
:10563000FD068091270790E09C01205F3F4F30934B
:105640002A0720932907499708F0BDCF80911107B9
:1056500090E09093FC068093FB0680911B0790E0FE
:105660009093FA068093F90680911D0790E090933D
:10567000F8068093F70680911F0790E09093F60656
:105680008093F5068091210790E090930307809323
:1056900002078091200790E09093F4068093F30630
:1056A000D401ED91FC9111970288F389E02D1296B7
:1056B0008D919C91DC018D919C91DC016D917C918F
:1056C0008091230725E734E04CE754E080FD02C0D9
:1056D0004FE754E0C40119958091F3069091F406C8
:1056E00080389105A9F4D4011296ED91FC9113979D
:1056F0000190F081E02D60817181ED91FC91028833
:10570000F389E02D23E834E04CE754E0C401199517
:105710008091F3069091F406892BA9F4D401129696
:10572000ED91FC9113970190F081E02D60817181E2
:10573000ED91FC910288F389E02D23E834E04FE7F6
:1057400054E0C401199569E874E085E19FE00E9486
:105750002F82609102077091030785E19FE00E940C
:105760005E9585E19FE00E949E8180910207F40191
:1057700020813181A281B3810D90BC91A02D6D91CA
:105780007C91D9015296ED91FC9120E934E04CE7EF
:1057900054E083FD02C04FE754E0C4011995D401E1
:1057A000ED91FC9111970288F389E02D12968D916D
:1057B0009C91DC018D919C91DC016D917C9180919B
:1057C000020727E934E04CE754E081FD02C04FE7CF
:1057D00054E0C40119952091F5063091F606032E88
:1057E000000C440B550BD4011296ED91FC911397CC
:1057F0000190F081E02D60817181ED91FC91068432
:10580000F785E02D03EA14E0C40119958091F706AD
:105810009091F806892BA9F4D4011296ED91FC9190
:1058200013970190F081E02D60817181ED91FC91E1
:105830000288F389E02D2AEA34E04FEA54E0C401FB
:1058400019958091F7069091F8060197A9F4D40173
:105850001296ED91FC9113970190F081E02D6081FB
:105860007181ED91FC910288F389E02D2AEA34E000
:1058700044EB54E0C40119958091F7069091F80625
:105880000297A9F4D4011296ED91FC91139701901F
:10589000F081E02D60817181ED91FC910288F389A6
:1058A000E02D2AEA34E04BEB54E0C40119958091D5
:1058B000F7069091F8060397A9F4D4011296ED919A
:1058C000FC9113970190F081E02D60817181ED9141
:1058D000FC910288F389E02D2AEA34E04FEB54E092
:1058E000C4011995D401ED91FC9111970288F389B7
:1058F000E02D12968D919C91DC018D919C91DC01A3
:105900006D917C918091F5069091F60623EA34E042
:105910004FE754E0892B11F04CE754E0C40119958E
:105920002091290730912A07032E000C440B550BB8
:10593000D4011296ED91FC9113970190F081E02D26
:1059400060817181ED91FC910684F785E02D04EC76
:1059500014E0C40119952091FB063091FC062F3FFD
:105960003105B9F0032E000C440B550BD4011296EF
:10597000ED91FC9113970190F081E02D6081718190
:10598000ED91FC910684F785E02D09EC14E0C4014B
:10599000199519828091F9069091FA0666EB73E1E8
:1059A0000097C9F061EB73E181309105A1F06CEAD9
:1059B00073E18230910579F06FE973E183309105ED
:1059C00051F068EA73E18430910529F08D36910534
:1059D00031F463E873E1CE0101960E940AC7209179
:1059E000F9063091FA06032E000C440B550BD40136
:1059F0001296ED91FC9113970190F081E02D60815A
:105A00007181ED91FC910684F785E02D0FEC14E097
:105A1000C401199580910207F40120813181A2818E
:105A2000B3810D90BC91A02D6D917C91D9015296BE
:105A3000ED91FC9125ED34E0AE014F5F5F4F80FDAD
:105A400002C04FE754E0C4011995BDCD90E080E05D
:105A5000BCCD8F929F92AF92BF92CF92DF92EF9286
:105A6000FF920F931F93CF93DF937C014A0159015B
:105A7000C0911208D0911308062F660F110B2097C2
:105A800009F45CC088858F70863009F055C06AEDD6
:105A900074E0CE010E94D5946C0182E088169104D6
:105AA00049F06CE374E0E3E08E16910429F0D0E055
:105AB000C0E006C06FED74E0CE010E94D594EC0109
:105AC000C114D104D9F1F60180858F708430B1F50D
:105AD00061857285A801C7010E94C5D4A80164EE42
:105AE00074E0C7010E94A7D4209779F188858F7050
:105AF000843059F569857A85A801C7010E94A7D429
:105B0000A80164EE74E0C7010E94A7D4A114B104F7
:105B100029F0A801B501C7010E94A7D4C701DF91F0
:105B2000CF911F910F91FF90EF90DF90CF90BF909A
:105B3000AF909F908F900895D0E0C0E0A80161ECF5
:105B400076E1C7010E9438C7C9CFF2E08F169104F1
:105B500081F083E08816910429F0609181087091AA
:105B60008208CACFA8016BEB76E1C7010E941AC771
:105B7000C7CFA80168EB76E1F8CFCF92DF92EF9222
:105B8000FF920F931F93CF93DF93CDB7DEB7C1542E
:105B9000D1090FB6F894DEBF0FBECDBF6C01AB01CB
:105BA00030E020E060E4CE0101967C010E94292DC6
:105BB000F70101900020E9F731978F010E191F09B5
:105BC000A801B701C6010E94B7D4892B11F010E0DB
:105BD00000E0C801CF5BDF4F0FB6F894DEBF0FBE09
:105BE000CDBFDF91CF911F910F91FF90EF90DF908C
:105BF000CF900895CF92DF92EF92FF920F931F9371
:105C0000CF93DF93CDB7DEB7C054D1090FB6F89468
:105C1000DEBF0FBECDBF809188089091890805979F
:105C200009F449C06115710509F445C069017A019B
:105C30008B0140E450E0CE0101960E94C5D46FE292
:105C400070E0CE0101960E948CD4892B41F498011A
:105C500043E050E060E4CE0101960E94292D4FE31D
:105C600050E0B601CE0101960E94A7D40E94F094A4
:105C7000882309F180918808909189080697D9F4C2
:105C800080911408811117C0B701CE0101960E94BE
:105C90006BA381E090E0C05CDF4F0FB6F894DEBFED
:105CA0000FBECDBFDF91CF911F910F91FF90EF906D
:105CB000DF90CF90089590E080E0EDCFAF92BF925B
:105CC000CF92DF92EF92FF921F93CF93DF9300D09A
:105CD00000D0CDB7DEB76C017C0110E08AE0A82EC1
:105CE000B12C133061F1F701828190E0B0E0A0E0C7
:105CF00089839A83AB83BC83BE82AD82BE016F5F12
:105D00007F4F84EE9DE00E94721A66EB76E10E945E
:105D100095821F5FFFEFEF1AFF0A143011F72696E6
:105D20000FB6F894DEBF0FBECDBFDF91CF911F91AC
:105D3000FF90EF90DF90CF90BF90AF900895F60165
:105D4000858190E0B0E0A0E089839A83AB83BC8337
:105D5000BE82AD82BE016F5F7F4F84EE9DE00E94E8
:105D6000721A64EB76E1D3CFEF92FF920F931F93F9
:105D7000CF93DF93EC01A881B981109761F18C91E9
:105D8000882349F108811981F8018081882351F025
:105D90008D3241F080538A3028F00F5F1F4F1983F6
:105DA0000883F0CFC8010E9495C67C016CE270E0C8
:105DB000C8010E948CD4009751F419821882C7013F
:105DC000DF91CF911F910F91FF90EF900895019671
:105DD00099838883F4CFF12CE12CF1CF65E372E154
:105DE00084EE9DE00E94958262E272E184EE9DE085
:105DF0000E94958264E172E184EE9DE00E949582AA
:105E00006CE072E184EE9DE00E94958284EE9DE05C
:105E10000E949E816FEF71E184EE9DE00E94958269
:105E20006FEE71E184EE9DE00E94958263EE71E178
:105E300084EE9DE00E9495826CEC71E184EE9DE021
:105E40000E9495826AEB71E184EE9DE00E9495824A
:105E500065EA71E184EE9DE00E94958266E971E158
:105E600084EE9DE00E94958267E871E184EE9DE0FA
:105E70000E9495826FE771E184EE9DE00E94958219
:105E800064E771E184EE9DE00E9495826AE671E12B
:105E900084EE9DE00E94958262E671E184EE9DE0D1
:105EA0000E94958266E571E184EE9DE00E949582F4
:105EB0006CE371E184EE9DE00E9495826DE171E1F9
:105EC00084EE9DE00E94958268E071E184EE9DE0A1
:105ED0000E9495826BEF70E184EE9DE00E949582B6
:105EE0006DEE70E184EE9DE00E94958261EE70E1BE
:105EF00084EE9DE00E94958269ED70E184EE9DE064
:105F00000E9495826EEC70E184EE9DE00E94958285
:105F100061EC70E184EE9DE00E94958269EB70E196
:105F200084EE9DE00E9495826EEA70E184EE9DE031
:105F30000E9495826FE970E184EE9DE00E94958257
:105F400066E970E184EE9DE00E94958268E870E168
:105F500084EE9DE00E9495826AE770E184EE9DE008
:105F60000E94958284EE9DE00C949E810F931F9376
:105F7000CF93DF9300D000D0CDB7DEB70E94EE2ED6
:105F80006EE17BE084EE9DE00E949582CE01019659
:105F90000E94D128CE0101960E945E2E09E214E0F3
:105FA0001A83098380915A0D90915B0DA0915C0D2D
:105FB000B0915D0D8B839C83AD83BE83CE01019632
:105FC0000E945E2E1A8309831B821C821D821E8200
:105FD00080E591E00E94209E44E050E0BE016D5FAC
:105FE0007F4F81E090E00E94978BCE0101960E9446
:105FF0005E2E1A8309831B821C821D821E8280E50D
:1060000091E00E94209E44E050E0BE016D5F7F4F12
:1060100085E090E00E94978BCE0101960E945E2E53
:1060200064E47BE084EE9DE00E94958288EC90E041
:1060300026960FB6F894DEBF0FBECDBFDF91CF918D
:106040001F910F910895009789F0FC0120852F7012
:10605000253061F40E944A95009741F0FC012085AB
:106060002F70243019F481859285089590E080E0A6
:106070000895CF92DF92EF92FF920F931F93CF93E9
:10608000DF9300D000D0CDB7DEB780911108811129
:106090009AC0809188089091890802970CF493C067
:1060A0008091EC069091ED06009709F48CC068EEA3
:1060B00074E00E94D5948C01009709F484C00E947A
:1060C0006695E82EF12CE114F10409F47CC070E02F
:1060D00060E0C8010E9423306C01EA94EF2809F4C3
:1060E00081C061E0C8010E944A95FC0101851285CA
:1060F000CE0101960E94D128CE0101960E94239ED6
:106100006FE07BE084EE9DE00E949582B60184EE14
:106110009DE00E942F826AE575E084EE9DE00E947A
:106120002F82B80184EE9DE00E945E956AE575E0DD
:1061300084EE9DE00E942F826AEC79E084EE9DE07F
:106140000E942F8284EE9DE00E949E8162E072E0B8
:1061500083E39FE00E945216D092290FC092280F2D
:1061600010932B0F00932A0F8AEC99E0892BE9F505
:1061700086EE94E090932D0F80932C0F80918308EE
:1061800090918408009741F070E060E00E94233015
:106190009093820880938108809181089091820871
:1061A000009721F090932F0F80932E0F1092310FB4
:1061B0001092300F81E08093110866EF7AE084EE50
:1061C0009DE00E94958226960FB6F894DEBF0FBE22
:1061D000CDBFDF91CF911F910F91FF90EF90DF9096
:1061E000CF90089502E012E083CF8AEC99E0C2CF0D
:1061F000CF92DF92EF92FF921F93CF93DF9300D065
:1062000000D0CDB7DEB761EF7AE084EE9DE00E946A
:10621000958289ECE82E8DE0F82E10E090E1C92EF1
:10622000D12CF70181917F01803130F46FEE74E061
:1062300084EE9DE00E942F82153041F1F7013197E5
:10624000808190E0B0E0A0E089839A83AB83BC8337
:10625000DE82CD82BE016F5F7F4F84EE9DE00E94A3
:10626000721A6FEE7AE00E9495821F5F1630C9F6AF
:1062700026960FB6F894DEBF0FBECDBFDF91CF914B
:106280001F91FF90EF90DF90CF9008958091CE0DF9
:1062900090E0B0E0A0E089839A83AB83BC83DE8288
:1062A000CD82BE016F5F7F4F84EE9DE00E94721A27
:1062B0000E949E81DACFEF92FF920F931F93CF93AC
:1062C000DF9300D000D01F92CDB7DEB77B01CE01A7
:1062D00007969F938F9301979F938F9301979F9317
:1062E0008F9301979F938F9301979F938F9301971C
:1062F0009F938F938E010F5F1F4F1F930F9381EF1B
:1063000094E09F938F93DB0113968C9113978F9357
:1063100012968C918F930E944CD50FB6F894DEBFE5
:106320000FBECDBF0697ECF46FEE7EE08EEE9DE0E3
:106330000E949582D70112966D917C918EEE9DE020
:106340000E942F8280E991E027960FB6F894DEBF75
:106350000FBECDBFDF91CF911F910F91FF90EF90B6
:1063600008958091C10D9091C20D892B09F44BC005
:106370000E949F95882309F446C0A091C10DB09159
:10638000C20D52961C921E92519754961C921E92C8
:10639000539784E890E01D969C938E931C971E96CD
:1063A0001C921E9780E090E350969C938E931F97CB
:1063B000ED91FC9111970088F189E02D64E070E087
:1063C000CD0119958091C10D9091C20DDC01ED9127
:1063D000FC910280F381E02D46E050E0B801199570
:1063E00086E0F801A9ECBDE001900D928A95E1F7F5
:1063F0008091C10D9091C20DDC01ED91FC9104885A
:10640000F589E02D19950E94F83061E07FE084EE77
:106410009DE00E94958288EC90E096CFEF92FF92EB
:106420000F93CF93DF93CDB7DEB7A0970FB6F89455
:10643000DEBF0FBECDBF7C0100E020E033E040E2D4
:1064400050E0BE016F5F7F4F0E94E11FBE016F5F92
:106450007F4F85E19FE00E942F826BE27AE085E129
:106460009FE00E949582F701618162956F7085E1DE
:106470009FE00E94579564E27AE085E19FE00E94E8
:106480009582F70161816F7085E19FE00E945795C9
:1064900085E19FE00E949E81A0960FB6F894DEBF32
:1064A0000FBECDBFDF91CF910F91FF90EF90089578
:1064B000AF92BF92CF92EF92FF920F931F93CF9321
:1064C000DF9300D000D01F921F92CDB7DEB75C01E2
:1064D00009831A832B833C834D835E836F83788784
:1064E00060E976E185E19FE00E949582CE01019608
:1064F0000E940E3269E876E1C7010E9401C7009749
:1065000009F45CC08981811132C00A810F700130A9
:1065100099F130F010E0023009F03FC0CC20C9F012
:1065200060E0CE0101960E945A12F50102811381AA
:10653000892B91F0C8010E94681B672B682B692B7F
:1065400041F480E00E946417AB01BC01C8010E94C5
:10655000262581E090E032C040E050E0BA01C80159
:106560000E94262560E0C5010E94B21CF2CF823055
:10657000E1F1A0F58130A9F16CE776E185E19FE0DA
:106580000E949582698185E19FE00E94579585E18F
:106590009FE00E949E8101E010E06CE676E185E1DB
:1065A0009FE00E949582B80185E19FE00E945E9580
:1065B00085E19FE00E949E8190E080E028960FB6E2
:1065C000F894DEBF0FBECDBFDF91CF911F910F9129
:1065D000FF90EF90CF90BF90AF9008958A50853094
:1065E00058F6F50102811381A5CF40E050E0BA01D1
:1065F000F50182819381B4CFCF92DF92FF920F9306
:106600001F93CF93DF93F12C6115710509F458C0E6
:106610006A01EB018C01CB010E949013F82E8823B4
:1066200009F44EC0D0FE05C0F8016081CE010E9481
:10663000751CD1FE3CC0F801918192959F704481F8
:10664000558166817781973030F09930D0F086EFB0
:10665000890F823090F0EC81FD81309771F0808558
:106660008F702EEF280F223010F0811106C0929506
:10667000907F80858F70982B9087CE010E949C130D
:1066800016C0EC81FD81309791F080858F709EEF70
:10669000980F923010F081110AC0418752876387AA
:1066A0007487EC81FD818085807F836080876DE1C8
:1066B0007AE085E19FE00E949582C8010E940E3237
:1066C0008F2DDF91CF911F910F91FF90DF90CF9091
:1066D0000895CF92DF92EF92FF920F931F93CF9383
:1066E000DF936115710509F474C06A017B018C01A7
:1066F000CB010E949013D82F8823C1F1D7011496A3
:106700008D919C91009709F446C0FC01C0852C2F07
:106710002F703EEF320F323010F0211131C0C5958D
:10672000C595C595C595D0FE72C0C7010E94A51C30
:10673000F8018083CC23F1F1C295C07F81818F70F5
:10674000C82BC183D70114968D919C91009771F14C
:10675000FC0120852F70223001F581859285A3856B
:10676000B485F80184839583A683B7838D2FDF9149
:10677000CF911F910F91FF90EF90DF90CF900895F0
:10678000253049F460E00E944A95009721F0DC0131
:106790001896CC91C4CFC0E0C6CF253039F460E064
:1067A0000E944A95009711F0FC01D7CF80E090E05D
:1067B000DC01D7CFD7011496ED91FC9180858295AD
:1067C000807F8595859585958595823021F08330EC
:1067D00081F0D0E0CBCF4185528563857485F80187
:1067E00081818F70806A8183448355836683778338
:1067F000BDCF4185528563857485F80181818F7095
:10680000806781834483558366837783AFCFCC23AE
:1068100089F2C295C07FF80191CF0F931F93CF9358
:10682000DF9300D000D01F921F92CDB7DEB7198240
:106830001A821B821C821D821E821F8218862A8158
:106840002F702A83FC0102811381C8010E94A51CBC
:106850008230C9F08530B9F040E052E0B801CE0195
:1068600001960E94693360E0CE0101960E945A129F
:1068700028960FB6F894DEBF0FBECDBFDF91CF9143
:106880001F910F91089590E080E0F2CFCF93DF93B6
:1068900000D000D01F921F92CDB7DEB7FC01862F2B
:1068A0008F706181607F682B618388E0DE011196C3
:1068B00001900D928A95E1F729813A814B815C81A3
:1068C0006D817E818F81988528960FB6F894DEBF02
:1068D0000FBECDBFDF91CF910895CF93DF9300D04E
:1068E00000D01F921F92CDB7DEB7FC01608398E005
:1068F000DE01119601900D929A95E1F729813A8176
:106900004B815C816D817E818F81988528960FB641
:10691000F894DEBF0FBECDBFDF91CF910895AF9247
:10692000BF92CF92DF92EF92FF920F931F93CF937C
:10693000DF93CDB7DEB7CC55D1090FB6F894DEBFE3
:106940000FBECDBF5C0166960FAF669767961FAF0F
:10695000679768962FAF689769963FAF69976A9671
:106960004FAF6A976B965FAF6B976C966FAF6C97F4
:106970006D967FAF6D971AAA19AAFE01F39682E170
:10698000DF011D928A95E9F77A961192119286E0BD
:10699000DF011D928A95E9F7CE018B5A9F4F0E9425
:1069A0000E32F0FE2CC06696EFAD6697E83108F027
:1069B0008DC0F0E08827E052FB4C8F4F0C9436D00E
:1069C0006C35F8346335663566356335F8346635CD
:1069D00066356635F834F834F8346635663566352C
:1069E00066356635663566356635663566356C35C9
:1069F00063E879E0CE01835B9F4F0E940AC76796E8
:106A00008FAD679782958F70813008F48DC0833089
:106A100018F0883009F088C00E94F094882309F4A7
:106A200023C18091140881111FC1C114D10409F040
:106A30001BC130E020E043E050E060E3CE0101966E
:106A40000E94292DD501ED91FC91608171814FE269
:106A500050E0CE0101960E94A7D401E020E032E090
:106A600044E150E0BE016F5C7F4FCE018B5A9F4FD7
:106A70000E94E11FF1FE07C066968FAD66978230D7
:106A800011F0853061F5F0FE4FC0BE01635B7F4FB2
:106A9000CE0101960E946BA362E679E085E19FE05A
:106AA0000E949582BE016F5F7F4F85E19FE00E944B
:106AB0002F826FE579E085E19FE00E949582BE011B
:106AC000635B7F4F29C06FE779E094CF61E779E09E
:106AD00085E19FE00E949582E894F0F890CFBE0196
:106AE0006F5C7F4FCE0101960E946BA36BE679E04D
:106AF00085E19FE00E949582BE016F5F7F4F85E137
:106B00009FE00E942F8268E679E085E19FE00E9485
:106B10009582BE016F5C7F4F85E19FE00E942F82CE
:106B200085E19FE00E949E8167968FAD6797807F89
:106B3000870100271071882311F0F1FC04C00115B2
:106B4000110509F4BDC030E020E043E050E060E30F
:106B5000CE0101960E94292DD501ED91FC91608115
:106B600071814FE250E0CE0101960E94A7D4C1147A
:106B7000D10469F064EE74E0CE0101960E9481D4E4
:106B80004FE250E0B601CE0101960E94A7D464EE18
:106B900074E0CE0101960E9481D44FE250E06BE593
:106BA00079E00115110511F467E579E0CE01019650
:106BB0000E941AC767968FAD679782958F70845031
:106BC000823008F069C067E1CE018B5A9F4F0E9466
:106BD0006D3426962FAF269727963FAF2797289696
:106BE0004FAF289729965FAF29972A966FAF2A97BC
:106BF0002B967FAF2B972C968FAF2C972D969FAF10
:106C00002D9700E020E033E044E150E0BE016F5CEE
:106C10007F4FCE018B5A9F4F0E94E11F61E579E0C3
:106C200085E19FE00E949582BE016F5F7F4F85E105
:106C30009FE00E942F826EE479E085E19FE00E9450
:106C40009582BE016F5C7F4F85E19FE00E942F829D
:106C500085E19FE00E949E810E94F094882321F0AC
:106C600080911408882301F1B701C5010E94351CE9
:106C700090E080E0C45ADF4F0FB6F894DEBF0FBE3D
:106C8000CDBFDF91CF911F910F91FF90EF90DF90DB
:106C9000CF90BF90AF90089520E032E0012B11F02B
:106CA00020E033E000E0B0CFBE016F5C7F4FCE014B
:106CB00001960E946BA360E072E0C5010E94111C66
:106CC000F0FE73C066968FAD66978A3009F478C07F
:106CD00008F06EC0813009F47EC0863009F47BC0B4
:106CE00030E020E043E050E060E3CE0101960E94F6
:106CF000292DD501ED91FC91608171814FE250E029
:106D0000CE0101960E94A7D4C114D10469F064EEAB
:106D100074E0CE0101960E9481D44FE250E0B601AA
:106D2000CE0101960E94A7D464EE74E0CE010196D4
:106D30000E9481D440E350E06BE379E0CE010196FC
:106D40000E941AC765E379E085E19FE00E94958281
:106D5000BE016F5F7F4F85E19FE00E942F8262E35B
:106D600079E085E19FE00E949582BE01635B7F4FE1
:106D700085E19FE00E942F8285E19FE00E949E8135
:106D80000E94F094882309F46FCF80911408811138
:106D90006BCFBE01635B7F4FCE0101960E946BA358
:106DA00060E071E0C5010E94111C81E090E062CFBB
:106DB0008B3071F08C3009F093CF69E479E002C038
:106DC00064E479E0CE01835B9F4F0E940AC788CFBD
:106DD0006FE379E0F7CFF5018085853009F080CF4A
:106DE000ECCFDC011196EC911197E295EF70E15038
:106DF000EB3008F037C0F0E08827EE5FF84C8F4F9B
:106E00000C9436D01437143732370D370D372337FB
:106E10001A371A371A370D370D3714966D917D9141
:106E20008D919C911797089514966C9170E090E065
:106E300080E0089514966D917D918D919C911797A6
:106E40000E9433D1089514966D917D918D919C91FE
:106E500017972AE030E040E050E00E94CDCFCA0111
:106E6000B901089560E070E0CB010895CF92DF9200
:106E7000EF92FF920F931F93CF93DF93CDB7DEB7BF
:106E800062970FB6F894DEBF0FBECDBF6C010B87C3
:106E90001C872D873E874F87588B698B7A8B6BECCD
:106EA00073E1C7010E9401C7EFE0F0E0892BF1F028
:106EB00065EC73E1C7010E9401C7E1E1F0E0892BB5
:106EC000A9F06FEB73E1C7010E9401C7E0E1F0E0B8
:106ED000892B61F01F706BEB73E1C7010E9401C742
:106EE000E12FF0E0892B11F4EEE0F0E09B8599238F
:106EF00009F48DC1309709F458C03197E131F1059B
:106F000008F041C08827E857F84C8F4F0C9436D0D2
:106F1000D5379937C337C337C337C3379638D338D4
:106F2000C337C337C337C337C337C337DA38F33848
:106F3000E638CE010B960E94F13670932A076093D3
:106F400029079B01205131092931310508F05AC127
:106F500020EF260F209327079B01770F440B550B3B
:106F6000D6011296ED91FC9113970190F081E02DDE
:106F700060817181ED91FC910684F785E02D04EC30
:106F800014E0C60119951092150781E080930D0752
:106F90008DE480930E078FE580930F0765E270E024
:106FA00084E097E00E94FA1A3BC0198291509E300B
:106FB00008F073C0E92FF0E08827EE51F84C8F4FAE
:106FC0000C9436D0F03721384D384D382138F03711
:106FD0004D384D384D386F386438403885387A38F8
:106FE000809102078160809321076DE070E08CE161
:106FF00092E00E94FA1AD6011296ED91FC91139735
:107000000190F081E02D60817181ED91FC91028809
:10701000F389E02D25ED34E04CE754E0C6011995E5
:1070200081E090E062960FB6F894DEBF0FBECDBF50
:10703000DF91CF911F910F91FF90EF90DF90CF9054
:107040000895809102078E7F809321076DE070E0A4
:107050008FE092E00E94FA1AD6011296ED91FC910F
:1070600013970190F081E02D60817181ED91FC9189
:107070000288F389E02D25ED34E04FE754E0CECFD0
:1070800010921B078091020781608093210766EBB5
:1070900073E1CE0101960E940AC7D6011296ED91C6
:1070A000FC9113970190F081E02D60817181ED9149
:1070B000FC910288F389E02D25ED34E0AE014F5FAD
:1070C0005F4FC60119955FCF81E080931B078091C8
:1070D000020781608093210761EB73E1DACF82E0E0
:1070E00080931B07809102078160809321076CEADF
:1070F00073E1CFCF84E080931B078091020781600A
:107100008093210768EA73E1C4CF83E080931B0773
:1071100065E075E085E19FE00E942F828091020783
:107120008160809321076FE973E1B3CF19829031B9
:1071300079F148F49C3089F0CE010B960E94F1362B
:1071400060931D0713C0913141F19231A9F782E09C
:1071500080931D076FE873E105C083E080931D07EE
:1071600066EB73E1CE0101960E940AC7D601129622
:10717000ED91FC9113970190F081E02D6081718178
:10718000ED91FC910288F389E02D2AEA34E096CF54
:1071900010921D076AE973E1E5CF81E080931D0736
:1071A00063E973E1DFCFCE010B960E94F136609365
:1071B0001B07E9CE913031F0923009F0E4CE109205
:1071C0002007E1CE80E580932007DDCE913049F0A5
:1071D0009230A9F3CE010B960E94F13660931F07FF
:1071E000D2CE83E0F0CF913039F0923009F0CBCE9F
:1071F00080912107877F03C0809121078860809359
:107200002107C1CE8FEF9FEF0DCF198246CFE2311C
:10721000F10508F0B8CE8827EF5EF64C8F4F0C943E
:1072200036D0023905399937C337C337C337C33727
:107230009638D338C337C337C337C337C337C33799
:10724000C337C337EA38CF93DF93EC01611571057B
:1072500039F48F8181708F8381E0DF91CF91089520
:107260008981982F92959F7029F180E09430A8F73A
:107270009B01770F440B550B2959310941095109DD
:10728000A4E6B0E00E94ECCF2BE531E040E050E016
:107290000E94CDCF37FF02C030E020E02536310517
:1072A00014F024E630E02F5F220F8F818170282BAD
:1072B0002F83D2CF8F7080628983DACF2F923F9253
:1072C0004F925F926F927F928F929F92AF92BF92F6
:1072D000CF92DF92EF92FF920F931F93CF93DF93A2
:1072E000CDB7DEB768970FB6F894DEBF0FBECDBF3F
:1072F0001C0109871A872B873C874D875E876F871C
:10730000788B22E1E216F10408F035C0F701EE5B5C
:10731000FC4F3081398BCE0109960E946E1397FD88
:1073200004C0BC01C1010E9423399A85892F8F7046
:10733000D1011196EC911197E07FE82B1196EC9317
:10734000119789858C93E295EF70EC3008F063C05B
:10735000F0E08827E155F64C8F4F0C9436D0B33BC4
:10736000D839D839523BBD39DD3B1B3B5C3B5C3BDC
:107370005C3B1B3B1B3B198ACECFB12C92959F7077
:107380009D3008F0BEC4E92FF0E08827E553F64CA5
:107390008F4F0C9436D00B3A173C373C173CE03BF0
:1073A000E03B173C173C813E813E173C173CEB3AD3
:1073B00092959F709D3008F01EC1E92FF0E088275C
:1073C000EB51F64C8F4F0C9436D00B3ABF3AB33A90
:1073D000753AF539F239963AC33AFB3AFB3A803AB4
:1073E000803AEB3A8889F10187838F85D10116961F
:1073F0008C9316978E8515968C9315978D8514967C
:107400008C9314979295907F11968C9111978F7011
:10741000982B11969C93B989BB2309F463C0F101A1
:10742000818182958F702B2F30E08217130609F42B
:1074300059C06BE879E085E19FE00E949582D10117
:1074400011966C9162956F7085E19FE00E9457954F
:1074500068E879E085E19FE00E949582698985E18D
:107460009FE00E94579566E879E085E19FE00E94E1
:107470009582F101008119821A821B821C821D8271
:107480001E821F82188689898295807F9A819F70CB
:10749000892B8A830983EE24EA94FE2C11812281B0
:1074A00033814481558166817781CE0101960E94A6
:1074B0005E39D1012C9311963C93119712964C93FF
:1074C000129713965C93139714966C9314971596D2
:1074D0007C93159716968C93169717969C93C101DB
:1074E0000E940E3288E0F1017BC18F859889F101FD
:1074F0008683878190FB80F987838E8585838BCFF8
:107500008D859E85AF85B8898F3F9105A105B10511
:1075100029F024F08FEF90E0A0E0B0E0B7FF03C0C7
:1075200080E090E0DC01F101848375CF6D857E857C
:107530008F8598892AE030E040E050E00E94CDCF6E
:107540002F3F31054105510529F024F02FEF30E0A0
:1075500040E050E057FF03C020E030E0A901D10136
:1075600014962C9358CF8F859889F1018683878153
:1075700090FB80F987838E8585838D85D5CF8D851A
:1075800014968C9348CFCD84DE84EF84F88820E075
:1075900030E0A901C701B6010E9461CE87FD17C086
:1075A00020E030E04FE753E4C701B6010E9469D103
:1075B000181634F4C12CD12CAFE7EA2EA3E4FA2E2E
:1075C000C701B6010E943AD1F101648324CFC12CD6
:1075D000D12C7601F5CFD10111968C9111978F7036
:1075E000806C11968C9311978D859E8515969C9332
:1075F0008E93149710CF6BE07AE085E19FE00E94B4
:1076000095826A8562956F7085E19FE00E9457952B
:1076100068E07AE085E19FE00E949582F101618156
:1076200062956F7085E19FE00E94579585E19FE02C
:107630000E949E81F0CE92959F70933091F09C3085
:1076400051F24D855E856F857889F10144835583BC
:10765000668377839295907F81818F70982B918339
:10766000DACE60E0C1010E945A12D10114968C93C7
:1076700014978F85988916968C93169717968C91E8
:10768000179790FB80F917968C9317978E85159610
:107690008C93159711968C9111978F70806211962B
:1076A0008C93B9CE60E0CE0109960E945A12D101A6
:1076B00014968C931497EECF92959F709D3008F09E
:1076C00065C0E92FF0E08827E759F44C8F4F0C9400
:1076D00036D00B3A883BB23B313BB23BB23B763BB8
:1076E000A23BA23BA23B963B9D3BEB3A6D857E8540
:1076F0008F8598890E9468CE20E030E040E251E416
:107700000E94C1D0F101648375838683978383CE01
:107710006D8570E090E080E00E9466CED101149605
:107720006D937D938D939C93179775CE6D857E8514
:107730008F8598890E9468CEE5CF6D857E858F857F
:107740009889EACF9295907FF10181818F70982B73
:1077500091838D859E85AF85B88984839583A68323
:10776000B78359CE9295907FD10111968C91119744
:107770008F70982B11969C938D859E85AF85B889C7
:10778000F10184839583A683B78345CE66EF79E0C4
:1077900085E19FE00E9495826A8562956F7085E120
:1077A0009FE00E94579563EF79E085E19FE00E949A
:1077B0009582D10111966C9133CFBB24B394DECD69
:1077C0004D855E856F857889F10144835583668395
:1077D00077839295907F81818F70982B918388E039
:1077E000DE01119601900D928A95E1F729813A8187
:1077F0004B815C816D817E818F81988568960FB603
:10780000F894DEBF0FBECDBFDF91CF911F910F91D6
:10781000FF90EF90DF90CF90BF90AF909F908F90B0
:107820007F906F905F904F903F902F90089596308B
:1078300009F43AC148F46D85913071F06FEF70E052
:10784000933051F060E008C0973009F439C19A5084
:107850006D857E859230B0F784E68F8788898E7F2C
:10786000888B1E868A858F7080628A876D872E85B9
:1078700030E0AFEFB0E00E94FFCF24E630E040E020
:1078800050E00E94CDCF69017A01FFEFCF16D104FD
:10789000E104F10429F024F0C12CD12C7601CA9422
:1078A00086012D852A8B622E712CBB2009F471C0B4
:1078B00088898695A82FA150BB0B2D01BFEF4B16D1
:1078C0005B0609F01EC1003811050CF000C18FE7FE
:1078D00090E08C199D09869DD001879DB00D969DE5
:1078E000B00D11242FEF30E00E944DD021E83EE78B
:1078F00040E050E00E94CDCFF1012783ABE9B0E03A
:10790000A70196010E94ECCFEFE78E2E912CA12CBF
:10791000B12CA50194010E94CDCF89019A010C5987
:107920001F4F2F4F3F4FAEEFB1E0A70196010E94CE
:10793000ECCFA50194010E94CDCFD3010E94ECCFE2
:107940002FEF30E040E050E00E94CDCF39012FEF23
:107950006216710421F01CF066246A94712C66EEA4
:1079600079E085E19FE00E949582B80185E19FE082
:107970000E945E9568ED79E085E19FE00E94958226
:10798000B30185E19FE00E945E9585E19FE00E9442
:107990009E81EEE6FBE1E491F0E0EE0FFF1FEC5A72
:1079A000F44E85919491E4ECFBE1E4912F853889C4
:1079B0003170AFEFBFEF0E94FFCF2DE631E040E026
:1079C00050E00E94CDCF44275527AAEFB5E00E9492
:1079D000ECCFDC01CB019058AF4FBF4FCD01BB279F
:1079E00097FDB095AB2F8E3FE1E09E0708F062C196
:1079F000382F8F3F910508F47FC14EEF481B50E0B0
:107A00003FEFF301319678012FEFE21AF20A009569
:107A100010E03E9DC0013F9D900D1124292F33277A
:107A2000200F311FDF010E944DD04B015C018824E3
:107A3000AA24BB245E9D90015F9D300D1124232F4D
:107A40003327200F311F0E944DD0BB27A92F982F1D
:107A5000872F882A992AAA2A4E9D90014F9D300D82
:107A60001124232F3327200F311FDF010E944DD017
:107A7000B82FA72F962F882788279927BB278829D3
:107A80009929AA29F101A683958384836CEA79E078
:107A900085E19FE00E949582C1010E940E3260E064
:107AA00080E00E9413A1B7CC6D857E858F85988973
:107AB0002AE030E040E050E00E94CDCFB901CCCECA
:107AC0006D857E858F8598890E9433D1C5CEA701AB
:107AD00096012058310941095109ABE9B0E00E94F3
:107AE000ECCF2FE730E040E050E00E94CDCF89019D
:107AF0009A010C591F4F2F4F3F4FD10117961C92DF
:107B00002ECF9201AAEBBFEF0E9445D044E6842E0F
:107B1000912CA12CB12CA50194010E94CDCFDA01AA
:107B2000C9018C599F4FAF4FBF4F8B8B9C8BAD8B37
:107B3000BE8B26E430E0D2010E944DD0A501940115
:107B40000E94CDCF49015A019EE1890E911CA11CD2
:107B5000B11C003811050CF093C08FE790E08C1930
:107B60009D09869DD001879DB00D969DB00D112475
:107B7000A50194010E94F7CF9B01AC01AFEFB0E0EB
:107B80000E94ECCF24E63AE640E050E00E94CDCFE0
:107B9000D10117962C932B893C894D895E892C0D38
:107BA0003D1D4E1D5F1DAEEFB1E00E94ECCF23EEF8
:107BB00030E040E050E00E94CDCF29013A01388FFB
:107BC0002F8BAFEFB0E0A70196010E94ECCF2FE71B
:107BD00030E040E050E00E94CDCF8901EA89AE2F2D
:107BE000B0E0A30192010E94ECCF2FEF30E040E023
:107BF00050E00E94CDCF39012F3F310521F01CF01C
:107C000066246A94712C62ED79E085E19FE00E9420
:107C100095822AE030E04B895C896D897E8985E117
:107C20009FE00E94A9816CEC79E085E19FE00E94D1
:107C300095822AE030E0B501A40185E19FE00E9431
:107C4000A98164EC79E085E19FE00E949582B8010A
:107C500085E19FE00E945E956CEB79E085E19FE015
:107C60000E949582B30185E19FE00E945E9563EBDF
:107C700079E085E19FE00E9495826F89788D81CEC1
:107C8000A70196012058310941095109ABE9B0E03B
:107C90000E94ECCF2FE730E040E050E00E94CDCFD3
:107CA00089019A010C591F4F2F4F3F4FD101179651
:107CB0001C92A9CF8C3FF3E09F0768F48D3F22E030
:107CC000920728F452E0580F3FEF40E09ACE3CEF85
:107CD000381B5FEFFACF8A3F35E0930781F08B3F87
:107CE000E4E09E0728F444E0480F5FEF30E089CEDF
:107CF0005AEF581B30E001C050E04FEF82CE50E009
:107D0000F9CF6AE979E085E19FE00E9495826A8572
:107D100062956F7085E19FE00E94579567E979E071
:107D200044CDAF92BF92CF92DF92EF92FF920F932A
:107D30001F93CF93DF93CDB7DEB768970FB6F89454
:107D4000DEBF0FBECDBFFC01098B1A8B2B8B3C8B8A
:107D50004D8B5E8B6F8B788F82819381009709F4B6
:107D60009FC024813581232B09F49AC0CC2009F4CB
:107D700097C06F0170E060E00E94841B192FD6014C
:107D8000ED91FC91028CF38DE02DC60119955C01FB
:107D90008230910509F478C0039709F447C095E053
:107DA000F1E0AF16B10409F091E019861A861B863E
:107DB0001C861D861E861F86188A9295907F8A854E
:107DC0008F70892B8A87EE24EA94FE2C09891A8900
:107DD0002B893C894D895E896F89788DCE01099602
:107DE0000E945E39F1E0AF16B10409F44FC082E0A1
:107DF000A816B10409F045C06F8570E0D60114964D
:107E00008C910E944FA161E070E0C6010E94AF1BFF
:107E10006E8570E00E944FA162E070E0C6010E9492
:107E2000AF1B6D8570E00E944FA12BC0612F661FB4
:107E30006627661FCE0141960E945A125C01BC0162
:107E4000D60114968C910E944FA164E076E185E101
:107E50009FE00E949582F6016481758185E19FE033
:107E60000E945E9562E076E185E19FE00E94958246
:107E7000B50185E19FE00E945E9585E19FE00E944B
:107E80009E8181E090E00EC094E08FCF63E070E0CF
:107E9000C6010E94AF1B688970E00E944FA1ACCF61
:107EA00090E080E068960FB6F894DEBF0FBECDBFBD
:107EB000DF91CF911F910F91FF90EF90DF90CF90C6
:107EC000BF90AF900895FC019181892F82958F70AA
:107ED00021F0823029F080E008959F7090629183B4
:107EE0009B0177FF02C030E020E02E3681E03807AA
:107EF00014F02DE631E02683878130FB80F98783FB
:107F000081E00895AF92BF92CF92DF92EF92FF92FD
:107F10000F931F93CF93DF9300D000D01F921F9237
:107F2000CDB7DEB75C017B0160FF03C0E894E0F8E9
:107F3000F3F8F3FC0DC00E947011663971058105DC
:107F4000910530F080918808909189080597F9F49F
:107F5000B70166277370C5010E94351C61E279E0A4
:107F600085E19FE00E9495828FEF9FEF28960FB6E4
:107F7000F894DEBF0FBECDBFDF91CF911F910F915F
:107F8000FF90EF90DF90CF90BF90AF90089519824F
:107F90001A821B821C821D821E821F8218868A8181
:107FA0008F708A8340E053E0B501CE0101960E94B4
:107FB000693360E073E0C5010E945B1CE82AF92A7E
:107FC000D12CC12C09811A812B813C814D815E818C
:107FD0006F817885C5010E948F34C8CF4F925F9220
:107FE0006F927F92AF92BF92CF92EF92FF920F93D8
:107FF0001F93CF93DF9300D000D01F921F92CDB775
:10800000DEB75C0109831A832B833C834D835E8337
:108010006F8378876BE976E085E19FE00E94958227
:10802000CE0101960E940E328981811134C00A81ED
:108030000F700130A9F160F1023021F010E005303D
:1080400009F03FC0D501ED91FC91068CF78DE02D34
:1080500009811A812B813C814D815E816F817885F8
:10806000C501199581E090E028960FB6F894DEBF1F
:108070000FBECDBFDF91CF911F910F91FF90EF9079
:10808000CF90BF90AF907F906F905F904F9008958A
:10809000CC24C394D7CF813051F1823009F4DEC0B3
:1080A0006EE876E085E19FE00E949582698185E136
:1080B0009FE00E94579585E19FE00E949E8101E02C
:1080C00010E06EE776E085E19FE00E949582B801BE
:1080D00085E19FE00E945E9585E19FE00E949E8180
:1080E000CE0101960E940E3290E080E0BDCF1A8151
:1080F00012951F70163009F478C088F48FEF810F45
:10810000823048F52D8130E0A4E6B0E00E94FFCF38
:108110002FEF30E040E050E00E94CDCF19C0173083
:10812000E9F186EF810F8230B0F48D819E81AF81BD
:10813000B88585369105A105B10524F084E690E067
:10814000A0E0B0E0B7FF03C080E090E0DC019C015C
:1081500029313105D4F4163009F47BC008F05EC033
:108160001150123008F469C0F5016281738140E05A
:1081700052E0CE0101960E94FC3260E07AE0D50127
:1081800012968D919C910E94823FD501ED91FC91B8
:10819000068CF78DE02DCC24C3945ACF4D805E80A1
:1081A0006F80788420E030E0A901C301B2010E9411
:1081B00061CE87FD11C020E030E048EC52E4C301FD
:1081C000B2010E9469D1181654F4412C512C88EC4C
:1081D000682E82E4782E03C0412C512C3201C30159
:1081E000B2010E9433D19B01B3CF6D817E818F811B
:1081F00098852AE030E040E050E00E94CDCF25365F
:1082000031054105510524F024E630E040E050E01E
:1082100057FF9ECF20E030E0A9019ACF173081F0C0
:108220001A5086E690E0A0E0B0E0123008F09CCF53
:108230008D839E83AF83B88797CF86E68D8394CF57
:1082400080E090E0ACECB2E48D839E83AF83B8878E
:108250008BCF8CEF93E0A0E0B0E0EACF1D821E82CE
:108260001F821886D501ED91FC91068CF78DE02DCB
:10827000CC24C39402E01A812B813C8140E0EDCEF6
:108280000F931F93CF93DF938C01FC01C081D181A9
:108290006FE270E0CE010E94D4D40097D9F0FC01C7
:1082A0001192CF010E948119EC0168E277E085E12B
:1082B0009FE00E949582BE0185E19FE00E945E954D
:1082C00085E19FE00E949E81CE01DF91CF911F91B9
:1082D0000F910895CE010E948119EC01892BA1F321
:1082E000F80111821082F0CF3F924F925F926F920D
:1082F0007F928F929F92AF92BF92CF92DF92EF9236
:10830000FF920F931F93CF93DF93CDB7DEB7CC5B74
:10831000D1090FB6F894DEBF0FBECDBF4C01C755D3
:10832000DF4F0883C95AD040C655DF4F1883CA5A59
:10833000D040C555DF4F2883CB5AD040C455DF4FBE
:108340003883CC5AD040C355DF4F4883CD5AD040F4
:10835000C255DF4F5883CE5AD040C155DF4F688396
:10836000CF5AD040C055DF4F7883C05BD040CF5448
:10837000DF4FF982E882C15BD0405C2C0E949DA255
:10838000C754DF4F688379838A839B83C95BD0405E
:10839000C655DF4F8881CA5AD0408F70682E712C25
:1083A000C0908808D0908908C954DF4FD982C8820C
:1083B000C75BD040CF54DF4FE881F981C15BD0402B
:1083C000309721F0808181110C94E34BD4011B96EE
:1083D0008C91882341F0C4010B96CF54DF4F9983D1
:1083E0008883C15BD0406114710411F00C942C4C53
:1083F000CF54DF4FE881F981C15BD040309711F055
:108400000C94E74BF401658876886114710411F4CB
:108410000C942C4CC655DF4F8881CA5AD0408F70BF
:1084200011F00C942C4C662DCE0187559F4F0E9465
:108430004634C756DF4F2883C959D040C656DF4F50
:108440003883CA59D040C556DF4F4883CB59D040F6
:10845000C456DF4F5883CC59D040C356DF4F688392
:10846000CD59D040C256DF4F7883CE59D040C15647
:10847000DF4F8883CF59D040C056DF4F9883C05A12
:10848000D0400C942C4CCE0187559F4F0E940E3249
:10849000CF54DF4FE881F981C15BD040309781F044
:1084A0008081843269F464E878E085E19FE00E948D
:1084B000958285E19FE00E949E810CEF1FEF32C004
:1084C000F40180819181009711F40C946F4CFDE0D0
:1084D0006F16710409F0ABC00E946695082F10E07A
:1084E00006301105A4F40E949E8A009739F0DC0141
:1084F00018962C911897207F18962C93BC01F401A4
:10850000808191810E9475990F5F1F4FE9CF65E0CF
:10851000D4018D919C910E944A958C01892BE1F4A4
:1085200010E000E0C801C454DF4F0FB6F894DEBF7E
:108530000FBECDBFDF91CF911F910F91FF90EF90B4
:10854000DF90CF90BF90AF909F908F907F906F9073
:108550005F904F903F900895C755DF4F8881C95A6B
:10856000D0408031E8F6CE0187559F4F0E94F1360A
:10857000161617061806190624F4F80180858D7062
:10858000A1F0D80118968C9118978F7018968C933B
:108590006AE778E085E19FE00E94958285E19FE0AF
:1085A0000E949E8101E010E0BDCF0E949DA26B0160
:1085B0007C01CE0187559F4F0E94F136C60ED71E13
:1085C000E81EF91EF801C186D286E386F486C755F7
:1085D000DF4F8881C95AD0408295807F8260808732
:1085E0006FE678E085E19FE00E949582CE01875595
:1085F0009F4F0E94F136AB01BC012AE030E085E1DB
:108600009FE00E94A98169E678E085E19FE00E94F1
:108610009582D80119964D915D916D917C911C9731
:108620002AE030E085E19FE00E94A981B7CFC755DD
:10863000DF4FF880C95AD040B4E0FB1609F4FEC2FF
:10864000BF1530F0FF2009F477C0B12CA12CB3C2C4
:1086500088EF8F0D8230C8F788E0FE01E755FF4FA5
:10866000DE01119601900D928A95E1F7C655DF4F14
:108670008881CA5AD040807F09F433C3CE01875520
:108680009F4F0E94F1368B01672B09F42AC369E0E2
:10869000C62EFC1003C0119501951109B401CE013D
:1086A00087559F4F0E94D09960E0CE0187559F4F1C
:1086B0000E946D346A962FAF6A976B963FAF6B97A7
:1086C0006C964FAF6C976D965FAF6D976E966FAF70
:1086D0006E976F967FAF6F97A0968FAFA097A1967A
:1086E0009FAFA19722E06216710409F445C30CF014
:1086F000FBC2CC24C3946114710409F0A6CFC65503
:10870000DF4FE881CA5AD040E295EF70E150EB307C
:1087100008F0B8C3F0E08827EF56FC4B8F4F0C945D
:1087200036D0BE46BE464247424742471D47F946FD
:10873000F946F946DB46DB4619821A821B821C8207
:108740001D821E821F8218868A818F708A83C65579
:10875000DF4F8881CA5AD040807F09F476CFE9E0A4
:108760006E16710409F429C20CF011C16114710470
:1087700009F431C122E06216710409F066CFB12C10
:10878000A12CC12C33243A94B401CE0101960E944D
:10879000D0998A81982F92959F70945F9F709230A4
:1087A00060F4C655DF4F9881CA5AD04092959F70A9
:1087B000923019F48F7080628A83D40118969C914C
:1087C000973071F4C655DF4F8881CA5AD040807EF9
:1087D000803211F0803421F48A818F7080628A8324
:1087E000F401A185B285892F90E0109741F0ED91B9
:1087F000FC911197028CF38DE02DCD0119957C0130
:10880000C755DF4F0881C95AD040C655DF4F188180
:10881000CA5AD040C555DF4F2881CB5AD040C455E5
:10882000DF4F3881CC5AD040C355DF4F4881CD5AF5
:10883000D040C255DF4F5881CE5AD040C155DF4F8E
:108840006881CF5AD040C055DF4F7881C05BD0409F
:10885000CE0101960E945E39CF57DF4F2883C15861
:10886000D040CE57DF4F3883C258D040CD57DF4F6E
:108870004883C358D040CC57DF4F5883C458D040AA
:10888000CB57DF4F6883C558D040CA57DF4F788336
:10889000C658D040C957DF4F8883C758D040C85703
:1088A000DF4F9883C858D040CE0101960E940E3207
:1088B000CC2069F1C655DF4F8881CA5AD0408295D5
:1088C0008F709FE0980F9F70923020F08A5F8F70BA
:1088D0008230E8F48A8182958F7081508230B8F4BA
:1088E0002D8130E0AFEFB0E00E94FFCF24E630E012
:1088F00040E050E00E94CDCF2F3F310541055105AA
:1089000029F024F02FEF30E040E050E02D8388E0A4
:10891000FE013196DE01A755BF4F01900D928A9559
:10892000E1F7FAE0BF2AD12CD40118968C91189760
:10893000873009F0FCC35520D9F01296ED91FC91D7
:1089400090859F709530A1F4C954DF4F888199813B
:10895000C75BD040059761F0CF54DF4F4881598104
:10896000C15BD040BE0167557F4FCF010E94FD4ED5
:10897000C755DF4F8881C95AD040853009F4ABC351
:1089800008F0EDC2833009F418C3312C86C38AE0A5
:108990006816710409F4BFC09BE06916710409F000
:1089A00054CEB401CE0101960E94D099CE018755D4
:1089B0009F4F0E946E13BC01CE0101960E94233985
:1089C00088E0FE013196DE01A755BF4F01900D9260
:1089D0008A95E1F7EDC0C4010E94BD4F8C0161E0B2
:1089E00070E01816190614F070E060E085E19FE071
:1089F0000E945E9560E474E085E19FE00E942F8212
:108A0000CE0187559F4F0E94F136AB01BC012AE091
:108A100030E085E19FE00E94A98185E19FE00E940E
:108A20009E81CE0187559F4F101611060CF0C1C6CE
:108A30000E94F136B12CA12C672B682B692B89F58C
:108A400062E0CE0187559F4F0E946D34CF56DF4FB5
:108A50002883C159D040CE56DF4F3883C259D04009
:108A6000CD56DF4F4883C359D040CC56DF4F588393
:108A7000C459D040CB56DF4F6883C559D040CA5641
:108A8000DF4F7883C659D040C956DF4F8883C75916
:108A9000D040C856DF4F9883C859D040AA24A39429
:108AA000BA2CCC24C394332433946ECE61E0CE012F
:108AB00087559F4F0E946D34C757DF4F2883C95891
:108AC000D040C657DF4F3883CA58D040C557DF4F14
:108AD0004883CB58D040C457DF4F5883CC58D04040
:108AE000C357DF4F6883CD58D040C257DF4F7883DC
:108AF000CE58D040C157DF4F8883CF58D040C057A1
:108B0000DF4F9883C059D040AA24A394BA2CCC2418
:108B1000C394312C39CEB401CE0101960E94D09974
:108B2000C255DF4F8881CE5AD0409A8192959F706E
:108B300041F0923051F0B12CA12CDD24D394C12C02
:108B400037C19A819F7090629A8390E08536910533
:108B500014F084E690E08E8388E0FE013196DE0119
:108B6000A755BF4F01900D928A95E1F762E0CE01C3
:108B700087559F4F0E944634EA962FAFEA97EB96AF
:108B80003FAFEB97EC964FAFEC97ED965FAFED975D
:108B9000EE966FAFEE97EF967FAFEF97C158DF4F2E
:108BA0008883CF57D040C058DF4F9883C058D040FB
:108BB000A12CFAE0BF2ED12CC2CFB401CE01019678
:108BC0000E94D099C155DF4F6881CF5AD040C0551F
:108BD000DF4F7881C05BD0407170CE0101960E945A
:108BE000633FC82E882309F457C188E0FE013196FF
:108BF000DE01A755BF4F01900D928A95E1F762E023
:108C0000CE0187559F4F0E944634E2962FAFE297E0
:108C1000E3963FAFE397E4964FAFE497E5965FAFF7
:108C2000E597E6966FAFE697E7967FAFE797E8960A
:108C30008FAFE897E9969FAFE997BACFC4010E943A
:108C4000BD4F181619063CF562E0CE0187559F4FBF
:108C50000E946D34AA962FAFAA97AB963FAFAB9701
:108C6000AC964FAFAC97AD965FAFAD97AE966FAF8A
:108C7000AE97AF967FAFAF97E0968FAFE097E19654
:108C80009FAFE197AA24A394BA2CD12CCC24C394EF
:108C90003324339449CE61E0CE0187559F4F0E9423
:108CA0006D34A2962FAFA297A3963FAFA397A49639
:108CB0004FAFA497A5965FAFA597A6966FAFA6975F
:108CC000A7967FAFA797A8968FAFA897A9969FAFB3
:108CD000A997AA24A394BA2CD12CCC24C394312CC8
:108CE00023CE05E010E0D3CC99E06916710409F4B5
:108CF000D8C0AAE06A16710409F0A7CCC655DF4FA8
:108D00008881CA5AD04082958F70823009F01CC188
:108D1000C255DF4F6881CE5AD040060F111D17FF94
:108D200002C010E000E00536110514F004E610E082
:108D3000C255DF4F0883CE5AD04062E0CE0187553E
:108D40009F4F0E9446342A962FAF2A972B963FAF0B
:108D50002B972C964FAF2C972D965FAF2D972E9675
:108D60006FAF2E972F967FAF2F9760968FAF60973C
:108D700061969FAF61971CCFC12CC1CCC355DF4F0B
:108D80006881CD5AD040060F111D17FF02C010E0B8
:108D900000E00F3F110519F014F00FEF10E0C3557C
:108DA000DF4F0883CD5AD040A12C5AE0B52ED12CEC
:108DB00033243A94B9CDC355DF4F68817981CD5AB8
:108DC000D040060F171F17FF02C010E000E0053665
:108DD000110514F004E610E0012E000C220B330BF9
:108DE000C355DF4F088319832A833B83CD5AD04074
:108DF000DBCFC355DF4F688179818A819B81CD5A52
:108E0000D0400E9433D1600F711F77FF02C070E025
:108E100060E06536710514F064E670E0072E000C22
:108E2000880B990B0E9468CEC355DF4F6883798306
:108E30008A839B83CD5AD040B7CFC355DF4F28815B
:108E40003981CD5AD0404AE0409FC001419F900DEA
:108E50001124820F931F97FF02C090E080E0893EAB
:108E6000B3E09B0714F088EE93E0092E000CAA0BE8
:108E7000BB0BC355DF4F88839983AA83BB83CD5A2D
:108E8000D04092CF88E0FE013196DE01A755BF4F5A
:108E900001900D928A95E1F7B12CA12CDD24D39499
:108EA00087CFC655DF4F8881CA5AD04082958F70D0
:108EB000823009F049C0C155DF4F6881CF5AD04098
:108EC000C055DF4F8881C05BD040782F7170060F8E
:108ED000171F0E36E1E01E072CF417FF05C00DE644
:108EE00011E002C010E000E0C155DF4F0883CF5A07
:108EF000D040C055DF4F8881C05BD04010FB80F967
:108F0000C055DF4F8883C05BD04062E0CE018755FB
:108F10009F4F0E94463462962FAF629763963FAF91
:108F2000639764964FAF649765965FAF6597669653
:108F30006FAF669767967FAF679768968FAF6897B2
:108F400069969FAF699734CE88E0FE013196DE01C5
:108F5000A755BF4F01900D928A95E1F7ECCD863071
:108F600009F47CC0873009F010CDC4010E94A51C13
:108F7000182F863009F061C069E478E085E19FE050
:108F80000E94958266E070E085E19FE00E945E9518
:108F900085E19FE00E949E8162E0CE0187559F4F50
:108FA0000E946D3429AF3AAF4BAF5CAF6DAF7EAF6F
:108FB0008FAF21969FAF21973CC0C4010E94A51C92
:108FC000853019F00DEF1FEFADCA6AE578E085E155
:108FD0009FE00E94958265E070E085E19FE00E943D
:108FE0005E9585E19FE00E949E81B401CE01875588
:108FF0009F4F0E94D09961E0CE0187559F4F0E94FC
:109000006D3422962FAF229723963FAF2397249655
:109010004FAF249725965FAF259726966FAF26977B
:1090200027967FAF279728968FAF289729969FAFCF
:1090300029976894A0F8B0F8A8CC61E378E085E1BE
:109040009FE00E949582612F70E085E19FE00E9481
:109050005E9585E19FE00E949E81B4CFC4010E948D
:10906000BD4F1816190684F1B401CE0187559F4FE4
:109070000E94D09961E0CE0187559F4F0E946D34C8
:1090800029AB3AAB4BAB5CAB6DAB7EAB8FAB98AF68
:109090006894A0F8B0F846E0342EC755DF4F8881B9
:1090A000C95AD040811134C06894A0F8C655DF4F2A
:1090B0008881CA5AD040807F79F16894B1F801E084
:1090C00010E0D110FAC91FC26DE178E085E19FE0A0
:1090D0000E94958277CFC4010E94BD4F18161906D1
:1090E000A4F462E0CE0187559F4F0E946D3429A7FA
:1090F0003AA74BA75CA76DA77EA78FA798AB6894EC
:10910000A0F8B0F835E0332EC8CF66E078E0DECFC7
:109110006894A0F8B0F8CACF40E052E0B401CE01A4
:1091200087559F4F0E9469338111C7CFC8CF9FEFEA
:109130003912B1C0C4010E94BD4F332433941816B4
:1091400019060CF4ABC0312C6EEF77E085E19FE09F
:109150000E949582E32C032C000CFF08CD54DF4FB6
:10916000F982E882C35BD040B70185E19FE00E94AD
:109170005E9567EF77E085E19FE00E9495826C2D18
:1091800070E085E19FE00E945E9585E19FE00E948E
:109190009E81CF54DF4F48805980C15BD04041143D
:1091A000510409F484C063E879E0C2010E9401C758
:1091B00001E010E0892B09F44BC06FE779E0C201B0
:1091C0000E9401C702E010E0892B09F441C065E468
:1091D00077E0C2010E9401C705E010E0892BC1F1D0
:1091E00061E477E0C2010E9401C706E010E0892B2C
:1091F00079F164E479E0C2010E9401C70AE010E05D
:10920000892B31F16FE379E0C2010E9401C70BE0C5
:1092100010E0892BE9F069E479E0C2010E9401C7FE
:109220000CE010E0892BA1F068E377E0C2010E9416
:1092300001C70DE010E0892B59F064E377E0C2012B
:109240000E9401C710E000E0892B11F40EE010E04D
:10925000C4010E94A51CE82EF12CE114F10431F4A4
:10926000CD54DF4FE880F980C35BD0400115110574
:1092700009F436C0E016F106A1F061EE77E085E171
:109280009FE00E949582B70185E19FE00E945E9574
:1092900085E19FE022C3332009F456CFCC24C39448
:1092A00053CFCF54DF4F19821882C15BD040C755CE
:1092B000DF4FE881C95AD040EA3008F00EC1F0E033
:1092C0008827EA59F64B8F4F0C9436D07A4A564A83
:1092D0004F4AA9497A4A364A134AEB497A4A7A4AA6
:1092E000D40119968D919C91009709F419C9DC015C
:1092F000ED91FC910488F589E02D7201C755DF4F8F
:109300000881C95AD040C655DF4F1881CA5AD0408B
:10931000C555DF4F2881CB5AD040C455DF4F388127
:10932000CC5AD040C355DF4F4881CD5AD040C255AA
:10933000DF4F5881CE5AD040C155DF4F6881CF5A98
:10934000D040C055DF4F7881C05BD04019958C016B
:10935000E9C8C4010E94A51C853009F033CE62ED36
:1093600077E085E19FE00E94958265E070E085E10D
:109370009FE00E945E9585E19FE00E949E81B4017E
:10938000CE0187559F4F0E94D099F401808585308A
:1093900099F46CE0CE0187559F4F0E946D3429A34C
:1093A0003AA34BA35CA36DA37EA38FA398A7689455
:1093B000A0F8B0F8312C52C061E0CE0187559F4F24
:1093C0000E946D34298F3A8F4B8F5C8F6D8F7E8F0B
:1093D0008F8F98A3ECCFC4010E94A51C182F863054
:1093E000F9F461EC77E085E19FE00E94958266E008
:1093F00070E085E19FE00E945E9585E19FE00E941C
:109400009E8162E0CE0187559F4F0E946D34298B6B
:109410003A8B4B8B5C8B6D8B7E8B8F8B988FC7CFF2
:1094200069EA77E00CCE31101EC0B401CE01875539
:109430009F4F0E94D09961E0CE0187559F4F0E94B7
:109440006D3429873A874B875C876D877E878F8746
:10945000988B6894A0F8B0F826E0322E0FEF1FEF3B
:10946000CC24C3942ECE65E977E030CE3320A1F032
:1094700062E0CE0187559F4F0E946D3429833A8365
:109480004B835C836D837E838F8398876894A0F879
:10949000B0F895E0392EE2CF6EE777E017CEC40141
:1094A0000E94A51C853009F082CF8CCD332019F0A5
:1094B0006BE677E00BCEC655DF4F8881CA5AD040A5
:1094C000807F31F4B401CE0187559F4F0E94D0991F
:1094D0006894A0F8F3E0BF2A6DCFC655DF4F8881AE
:1094E000CA5AD040807F19F46894B0F863CF23E063
:1094F000B22A60CFD1100C945D42312C0FEF1FEFD8
:10950000A114B10439F0A501B401CE0187559F4FD4
:109510000E94FC32D40119968D919C91009709F418
:1095200074C0CF54DF4FE880F980C15BD040DC01CC
:10953000ED91FC910488F589E02DC755DF4F088136
:10954000C95AD040C655DF4F1881CA5AD040C555B8
:10955000DF4F2881CB5AD040C455DF4F3881CC5AD9
:10956000D040C355DF4F4881CD5AD040C255DF4F60
:109570005881CE5AD040C155DF4F6881CF5AD04074
:10958000C055DF4F7881C05BD04019958C013320E6
:1095900021F0632DC4010E94751CC954DF4FE8817E
:1095A000F981C75BD040359721F0B501C4010E9415
:1095B000823F61E577E085E19FE00E949582B801F6
:1095C00085E19FE00E945E956AE477E085E19FE097
:1095D0000E9495820E949DA2AB01BC01C754DF4F3F
:1095E000C880D980EA80FB80C95BD0404C195D09F6
:1095F0006E097F092AE085E19FE00E94528185E1A2
:109600009FE00E949E810C949242F40180858530F7
:1096100009F464C0863009F0BACF70E060E0C4019C
:109620000E94841B7C01009709F4B1CF712C612C3E
:1096300097FF06C0F194E194F10866246394712CBD
:10964000C70101978635910508F0A1CFC755DF4FB7
:109650000881C95AD04010E0DE2C61E08E2D0E94B6
:1096600013A1672859F10130110521F061E00C3098
:10967000110509F460E0062F10E08D2D0E94E5A091
:1096800066E677E085E19FE00E949582B70185E17B
:109690009FE00E945E9564E677E085E19FE00E948E
:1096A0009582B80185E19FE00E945E9585E19FE08B
:1096B0000E949E816894A0F8B0F874C00130110532
:1096C00051F091E080E00C30110509F090E0092F95
:1096D000182F602FD2CF01E010E0FBCFF2E06F1621
:1096E000710409F462C02CE06216710429F06A94D6
:1096F000672809F04CCFDECFC4010E94681B892B7C
:1097000049F4D401ED91FC91608171818AE095E08A
:109710000E9486A3CE0187559F4F0E94271320E009
:1097200030E048EC52E40E94C7CE0E9433D1CD54C1
:10973000DF4F688379838A839B83C35BD040CD549A
:10974000DF4F48805980C35BD04088E00E94641797
:109750006B017C0160E677E085E19FE00E949582E5
:10976000CD54DF4F68817981C35BD04085E19FE0B4
:109770000E945E956BE577E085E19FE00E9495820F
:10978000B701A601662777272AE085E19FE00E94BE
:10979000528185E19FE00E949E81B601A201C40131
:1097A0000E94262501E010E0F2CE6894A0F8B1F8FE
:1097B000F9CF0E94F136672B682B692B09F076C927
:1097C000B12CA12CA4C96114710409F045C0808199
:1097D000882311F40C940242CE018F549F4F0E94B3
:1097E00040413C01C655DF4F8881CA5AD0408F7036
:1097F00071F5662DCE0187559F4F0E944634CF5597
:10980000DF4F2883C15AD040CE55DF4F3883C25A2C
:10981000D040CD55DF4F4883C35AD040CC55DF4FA1
:109820005883C45AD040CB55DF4F6883C55AD040C7
:10983000CA55DF4F7883C65AD040C955DF4F888359
:10984000C75AD040C855DF4F9883C85AD0406114DA
:10985000710411F40C9402420E9470116B018B018F
:1098600069EB78E085E19FE00E949582B60185E191
:109870009FE00E945E9562EB78E085E19FE00E94A8
:109880009582D401ED91FC916081718185E19FE029
:109890000E942F826CEA78E085E19FE00E94958229
:1098A000CF54DF4F68817981C15BD04085E19FE073
:1098B0000E942F8266EA78E085E19FE00E9495820F
:1098C000083C110514F00C94434268E978E08EEEF0
:1098D0009DE00E9495828EEE9DE00E949E810FEF9A
:1098E0001FEF0C9492422F923F924F925F926F9291
:1098F0007F928F929F92AF92BF92CF92DF92EF9220
:10990000FF920F931F93CF93DF93CDB7DEB7A4974A
:109910000FB6F894DEBF0FBECDBF5C011B01709087
:10992000D406772009F4B8C0809186088F5F8093B1
:109930008608E0918A08F0918B08309709F4A4C05A
:109940008680978040908A0850908B08411451047B
:1099500009F496C08114910409F492C0D4011896B8
:109960008C918F70853091F7C4010E94669582308A
:1099700068F3B401CE0101960E942D23CE01019619
:109980000E949013882309F45EC060E074E0CE0169
:1099900001960E945B1C892B09F455C0188E198E04
:1099A0001A8E1B8E1C8E1D8E1E8E1F8E898D8F70A3
:1099B000898F40E053E0BE016F5F7F4FCE01489634
:1099C0000E9469336DEF78E085E19FE00E94958207
:1099D00060E074E0CE0101960E94111C8A859B858F
:1099E000009789F1DC01ED91FC910488F589E02D67
:1099F000CC24C394F12CE12C088D198D2A8D3B8D3C
:109A00004C8D5D8D6E8D7F8D19958F3F9807D9F0A8
:109A1000E981FA8160817181892BE9F485E19FE018
:109A20000E942F826BEF78E085E19FE00E94958293
:109A300063EF78E085E19FE00E94958285E19FE0F9
:109A40000E949E81712CF40182809380CE01019648
:109A50000E94B71377CF85E19FE00E942F8261EFCC
:109A600078E085E19FE00E9495826DEE78E085E1E7
:109A70009FE00E94958285E19FE00E949E81E3CF56
:109A800085E19FE00E949E818091860881508093AD
:109A9000860871101092D40665E0D5018D919C91D5
:109AA0000E944A954C01009709F490C0FC01808502
:109AB000859585958595859588A341845284638491
:109AC00074840E949DA2F8A1FF2309F47FC0461A66
:109AD000570A680A790A188E198E1A8E1B8EF88F0B
:109AE000198D1F70106A198F4C8E5D8E6E8E7F8E51
:109AF000C301B20128EE33E040E050E00E94CDCF38
:109B000029A33AA34BA35CA3672B682B692B19F5F8
:109B1000D12CC12CE12C90E1F92E08A12A8D3B8D8E
:109B20004C8D5D8D6E8D7F8DC5010E948F342AE036
:109B300030E049A15AA16BA17CA185E19FE00E9480
:109B4000A98162E179E085E19FE00E94958285E14B
:109B50009FE00E949E8177FE39C022E042165104A8
:109B6000610420E8720694F1D12CC12CE12C80E133
:109B7000F82E088D198D2A8D3B8D4C8D5D8D6E8D47
:109B80007F8DC5010E948F3419821A821B821C822C
:109B90001D821E821F8218861A811F701A8388A157
:109BA0008983CC24C394F12CE12C082F2B813C8198
:109BB00040E05E816F817885C5010E947441D401C7
:109BC00018968C9118978F7018968C93B1E02B167D
:109BD0003104B9F460E073E0C5010E945B1C00979A
:109BE00081F020918808309189082630310549F4A8
:109BF000BC01C5010E94823F60E073E0C5010E9484
:109C0000111CF501818592850097D9F490E080E0E0
:109C1000A4960FB6F894DEBF0FBECDBFDF91CF91F3
:109C20001F910F91FF90EF90DF90CF90BF90AF907A
:109C30009F908F907F906F905F904F903F902F906C
:109C40000895DC01ED91FC910484F585E02D1995D2
:109C5000892BE1F2F50181859285DC01ED91FC9182
:109C60000480F581E02DB1011995D2CFAF92BF925A
:109C7000CF92DF92EF92FF920F931F93CF93DF93D8
:109C8000CDB7DEB767970FB6F894DEBF0FBECDBF76
:109C9000E0918A08F0918B08309709F49DC080917B
:109CA00086088F5F8093860806811781E0908A0876
:109CB000F0908B08E114F10431F10115110519F14F
:109CC000F80180858F708530A9F7C8010E946695DC
:109CD000823080F3B801CE0101960E942D23CE017F
:109CE00001960E949013882331F062E070E0CE016B
:109CF00001960E94734CF80102811381CE010196F6
:109D00000E94B713D3CF8091860881508093860834
:109D10008091880890918908059709F45DC00E9498
:109D20009DA29B01AC016091DE067091DF068091DF
:109D3000E0069091E106A12CB12C650118EEE12E10
:109D400013E0F12E00E010E00E94342A082F88234F
:109D500009F442C010E06091EE067091EF066115C3
:109D60007105D1F1111138C0FB0180858F708530EC
:109D7000D9F4CE0101960E942D2361E070E0CE015E
:109D800001960E94734C892B59F00E949DA260930A
:109D9000DE067093DF068093E0069093E106102FB5
:109DA000CE0101960E94B713E091EE06F091EF0606
:109DB000309791F0828193819093EF068093EE0625
:109DC000892B49F6E0918A08F0918B08868197816A
:109DD0009093EF068093EE0667960FB6F894DEBF79
:109DE0000FBECDBFDF91CF911F910F91FF90EF90EC
:109DF000DF90CF90BF90AF9008954F925F926F9297
:109E00007F928F929F92AF92BF92CF92EF92FF92EA
:109E10000F931F93CF93DF93CDB7DEB767970FB63E
:109E2000F894DEBF0FBECDBF009709F4A4C0FC01BB
:109E300020852F70253009F09EC02A015B018680A5
:109E40009780809186088F5F8093860881149104A3
:109E500009F48CC0F40180858F70843009F082C0D1
:109E60006185728580918A0890918B080E94D594B3
:109E70003C01009709F476C0FC0180858F70853025
:109E800009F070C0B301CE0101960E942D23A114E8
:109E9000B104A9F0CE0101960E949013882379F0B5
:109EA000C12C7201F501008111812281338144812D
:109EB000558166817781CE0101960E94744160E0F0
:109EC000C3010E944A950097D1F1FC0120852F70B3
:109ED0002230A9F581859285A385B4850797A105D0
:109EE000B10569F561E0C3010E944A95A201B5017F
:109EF0000E94FD4EA114B10489F5882379F1809167
:109F00008608815080938608CE0101960E94B7137F
:109F100081E067960FB6F894DEBF0FBECDBFDF912C
:109F2000CF911F910F91FF90EF90CF90BF90AF9086
:109F30009F908F907F906F905F904F900895A114A5
:109F4000B10461F4CE0101960E949013882331F090
:109F5000CE0101960E94BD4F892B89F6CE01019654
:109F60000E94B713F4018280938070CF809186089D
:109F700081508093860880E0CCCFFF920F931F938F
:109F8000CF93DF9300D000D01F921F92CDB7DEB7E2
:109F90008C0119821A821B821C821D821E821F82E2
:109FA00018868A818F708A83D801ED91FC91608137
:109FB000718185E19FE00E942F826BEE78E085E160
:109FC0009FE00E949582C8010E949013811119C0E0
:109FD00062EE78E085E19FE00E94958285E19FE056
:109FE0000E949E810FEF1FEFC80128960FB6F894CC
:109FF000DEBF0FBECDBFDF91CF911F910F91FF90BC
:10A000000895C8010E94A51CF8019085973039F089
:10A01000853049F1D0F48130E9F0823021F1D80166
:10A0200019968D919C91009721F1DC01ED91FC91A5
:10A030000688F789E02D199501E0892B09F400E0E5
:10A04000802F0E94D01710E0CFCF863019F08A50B1
:10A05000833028F763EC78E085E19FE00E949582E9
:10A0600001E010E0C1CF80E00E94D01710E000E0D6
:10A07000BBCF40E052E0B801CE0101960E946933A7
:10A08000F8018085873079F160F4833009F452C09B
:10A09000843061F063ED78E085E19FE00E94958275
:10A0A000E5CF883009F446C08930A1F760E0CE01E1
:10A0B00001960E945A128C0168EC78E085E19FE0DD
:10A0C0000E949582B80185E19FE00E945E9585E13E
:10A0D0009FE00E949E8191E080E0012B09F490E0D6
:10A0E000092F182F81CF0280F381E02D80858F709A
:10A0F000853031F560EE78E085E19FE00E94958241
:10A1000050E040E070E060E0F801828193810E94BD
:10A11000FD4EF82E082F10E06DED78E085E19FE010
:10A120000E9495828F2D0E94D01785E19FE00E94AA
:10A130009E815ACFCE0101960E94F1368B01BCCF91
:10A1400010E000E0B9CF2F923F924F925F926F9252
:10A150007F928F929F92AF92BF92CF92DF92EF92B7
:10A16000FF920F931F93CF93DF93CDB7DEB7609726
:10A170000FB6F894DEBF0FBECDBFDC0112966D9115
:10A180007C916115710509F48DC04C0119821A8208
:10A190001B821C821D821E821F8218868A818F70FC
:10A1A0008A8340E052E0CE0101960E94693360E06C
:10A1B000CE0101960E945A121C01F4018281938102
:10A1C0000E94681B2B013C01D40117962D913D91F3
:10A1D0004D915C911A97D1010E94F7CF2FEF30E09B
:10A1E00040E050E00E94ABCF29873A874B875C87DD
:10A1F0000E949DA29B01AC0189859A85AB85BC8597
:10A200000097A105B10509F468C0A12CB12C650126
:10A210007C018D01C301B2010E94342A8987411457
:10A22000510461047104F1F1D40117968D919D914F
:10A230000D90BC91A02D8D879E87AF87B88B0E9413
:10A240009DA29B01AC018D859E85AF85B889009745
:10A25000A105B10561F0A12CB12C65017C018D0136
:10A26000C301B2010E94342A882309F451C0D401E9
:10A2700012966D907C9080E00E946417AB01BC0147
:10A28000C3010E942625232869F0F40184810E94DD
:10A290009E11D40116969C91891304C061E0C401FB
:10A2A0000E94B21C90E080E060960FB6F894DEBF8A
:10A2B0000FBECDBFDF91CF911F910F91FF90EF9017
:10A2C000DF90CF90BF90AF909F908F907F906F90D6
:10A2D0005F904F903F902F90089591E099879FCF86
:10A2E000B985BB23F1F060E0C4010E94B21CF40107
:10A2F000828193810E94BD4F892BA1F640E050E0FE
:10A30000BA01D40112968D919C910E942625CACF44
:10A31000F40184810E949E11D40116969C918913A8
:10A32000DFCF232809F4BECFF40184810E949E115F
:10A33000D40116969C918913B5CFB985B111B2CFCE
:10A34000ADCFCF93DF93EC016FE076E185E19FE045
:10A350000E9495826C817D8185E19FE00E945E95DF
:10A3600069E076E185E19FE00E94958285E19FE0CA
:10A370000E949E8161E08C810E9413A16E818C817C
:10A380000E94E5A08A819B81009729F040E050E07F
:10A39000BA010E94262581E090E09093BE07809349
:10A3A000BD078A819B810E94BD4F892B59F40A8089
:10A3B000DB81C02D80E00E946417AB01BC01CE019F
:10A3C0000E94262581E090E0DF91CF9108952F92A1
:10A3D0003F924F925F926F927F928F929F92AF9235
:10A3E000BF92CF92DF92EF92FF920F931F93CF9382
:10A3F000DF93CDB7DEB7C955D1090FB6F894DEBFEC
:10A400000FBECDBF0E949DA29B01AC016091E606EC
:10A410007091E7068091E8069091E906A12CB12C95
:10A42000650110E3E12E15E7F12E00E010E00E9437
:10A43000342A882309F401C2E0918A08F0918B083C
:10A44000309709F4FAC1809186088F5F809386085F
:10A450002680378010E02114310409F434C1F10161
:10A4600080858F708530F9F460E0C1010E944A95C3
:10A47000FC0181859285A385B4850597A105B10569
:10A4800091F4B101CE0101960E942D23CE010196D7
:10A490000E94901366968FAF6697811108C0CE0117
:10A4A00001960E94B713F10122803380D4CF259604
:10A4B0001CAE1DAE1EAE1FAE259729961CAE1DAE5E
:10A4C0001EAE1FAE299740E052E0BE016F5F7F4F86
:10A4D000CE018F5B9F4F0E946933CE0101960E948F
:10A4E000681B6B017C0169966FAF69976A96DFAE56
:10A4F0006A9770E060E0CE0101960E94841B4C01D7
:10A50000CE018F5B9F4F0E94271365966CAF7DAF86
:10A510008EAF9FAF6597CE0101960E94A51C182FA4
:10A52000B601DD0C880B990B0E9468CE20E030E06C
:10A5300048EC52E40E94C1D02B013C01CE010196AF
:10A540000E94BD4F68969FAF8EAF68976DEC72E129
:10A5500085E19FE00E94958265966CAD7DAD8EADE4
:10A560009FAD65970E94FB9C67EC72E185E19FE0DF
:10A570000E949582C301B2010E94FB9C61EC72E1D2
:10A5800085E19FE00E949582612F70E085E19FE068
:10A590000E945E95E114F10409F48EC088E00E94E7
:10A5A00064179B01AC0144275527B70190E080E078
:10A5B000AA24AA94BA2CC12CD12C17E2E12E19E0BE
:10A5C000F12E00E010E00E94342A882371F1F1019D
:10A5D000608171818EEE9DE00E942F8261EB72E1BD
:10A5E0008EEE9DE00E949582F1016081718189E18A
:10A5F00095E00E9486A390E080E0BC0169964FAD93
:10A6000069976A965FAD6A97CE0101960E942625EA
:10A6100062E070E0C4010E94331ACE0101960E94EC
:10A62000B71366961FAD66973ECF20E030E048E155
:10A6300052E4C301B2010E9469D118163CF4F10141
:10A640006081718185E295E00E9486A368968EAD57
:10A650009FAD6897892B19F461E070E0DBCF20E0B3
:10A6600030E040E85FE365966CAD7DAD8EAD9FADAB
:10A6700065970E9454D09B01AC01C301B2010E94B6
:10A6800061CE70E060E087FDC5CFA30192016596C1
:10A690006CAD7DAD8EAD9FAD65970E9461CE1816F5
:10A6A000DCF662EA72E185E19FE00E94958285E135
:10A6B0009FE00E949E81B1CF68E972E185E19FE051
:10A6C0000E949582AACF8091860881508093860847
:10A6D0000E949DA26093E6067093E7068093E806C9
:10A6E0009093E9060E9470112B013C010E949DA2EB
:10A6F0006B017C010E94F094882309F466C080916C
:10A700001408811162C030E020E041E050E060E4D4
:10A71000CE0101960E94292D40E450E068EC78E1DA
:10A72000CE0101960E941AC764EE74E0CE01019634
:10A730000E9481D440E450E06FE672E1CE010196C0
:10A740000E941AC7B301A201CE018F5B9F4F0E94E6
:10A75000DB10BE016F5B7F4FCE0101960E946BA3A1
:10A7600030E020E041E050E060E4CE0101960E943C
:10A77000292D40E450E068EC78E1CE0101960E947A
:10A780001AC764EE74E0CE0101960E9481D440E4C1
:10A7900050E068E672E1CE0101960E941AC7C70137
:10A7A000B60128EE33E040E050E00E94ABCFBA01A2
:10A7B000A901CE018F5B9F4F0E94DB10BE016F5B32
:10A7C0007F4FCE0101960E946BA3112309F44FC065
:10A7D00062E972E185E19FE00E9495820E9470111A
:10A7E000AB01BC012AE085E19FE00E9452816AE84A
:10A7F00072E185E19FE00E94958260918608062EB5
:10A80000000C770B85E19FE00E945E9568E772E19E
:10A8100085E19FE00E9495824091E2065091E30617
:10A820006091E4067091E5062AE085E19FE00E94D0
:10A83000528185E19FE00E949E81C75ADF4F0FB68B
:10A84000F894DEBF0FBECDBFDF91CF911F910F9166
:10A85000FF90EF90DF90CF90BF90AF909F908F9040
:10A860007F906F905F904F903F902F90089568E891
:10A8700072E185E19FE00E9495820E947011AB0118
:10A88000BC012AE085E19FE00E94528160E872E10C
:10A89000B0CF8F929F92AF92BF92CF92DF92EF9202
:10A8A000FF920F931F93CF93DF93CDB7DEB76797D8
:10A8B0000FB6F894DEBF0FBECDBF8C017B014C01FB
:10A8C0008BE0880E911C9F8A8E8AF8011286118671
:10A8D0001386168A158A672B09F463C0A0908A082C
:10A8E000B0908B08A114B10409F45BC06FE270E072
:10A8F000C7010E948CD46C01892B09F44AC0F7016E
:10A90000DE01119690E080E0BD012191222341F00B
:10A910002F3231F08431910519F02D930196F5CF46
:10A92000860F971FFC011082C5010E94D594F80183
:10A9300091838083B6016F5F7F4F4AE050E0C4018E
:10A940000E94C5D4CE0146960E944041F801968BE4
:10A95000858B8E899F89892B09F41386C8010E94F3
:10A960009013882319F0C8010E94C72167960FB67B
:10A97000F894DEBF0FBECDBFDF91CF911F910F9135
:10A98000FF90EF90DF90CF90BF90AF909F908F900F
:10A990000895B701C5010E94D594F8019183808381
:10A9A000DDCFF80111821082D9CF2F923F924F92C2
:10A9B0005F926F927F928F929F92AF92BF92CF924F
:10A9C000DF92EF92FF920F931F93CF93DF93CDB758
:10A9D000DEB7C955D1090FB6F894DEBF0FBECDBFA3
:10A9E0003C01562E6296EFAE62976396FFAE639778
:10A9F00064960FAF649765961FAF659766962FAF05
:10AA0000669767963FAF679768964FAF6897699666
:10AA10005FAF69976A96CFAE6A972D2C4A2C3B2C74
:10AA2000009709F45CC1FC0180858295807F859543
:10AA3000859585958595843009F43CC12CF488234F
:10AA400009F441C180E02DC0853009F444C086304E
:10AA5000C9F762E375E0C3010E94D5944C010097E9
:10AA600009F46FC0B12CA12CD12CC12C6296EFAC93
:10AA700062976396FFAC639764960FAD6497659693
:10AA80001FAD659766962FAD669767963FAD679742
:10AA900068964FAD689769965FAD6997652D0E947E
:10AAA000D554C75ADF4F0FB6F894DEBF0FBECDBFE7
:10AAB000DF91CF911F910F91FF90EF90DF90CF909A
:10AAC000BF90AF909F908F907F906F905F904F90CE
:10AAD0003F902F900895809186088F5F809386081D
:10AAE000868097808114910431F1A42CB32C6A964E
:10AAF000CFAC6A97D22C6296EFAC62976396FFACAC
:10AB0000639764960FAD649765961FAD65976696DB
:10AB10002FAD669767963FAD679768964FAD68977C
:10AB200069965FAD6997652DC4010E94D554F40103
:10AB300082809380D7CF8091860881508093860849
:10AB400081CF66E375E0C3010E94D5947C016BE37D
:10AB500075E0C3010E94D5946C01552039F0F1E0F5
:10AB60005F1609F488C010E000E00CC060E475E0F6
:10AB7000C3010E94D5944C0165E475E0C3010E94B5
:10AB8000D5948C018114910409F443010115110538
:10AB900009F48301E114F10421F46A96EFAC6A9799
:10ABA000F22CC114D10411F4C42CD32C81149104BF
:10ABB00009F492C0F40180858F70843009F08CC054
:10ABC000818492840115110509F491C0F8018085F2
:10ABD0008F70843009F08BC001851285E114F10477
:10ABE00009F4C9C08114910409F490C068EE76E1BB
:10ABF00085E19FE00E949582F7016185728585E17C
:10AC00009FE00E942F8263EE76E185E19FE00E9443
:10AC10009582B40185E19FE00E942F8285E19FE04B
:10AC20000E949E81CE018F5A9F4F0E940E32C11406
:10AC3000D10409F0F8C0F70180858F70843009F0E5
:10AC4000F0C061857285CE0101960E944954CE0103
:10AC500001960E949013882349F08114910409F40D
:10AC600069C0B401CE0101960E94639ACE0101969B
:10AC70000E94B713D6C06AE475E0C3010E94D59460
:10AC80004C016FE475E0C3010E94D5948C018114DE
:10AC9000910409F0CDC060E475E0C3010E94D59431
:10ACA0004C010115110509F467CF892B09F072CF0A
:10ACB000430170CF10E000E0912C812CD12CC12CED
:10ACC000F12CE12C5FCF10E000E0912C812CD12CF5
:10ACD000C12CF12CE12C5ECF912C812C73CFCA2C8E
:10ACE000DB2C6A96EFAC6A97F22C912C812C00E059
:10ACF00020E033E040E150E0BE016F5B7F4FCE01CA
:10AD00008F5A9F4F0E94E11F8C0168CF69ED76E159
:10AD100085E19FE00E949582F7016185728585E15A
:10AD20009FE00E942F8264ED76E185E19FE00E9422
:10AD3000958278CFCC24C394F12CE12C62960FAD90
:10AD4000629763961FAD639764962FAD649765967F
:10AD50003FAD659766964FAD669767965FAD67970F
:10AD600068966FAD689769967FAD6997CE01019639
:10AD70000E9474417BCFC114D10409F452C0011563
:10AD8000110509F44EC0F60180858F70843009F0FA
:10AD900044C06DEC76E185E19FE00E949582F6016A
:10ADA0006185728585E19FE00E942F8268EC76E1E3
:10ADB00085E19FE00E949582B80185E19FE00E94B5
:10ADC0002F8285E19FE00E949E81F6016185728558
:10ADD00040E450E0CE0101960E94C5D40E94F09458
:10ADE0008823D9F080911408811117C06FE270E0B8
:10ADF000CE0101960E948CD4892B51F4F601218555
:10AE0000328543E050E060E4CE0101960E94292D96
:10AE1000B801CE0101960E946BA3E114F10409F080
:10AE20000ACF81E03ECE0115110509F0ACCF03CF6A
:10AE3000892B09F0AFCEA0CE2F923F924F925F9216
:10AE40006F927F928F929F92AF92BF92CF92DF923A
:10AE5000EF92FF920F931F93CF93DF93CDB7DEB79F
:10AE6000E2970FB6F894DEBF0FBECDBF9AA389A3B9
:10AE7000098F1A8F2B8F3C8F4D8F5E8F6F8F78A32A
:10AE8000FAAAE9AADC011496ED91FC91309709F435
:10AE9000D8C06680778018AA1FA61AA619A6312CDA
:10AEA000212C912C812C512C412C6114710409F41A
:10AEB000D0C065EC74E0C3010E94D5945C0166EDDE
:10AEC00074E0C3010E94D5949EA38DA3A114B10484
:10AED00009F4AFC0892B09F4ACC0F50180858F70EF
:10AEE000823009F0A6C0ADA1BEA118968C918F70DA
:10AEF000823009F09EC064E575E0C3010E94D594DC
:10AF0000DC0119962D913D914D915C911C972BA7D9
:10AF10003CA74DA75EA7E9A9FAA9309709F459C043
:10AF2000D301CD90DC90BF01C6010E9497D4892B3C
:10AF300009F04FC0098D002309F1802F90E0B0E0A7
:10AF4000A0E0EDA1FEA181879287A387B4878091BD
:10AF5000880890918908059789F0E12CFF24F394E3
:10AF60001A8D2B8D3C8D4D8D5E8D6F8D78A1A9A195
:10AF7000BAA112968D919C910E948F341A8D812FC7
:10AF8000807F39F160E0CE0149960E945A12092E65
:10AF9000000CAA0BBB0BF50181879287A387B487AE
:10AFA0008091880890918908059799F0D301CD90F8
:10AFB000DC90E12C92E0F92E098D2B8D3C8D4D8D8E
:10AFC0005E8D6F8D78A1E9A1FAA1828193810E94A3
:10AFD0008F34D50119964D915D916D917C911C979F
:10AFE000EDA1FEA181859285A385B4850297A10577
:10AFF000B10521F12BA53CA5429FC001439F900DB7
:10B00000529F900D1124480E591EABA5BCA58A0E67
:10B010009B1EEFA5F8A98F01FF0F220B330B04171E
:10B020001507260737072CF458AB4FA79AA789A70F
:10B030001D01D30112966D907C9037CF90E080E097
:10B04000E4CF1AA619A6312C212C912C812C512C3D
:10B05000412C8114910409F486C0C201B4010E94FC
:10B0600022D07B0169EB75E185E19FE00E9495822A
:10B07000B40185E19FE00E945E956EEA75E185E18D
:10B080009FE00E9495820FEF10E0C201B8010E947C
:10B0900022D085E19FE00E945E9567EA75E185E137
:10B0A0009FE00E949582B70185E19FE00E945E9536
:10B0B00069E975E185E19FE00E94958289A59AA5DD
:10B0C000B8010E9422D085E19FE00E945E9562E96E
:10B0D00075E185E19FE00E949582B10185E19FE0E5
:10B0E0000E945E956EE875E185E19FE00E94958281
:10B0F00085E19FE00E949E8119821A821B821C8238
:10B100001D821E821F8218868A818F708A83B701F2
:10B11000CE0101960E94251279018A013B014C0162
:10B12000298BFA8A4B8B1C8B6D8B7E8A8F8B988E2A
:10B1300067E576E0E9A1FAA1848195810E94D59422
:10B14000B12CA12CD12CC12C9301A4016FEF0E9432
:10B15000D554A9A1BAA11496ED91FC913097E9F4C8
:10B1600088248394912CC401E2960FB6F894DEBF34
:10B170000FBECDBFDF91CF911F910F91FF90EF9048
:10B18000DF90CF90BF90AF909F908F907F906F9007
:10B190005F904F903F902F90089586809780910107
:10B1A000330C440B550B29A33AA34BA35CA389A5ED
:10B1B0009AA5092E000CAA0BBB0B8DA39EA3AFA3CF
:10B1C000B8A78114910461F264E575E0C4010E949E
:10B1D000D5947C016CE374E0C4010E94D5943C01D9
:10B1E00065EC74E0C4010E94D5945C0166ED74E0E6
:10B1F000C4010E94D5946114710409F4B6C0A1146D
:10B20000B10409F4B2C0009709F4AFC0D301189695
:10B210002C912F70223009F0A8C0F50120852F70E5
:10B22000223009F0A2C0DC0118962C9118972F70DB
:10B23000223009F09AC0F701C184D284E384F484F7
:10B24000C114D10409F491C019968D919D910D906E
:10B25000BC91A02D0297A105B10509F48AC029A5CA
:10B260003AA5232B09F485C0D50119968D919C919F
:10B270008C9D50018D9DB00C9C9DB00C11242FEF26
:10B2800030E0D5010E944DD09601DD0C440B550BEA
:10B290000E94CDCF69A17AA18BA19CA10E949BCFD6
:10B2A0002DA13EA14FA158A50E94CDCF19012A0181
:10B2B000F4016081718185E19FE00E942F8266E543
:10B2C00075E085E19FE00E942F82C5016FEF70E07D
:10B2D0000E9422D085E19FE00E945E9568E875E1BA
:10B2E00085E19FE00E9495822AE030E0B201A10151
:10B2F00085E19FE00E94A98185E19FE00E949E81F7
:10B30000F30181859285A385B48582159305A405F3
:10B31000B50559F119861A861B861C861D861E8660
:10B320001F86188A8A858F708A87B101CE01099697
:10B330000E94251229833A834B835C836D837E832D
:10B340008F839887B12CA12CD12CC12C79018A0133
:10B350009B01AC016FEFC4010E94D554D301199633
:10B360002D923D924D925C921C97F40182809380C5
:10B3700028CF212C312C2101C3CF6F927F928F9245
:10B380009F92AF92BF92CF92DF92EF92FF920F9374
:10B390001F93CF93DF93CDB7DEB7A0970FB6F89486
:10B3A000DEBF0FBECDBF8C01862E7A01DC018D91F0
:10B3B0009C911197892B09F460C01496ED91FC9132
:10B3C000309709F45AC080818071BFEF6B1357C06A
:10B3D000B1F481E0A0960FB6F894DEBF0FBECDBFEA
:10B3E000DF91CF911F910F91FF90EF90DF90CF9061
:10B3F000BF90AF909F908F907F906F900895433053
:10B40000510539F3818082942FE0822264EE76E048
:10B4100085E19FE00E949582D80113966C9185E1A9
:10B420009FE00E94579562EE76E085E19FE00E94E2
:10B430009582D8011496ED91FC9161816F7085E140
:10B440009FE00E9457956FED76E085E19FE00E94B6
:10B450009582682D85E19FE00E94579585E19FE0E8
:10B460000E949E81D8011496ED91FC9181818F708C
:10B47000881207C080818F7E808380E0ABCF8111EE
:10B48000FCCF198E1A8E1B8E1C8E1D8E1E8E1F8E4B
:10B4900018A28A8D8F708A8FD8011496ED91FC9135
:10B4A00081818F70881579F1B3E0EB16F10459F1C1
:10B4B0006DED76E085E19FE00E949582F801638161
:10B4C00085E19FE00E9457956BED76E085E19FE076
:10B4D0000E949582D8011496ED91FC9161816F7064
:10B4E00085E19FE00E94579568ED76E085E19FE059
:10B4F0000E949582682D85E19FE00E94579585E125
:10B500009FE00E949E81F80120813181FCE0F815C6
:10B5100008F416C1E82DF0E08827EE56F54A8F4F63
:10B520000C9436D09F5ADC5A5D5B745B805B5D5B2C
:10B53000365B5D5B835B8E5B4A5B915B9D5BD80199
:10B540001496CD90DC90F60181818F70853009F4DE
:10B55000F7C050F48230C1F06AE675E0C9010E947C
:10B56000D5943C01912C4BC08730D1F08A30A1F7A3
:10B5700063E675E0C9010E94D5943C01D6019C9018
:10B5800092FA992490F83BC06DE575E0C9010E94DC
:10B59000D5943C01D6019C9090FA992490F82FC044
:10B5A0006CE575E0C9010E94D5943C01F6019080DC
:10B5B00091FA992490F823C06FE675E0C9010E94C2
:10B5C000D5943C01D8011496ED91FC91808180FBCB
:10B5D000992490F8982F9E7F80FF9160908361144A
:10B5E000710469F461E0CE0149960E946D34298BA3
:10B5F0003A8B4B8B5C8B6D8B7E8B8F8B988FF8018E
:10B60000A080B18066E375E0C5010E94D5946C010D
:10B610006BE375E0C5010E94D5945C01892B81F430
:10B62000C114D10469F460E0CE0149960E946D34E2
:10B6300029833A834B835C836D837E838F839887D2
:10B64000D8011496ED91FC916114710409F07CC04D
:10B65000898D811179C0B82DBF708B2E8181807F3B
:10B66000882A818280818F7E8083B3CE64E775E0F3
:10B67000C9010E94D5943C01D8011496ED91FC912A
:10B68000808181FB992490F8982F9D7F81FF9260A3
:10B690009083B5CF6AE775E0C9010E94D5943C015B
:10B6A000D8011496ED91FC91808182FB992490F849
:10B6B000982F9B7F82FF9460EBCF6AE675E0C9010B
:10B6C0000E94D5943C01892B09F04CCF62E0CE0159
:10B6D00049960E946D3429873A874B875C876D872E
:10B6E0007E878F87988B3ECF60E875E0C9010E9406
:10B6F000D5943C01D8011496ED91FC9190804CCFEB
:10B7000065E875E0F3CF6BE875E0C9010E94D59458
:10B710003C01D8011496ED91FC9149CF61E975E0A7
:10B72000F4CF68E975E0C9010E94D5943C01D801C5
:10B730001496ED91FC91908023CF6EE975E0F3CFE4
:10B74000912C712C612C5BCF83E0E816F104B9F0E9
:10B75000982D9F70892E8181807F882A81828081A7
:10B760008F7E8083E98CFA8C0B8D1C8D2D8D3E8D08
:10B770004F8D58A1692DC3010E94D5542ACE8181D5
:10B780008F70881509F425CE829490EF8922882A3B
:10B7900081828081806168CF8F929F92AF92BF92A9
:10B7A000CF92DF92EF92FF920F931F93CF93DF938D
:10B7B000CDB7DEB767970FB6F894DEBF0FBECDBF2B
:10B7C0006115710599F1FA017B018C01E60FF71FF4
:10B7D00010820E9470114B016DEE7AE085E19FE0CE
:10B7E0000E949582B40185E19FE00E945E956AEE19
:10B7F0007AE085E19FE00E949582B80185E19FE0B3
:10B800000E942F8267EE7AE085E19FE00E94958298
:10B810008AEF88169104ECF46AED7AE08EEE9DE0F2
:10B820000E9495828EEE9DE00E949E8167960FB6E3
:10B83000F894DEBF0FBECDBFDF91CF911F910F9166
:10B84000FF90EF90DF90CF90BF90AF909F908F9040
:10B850000895B70185E19FE00E942F8285E19FE076
:10B860000E949E81809188089091890863E070E031
:10B87000059749F062E070E0C8010E94BD2D009775
:10B8800081F461E070E0C8010E94BD2D009749F489
:10B890006FEC7AE085E19FE00E94958285E19FE070
:10B8A000C3CF080F191F65EA75E0C8010E9497D43D
:10B8B000892B69F4F70101900020E9F73197EE191F
:10B8C000FF09329720F0C7010E94D287AFCFF8015D
:10B8D0008081843209F4AACFB801CE0101960E947A
:10B8E0004954CE0101960E949013882329F0B70194
:10B8F000CE0101960E94639ACE0101960E94B71371
:10B9000095CF3F924F925F926F927F928F929F92CC
:10B91000AF92BF92CF92DF92EF92FF920F931F935D
:10B92000CF93DF93CDB7DEB7CE56D1090FB6F894DB
:10B93000DEBF0FBECDBFDC0114962D913C91232BB1
:10B9400009F419C69B01225031092230310508F053
:10B9500091C23B014C01FC018281803409F4F7C2A1
:10B9600008F04AC0843008F085C28091D3068F5F0A
:10B970008093D306A3016FEFC4010E94BD59D40187
:10B9800012960C9112970695017013961C911397BD
:10B990008AEC810F803108F043C06EEA75E08D912A
:10B9A0009C910E94D5947C010097D1F1FC01808587
:10B9B0008F708530A9F580915E0D181324C0809199
:10B9C0005F0D803401F58091600D9091610D5C01F7
:10B9D000990FCC08DD0860E0C7010E944A95FC0180
:10B9E00081859285A385B485A816B906CA06DB06AB
:10B9F0000CF065C0512C3EC0823409F4A8C208F492
:10BA000039C28058AFCF10935E0D80E480935F0DF4
:10BA1000812F0E9426A29093610D8093600DD7CF55
:10BA2000212F30E0F901E65EF34E8491F901EC53E9
:10BA3000F44E1491F901E259F44EF490FF2009F408
:10BA40003BC081110E947EA0EF2DF0E0EE0FFF1FA2
:10BA5000E254F94FA591B491EC911E2331E020E01E
:10BA600009F430E0832F922F5524539408171906B8
:10BA700009F0C0CFF3E06F16710409F488C0D40157
:10BA80001496ED91FC91E181EF70E150EC3008F0FB
:10BA90007EC0F0E08827E05BF24A8F4F0C9436D0EE
:10BAA000715DED5EA75DDD5DED5EF65DED5E2A5ECE
:10BAB000575E705EB25ED45E90E080E0D5CF61E00C
:10BAC000C7010E944A9555245394FC0181859285B3
:10BAD000A385B4858A159B05AC05BD050CF0CACFBE
:10BAE00089CF0E949DA29B01AC0144275527D40118
:10BAF0001496ED91FC916281738190E080E0AA241C
:10BB0000AA94BA2CC12CD12C18EEE12E13E0F12E00
:10BB100000E010E00E94342A8823C9F1F40100817A
:10BB2000118160E875E0C8010E94D594892B41F429
:10BB300065E875E0C8010E94D594892B09F40EC10F
:10BB400042E050E063E0C4010E94BD5920C00E9461
:10BB50009DA29B01AC0144275527D4011496ED9179
:10BB6000FC916281738190E080E0AA24AA94BA2CAF
:10BB7000C12CD12C1CE2E12EFF24F39400E010E054
:10BB80000E94342A42E050E064E0811184C0D40174
:10BB90001496ED91FC91808183FB992790F995157E
:10BBA00009F4D2C1982F907E09F439C1982F907E64
:10BBB00090528F71892B808358C10E949DA29B0156
:10BBC000AC0144275527D4011496ED91FC91628174
:10BBD000738190E080E0AA24AA94BA2CC12CD12CC5
:10BBE00016E9E12EF12C00E010E0CACF0E949DA2E0
:10BBF0009B01AC0144275527D4011496ED91FC918B
:10BC00006281738190E080E0AA24AA94BA2CC12CAE
:10BC1000D12C18EEE12E13E0F12E00E010E00E948E
:10BC2000342A882309F4B3CFF401008111816BE831
:10BC300075E0C8010E94D594892B41F461E975E053
:10BC4000C8010E94D594892B09F488C042E050E0D5
:10BC500068E079CF0E949DA29B01AC014427552743
:10BC6000D4011496ED91FC916281738190E080E0A3
:10BC7000AA24AA94BA2CC12CD12C1CE2E12EFF24B8
:10BC8000F39400E010E00E94342A42E050E069E0C2
:10BC9000882309F47CCFC4010E94BD590E949DA253
:10BCA000D4011496ED91FC917383628370CF0E944E
:10BCB0009DA29B01AC0144275527D4011496ED9118
:10BCC000FC916281738190E080E0AA24AA94BA2C4E
:10BCD000C12CD12C16E9E12EF12C00E010E0D3CFDD
:10BCE0000E949DA29B01AC0144275527D4011496C4
:10BCF000ED91FC916281738190E080E0AA24AA9486
:10BD0000BA2CC12CD12C18EEE12E13E0F12E00E05C
:10BD100010E00E94342A882309F439CFF40100810D
:10BD2000118168E975E0C8010E94D594892B39F426
:10BD30006EE975E0C8010E94D594892B21F042E09C
:10BD400050E06BE000CF6AE775E0C8010E94D5942F
:10BD500042E050E066E0892B09F4F5CE42E050E085
:10BD60006DE0F1CE0E949DA29B01AC0144275527B6
:10BD7000D4011496ED91FC916281738190E080E092
:10BD8000AA24AA94BA2CC12CD12C1CE2E12EFF24A7
:10BD9000F39400E010E00E94342A882309F4F7CEDF
:10BDA00042E050E06CE077CF0E949DA29B01AC0185
:10BDB00044275527D4011496ED91FC91628173813B
:10BDC00090E080E0AA24AA94BA2CC12CD12C16E9C8
:10BDD000E12EF12C00E010E0DECF0E949DA29B013D
:10BDE000AC0144275527D4011496ED91FC91628152
:10BDF000738190E080E0AA24AA94BA2CC12CD12CA3
:10BE000018E5E12E12E0F12E00E010E00E94342A45
:10BE1000882309F4BCCE42E050E060E094CE0E945A
:10BE20009DA2D4011496ED91FC91159773836283C2
:10BE3000E181EF70552009F445C0E230F1F050F493
:10BE4000EE23E9F1D4011496ED91FC91808150FA32
:10BE500083F9B1CEE53089F0A3016AE0E73091F7CC
:10BE6000C4010E94BD598111EDCF8091D30681504C
:10BE70008093D30690E080E080C3F40100811181BB
:10BE800064E775E0C8010E94D594892BA9F46BE89A
:10BE900075E0C8010E94D594892B71F461E975E0C1
:10BEA000C8010E94D594892B39F46CE575E0C8016E
:10BEB0000E94D594892B19F0A30166E0D1CFA3018C
:10BEC00061E0CECFE150ED3008F0BCCFF0E0882744
:10BED000E359F04A8F4F0C9436D07A5F225F7D5F32
:10BEE0007D5F225F805F225FA15FA15FA15FA15F95
:10BEF000A15F7D5FA30162E0B3CFA30165E0B0CF96
:10BF00000D911C9164E775E0C8010E94D594892BBE
:10BF1000A9F46BE875E0C8010E94D594892B71F4EF
:10BF200061E975E0C8010E94D594892B39F46CE56C
:10BF300075E0C8010E94D594892B19F0A30167E030
:10BF40008FCFA30160E08CCF8F71806434CEB3E0DB
:10BF50006B16710409F48ECF6EEA75E0F4018081EE
:10BF600091810E94D5948C01D40113968C9190916B
:10BF70005E0D8913EBC090915F0D903409F0E6C01F
:10BF80008091600D9091610D3C010115110509F43E
:10BF90000DC1F80120852F70253009F007C1C801B7
:10BFA0000E946695382EF3E0F81708F0DBC063E0D6
:10BFB000C8010E944A95DC0119968D919C913AE046
:10BFC000E32EE89E6001E99ED00C1124A396DFAE1B
:10BFD000CEAEA39762E0C8010E944A95DC01199693
:10BFE0008D919C91E89E2001E99E500C11246201E4
:10BFF000052C000CEE08FF08AF96CCAEDDAEEEAE21
:10C00000FFAEAF9761E0C8010E944A955C0160E015
:10C01000C8010E944A95DC011996CD90DD90ED9003
:10C02000FC901C97A796CCAEDDAEEEAEFFAEA79708
:10C030009301072C000C440B550B2C193D094E099C
:10C040005F09A396CEACDFACA397B601DD0C880BDD
:10C05000990BAF96CCACDDACEEACFFACAF976C19E6
:10C060007D098E099F090E949BCFD50119962D91BC
:10C070003D914D915C911C97A796CCACDDACEEAC9C
:10C08000FFACA7972C193D094E095F09A7962CAF65
:10C090003DAF4EAF5FAFA7970E94CDCFAF96ACAC90
:10C0A000BDACCEACDFACAF97A20EB31EC41ED51E86
:10C0B00045E0E42E3E1409F468C081E090E0A396C8
:10C0C000EEACFFACA397A701FF0C660B770B4A15EC
:10C0D0005B056C057D050CF461C0B601A50162012C
:10C0E000052C000CEE08FF084C155D056E057F055C
:10C0F0000CF459C06A017B0122E032126BC063016B
:10C10000770CEE08FF0860E0C8010E944A95FC0128
:10C1100081859285A385B485C816D906EA06FB06F3
:10C120000CF444C261E0C8010E944A95FC0181857B
:10C130009285A385B4858C159D05AE05BF050CF0D1
:10C1400099CE81E090E0A0E0B0E033C280935E0D34
:10C1500090E490935F0D0E9426A29093610D8093CE
:10C16000600D12CF8AE0869D5001879DB00C11248E
:10C170000B2C000CCC08DD08512C412C20E038E2BF
:10C18000A3963FAF2EAFA39798CF64E0C8010E945B
:10C190004A95DC0119968D919C9191CF66246A9401
:10C1A00023E0722E9CCF712C612CA6CF2AE0289F11
:10C1B0006001299FD00C11240D2C000CEE08FF0803
:10C1C000512C412C20E038E2A3963FAF2EAFA3972D
:10C1D00081E090E0D4011496ED91FC91428153816D
:10C1E0009301241B350B37FF03C03195219531098D
:10C1F000821793070CF4BFC08081982F9295969573
:10C200009770963008F0BAC09F5F9295990F907E14
:10C210008F71892BB2C0F70161857285DB018C912A
:10C22000811154C2A114B10409F472C0D501189649
:10C230008C9118978F70843009F06AC019966D91AF
:10C240007C91CE0101960E944954CE0101960E9434
:10C250009013882309F458C06114710409F45FC075
:10C26000E114F10431F0F70180858F70843009F416
:10C2700041C025961CAE1DAE1EAE1FAE2597299659
:10C280001CAE1DAE1EAE1FAE299723961FAD239781
:10C290001F7023961FAF239781E022968FAF2297BE
:10C2A000CC24C394F12CE12C01E024962FAD2497EB
:10C2B00025963FAD259740E027965FAD27972896B6
:10C2C0006FAD289729967FAD2997CE0101960E94E0
:10C2D00074411AC00115110529F0F80180858F708D
:10C2E000843019F06FE774E0F1C161857285FB015C
:10C2F000808196CF61857285FB018081882321F042
:10C30000CE0101960E94639ACE0101960E94B71356
:10C31000D4011496ED91FC9173826282ABCD01152C
:10C32000110531F0D80118968C918F708430E9F0A6
:10C3300025961CAE1DAE1EAE1FAE259729961CAECF
:10C340001DAE1EAE1FAE299723961FAD23971F70FB
:10C3500023961FAF239782E022968FAF2297CC249B
:10C36000C394F12CE12C02E0A0CFF8016185728525
:10C37000DB018C91C3CF80818F7180838081803A73
:10C38000B8F0C201550CAA0BBB0BC816D906EA06B9
:10C39000FB0671F0A396EEADFFADA397CF01FF0FA3
:10C3A000AA0BBB0BC816D906EA06FB0609F062CD3C
:10C3B0006416750609F45ECD6D961CAE1DAE1EAEFC
:10C3C0001FAE6D976B968FAD6B978F7080666B9677
:10C3D0008FAF6B976D968CAD9DADAEADBFAD6D97CC
:10C3E00065968CAF9DAFAEAFBFAF65976996CCAE8B
:10C3F000DDAEEEAEFFAE69976DEA76E085E19FE0D7
:10C400000E949582D40113966C9185E19FE00E9471
:10C4100057956BEA76E085E19FE00E949582CE0118
:10C420008F5A9F4F0E940E3262E375E0F4018081C3
:10C4300091810E94D594B12CA12CD12CC12C629653
:10C44000EFAC62976396FFAC639764960FAD649709
:10C4500065961FAD659766962FAD669767963FAD5B
:10C46000679768964FAD689769965FAD69976FEF6C
:10C470000E94D554D4010D911C9166E375E0C8016A
:10C480000E94D5947C016BE375E0C8010E94D594AD
:10C490008C010097E1F1FC0180858F708430B9F543
:10C4A0006185728540E450E0CE0101960E94C5D4BA
:10C4B0006FE270E0CE0101960E948CD4892B59F472
:10C4C000D80119962D913C9143E050E060E4CE01F3
:10C4D00001960E94292D00E020E032E040E150E08A
:10C4E000BE016F5B7F4FCE018F5A9F4F0E94E11FAD
:10C4F0000E94F094882359F080911408811107C09C
:10C50000BE016F5B7F4FCE0101960E946BA3E114C9
:10C51000F10409F4FDCEF70180858F70843009F0B5
:10C52000F7CE61857285CE0101960E944954CE01F5
:10C5300001960E949013882309F4E6CECC24C3947C
:10C54000F12CE12C62960FAD629763961FAD639755
:10C5500064962FAD649765963FAD659766964FAD2F
:10C56000669767965FAD679768966FAD68976996AF
:10C570007FAD6997AACE8FEF9FEFC259DF4F0FB6FD
:10C58000F894DEBF0FBECDBFDF91CF911F910F9109
:10C59000FF90EF90DF90CF90BF90AF909F908F90E3
:10C5A0007F906F905F904F903F90089580E090E073
:10C5B000DC01F40124813581F90142815381052E8A
:10C5C000000C660B770B84179507A607B70709F4CD
:10C5D00051CC3C01D4010D911C9166E375E0C8017A
:10C5E0000E94D5945C016BE375E0C8010E94D5946C
:10C5F0006C01A114B10419F4892B09F489CE6FE6FA
:10C6000075E0C8010E94D5947C016AE675E0C80116
:10C610000E94D5948C0163EB76E085E19FE00E9457
:10C620009582F401638185E19FE00E94579561EB5B
:10C6300076E085E19FE00E949582B30185E19FE06D
:10C640000E945E9585E19FE00E949E81C114D10405
:10C6500009F4E8CDD60118968C9118978F70843024
:10C6600009F0E0CD19966D917C9140E450E0CE0147
:10C6700001960E94C5D40E94F094882309F4D2CD7B
:10C68000809114088111CECD6FE270E0CE01019649
:10C690000E948CD4892B51F4F6012185328543E028
:10C6A00050E060E4CE0101960E94292D61147104CE
:10C6B00009F410CEE114F10439F0D70118968C91E9
:10C6C0008F70843009F4A7CD6CE774E0CE01019639
:10C6D0000E946BA3A7CD8F929F92AF92BF92CF92F1
:10C6E000DF92EF92FF920F931F93CF93DF9300D0CF
:10C6F00000D0CDB7DEB72091EA063091EB06232BB0
:10C7000009F4C5C02091DD062111C1C04C01809102
:10C71000DD068F5F8093DD06809186088F5F8093B2
:10C7200086080E949DA29B01AC016091D906709180
:10C73000DA068091DB069091DC06A12CB12C650114
:10C740001BE0E12EF12C00E010E00E94342A882347
:10C7500009F452C0E091EA06F091EB0606811781D8
:10C7600001151105B9F1F80180858F70863071F5DA
:10C7700062E375E0C8010E94D5940097D1F0FC01F6
:10C7800020852F702530A9F4E680F780E114F104AC
:10C79000E9F0FA82E982B801CE0101960E94821A7C
:10C7A000B401CE0101960E94815CF701E280F38022
:10C7B000EDCF1A83098370E060E0CE0101960E94FC
:10C7C000821AB401CE0101960E94815CF8010281B7
:10C7D0001381C6CFF3E08F16910451F00E949DA201
:10C7E0006093D9067093DA068093DB069093DC069B
:10C7F00010925E0D10925F0D83E088169104E9F1AE
:10C800000E949DA29B01AC016091D5067091D60655
:10C810008091D7069091D806A12CB12C650118E81B
:10C82000E12E13E1F12E00E010E00E94342A88236B
:10C8300021F1E091EA06F091EB06068117810115DE
:10C84000110589F0F80180858F70863041F41A83D4
:10C85000098370E060E0CE0101960E94821AF8011F
:10C8600002811381ECCF0E949DA26093D506709344
:10C87000D6068093D7069093D8068091860881507B
:10C88000809386088091DD0681508093DD06269690
:10C890000FB6F894DEBF0FBECDBFDF91CF911F91D1
:10C8A0000F91FF90EF90DF90CF90BF90AF909F904F
:10C8B0008F9008954F925F926F927F92AF92BF9246
:10C8C000CF92DF92EF92FF920F931F93CF93DF935C
:10C8D000CDB7DEB767970FB6F894DEBF0FBECDBFFA
:10C8E0006BE573E185E19FE00E94958285E19FE021
:10C8F0000E949E810E949DA22B013C01809186088E
:10C90000882321F10E949DA29B01AC01A12CB12C96
:10C91000650110E1E12E17E2F12E00E010E0C30105
:10C92000B2010E94342A811111C00E945388809163
:10C93000880890918908059711F00E94364E0E9450
:10C94000E75182E090E00E946B63D8CF8091860827
:10C95000882351F068E373E18EEE9DE00E9495829A
:10C960008EEE9DE00E949E8162E273E185E19FE090
:10C970000E94958285E19FE00E949E818091F00651
:10C980008F5F8093F006E0918A08F0918B083097D2
:10C9900081F1068117810115110559F1D801189609
:10C9A0008C918F708530B9F7C8010E9466958823F5
:10C9B00091F3F80160817181CE0101960E94495482
:10C9C000CE0101960E949013882359F08A859B8599
:10C9D000009739F0DC01ED91FC910284F385E02DA4
:10C9E0001995CE0101960E94B713F80102811381B7
:10C9F000D2CF1092EF061092EE066AE173E185E164
:10CA00009FE00E94958285E19FE00E949E8164E6FE
:10CA100070E080E090E00E946BA2109211081092EA
:10CA2000870862E073E185E19FE00E9495820E94A1
:10CA30007011AB01BC012AE085E19FE00E945281A8
:10CA40008091EC069091ED060E94D09D1092ED062B
:10CA50001092EC061092EB061092EA0610928B08E8
:10CA600010928A08109213081092120810928408EB
:10CA70001092830810928208109281086DEF72E183
:10CA800085E19FE00E9495820E947011AB01BC017C
:10CA90002AE085E19FE00E94528185E19FE00E94AB
:10CAA0009E81109285088091F00681508093F00657
:10CAB00067960FB6F894DEBF0FBECDBFDF91CF9162
:10CAC0001F910F91FF90EF90DF90CF90BF90AF90AC
:10CAD0007F906F905F904F900895809114088F5FC2
:10CAE00080931408A89583E090E00E946B630E94F5
:10CAF0005388809114088150809314080895CF9230
:10CB0000DF92EF92FF92CF93DF93EC018C85883018
:10CB100068F40E944F900E949DA26B017C018C855D
:10CB20000E946B90811109C088E08C87DF91CF91C2
:10CB3000FF90EF90DF90CF9008950E946D6561E0C7
:10CB400070E080E090E00E946BA20E949DA2AB0189
:10CB5000BC014C195D096E097F098D859E85B0E089
:10CB6000A0E0481759076A077B07C8F28C850E9426
:10CB70005D90DACFCF92DF92EF92FF921F93CF9327
:10CB8000DF93EC017B016A018C85883048F40E94B8
:10CB90006B90882319F08C850E944F9088E08C87D9
:10CBA000F70182819381A481B5810097A105B10528
:10CBB00051F490E080E0DF91CF911F91FF90EF90D2
:10CBC000DF90CF9008958F3F9F4FAF4FBF4F89F3B6
:10CBD00070E060E081E20E94A690182F8C87883078
:10CBE00040F780E591E00E94209EA7014E5F5F4FD5
:10CBF00024E030E06CE070E0812F0E945326B60103
:10CC0000812F0E947A9064E070E0812F0E94878BD0
:10CC10000E949DA26B017C018C850E946B908731E4
:10CC200021F18C3111F1882321F20E949DA2AB01E8
:10CC3000BC014C195D096E097F098D859E85B0E0A8
:10CC4000A0E084179507A607B70748F00E946D6516
:10CC500061E070E080E090E00E946BA2DDCF8C8507
:10CC60000E945D9088E08C87A4CF81E090E0A3CF04
:10CC70008F929F92BF92CF92DF92EF92FF920F938B
:10CC80001F93CF93DF93CDB7DEB76D970FB6F894B0
:10CC9000DEBF0FBECDBF8091EC069091ED06892BD3
:10CCA00009F45AC280918608811156C28091860883
:10CCB0008F5F8093860869EF7DE084EE9DE00E949F
:10CCC000958284EE9DE00E949E810091EC06109179
:10CCD000ED0662EB75E0C8010E94D59490938B0835
:10CCE00080938A0868EB75E0C8010E94D594909300
:10CCF00013088093120869E176E0C8010E94D59478
:10CD00009093EB068093EA066FEB75E0C8010E94F2
:10CD1000D59490938408809383080E9439301092B0
:10CD2000EF061092EE06E0918A08F0918B0830979A
:10CD300009F4F2C0E680F78000918A0810918B0810
:10CD40000115110509F4E1C0E114F10409F4DDC095
:10CD5000D70118968C918F70853091F7C7010E948A
:10CD60006695823068F3B701CE0101960E942D23AB
:10CD7000CE0101960E949013882309F464C08A852D
:10CD80009B85009769F570E060E0CE0101960E94F6
:10CD9000841B8C01912C812C97FF06C01195019565
:10CDA000110988248394912CCE0101960E94A51C20
:10CDB000C82ED12C8985853009F44EC0863009F003
:10CDC00042C0B02E61E0802F0E9413A161E089284B
:10CDD00009F479C0CA94CD2809F079C060E077C021
:10CDE000DC01ED91FC910484F585E02D1995892BEA
:10CDF00049F08A859B85DC01ED91FC910284F385E5
:10CE0000E02D19958A859B85DC01ED91FC910680CA
:10CE1000F781E02D1995892BB1F0CE0101960E9482
:10CE2000A51C882331F060E071E0CE0101960E94DC
:10CE3000351C8D819E81892B31F060E072E0CE013E
:10CE400001960E94351CD7011296ED90FC90CE0100
:10CE500001960E94B71370CFCD2829F462E0CE016D
:10CE600001960E94751C60E071E0CE0101960E945F
:10CE7000351C8D819E81892B31F060E072E0CE01FE
:10CE800001960E94351C61E0802F0E9413A160E092
:10CE9000802F0E94E5A061EF7DE085E19FE00E9488
:10CEA0009582B80185E19FE00E945E956CEE7DE081
:10CEB00085E19FE00E9495826AEE7DE085E19FE03A
:10CEC0000E949582C0CFCA94CD2809F087CFC62E84
:10CED000D12C8B2D0E94E5A065EE7DE085E19FE0E1
:10CEE0000E949582B80185E19FE00E945E9563EE05
:10CEF0007DE085E19FE00E949582B60185E19FE09B
:10CF00000E945E9561EE7DE0D9CFF8018681978120
:10CF10009093EF068093EE0685E19FE00E949E814C
:10CF2000E091EA06F091EB06309709F48AC080910F
:10CF300086088F5F80938608068117810115110589
:10CF400009F47AC0D80118968C918F70863009F058
:10CF500069C0198F088F70E060E0CE0148960E948A
:10CF6000821A8C8D9D8D892B09F45CC08091EC0612
:10CF70009091ED06892B09F455C0E88CF98CF701E6
:10CF800080858F70863099F562E375E0C7010E9455
:10CF9000D5940097F1F0DC0118962C9118972F701A
:10CFA0002530B9F41696CD90DC90C114D104F9F077
:10CFB000DA82C982B701CE0101960E94821AED8100
:10CFC000FE811082118212821382F601C280D38008
:10CFD000ECCFFA82E98270E060E0CE0101960E9417
:10CFE000821A62E070E0CE0101960E94815CEC8DB5
:10CFF000FD8D10821182128213828A8D843068F432
:10D0000062E0823008F060E08B8D0E9413A1EC8D0D
:10D01000FD8D8181807F818305C0803441F060E097
:10D02000823431F0D80112960D911C9187CF62E0C5
:10D030008B8D0E9413A1F6CF80918608815080933A
:10D04000860864ED7DE084EE9DE00E9495826CECA4
:10D050007DE084EE9DE00E94958281E020918A0827
:10D0600030918B08232B09F480E00E94BA1763ECFF
:10D070007DE084EE9DE00E94958281E02091EA06A9
:10D080003091EB06232B09F480E00E94BA176CEB79
:10D090007DE084EE9DE00E94958281E020918308EE
:10D0A00030918408232B09F480E00E94BA1763EBC7
:10D0B0007DE084EE9DE00E949582809111080E949F
:10D0C000BA176CEA7DE084EE9DE00E94958281E0D3
:10D0D0002091830830918408232B09F480E00E947A
:10D0E000BA1784EE9DE00E949E8167EA7DE084EE9F
:10D0F0009DE00E9495820E947011AB01BC012AE064
:10D1000084EE9DE00E94528184EE9DE00E949E810B
:10D1100081E08093870882EB9DE00E94B716882308
:10D1200051F082EB9DE00E947F6584E090E0909357
:10D1300089088093880880918808909189080797CA
:10D1400031F484E090E0909389088093880880917E
:10D1500086088150809386086D960FB6F894DEBFDE
:10D160000FBECDBFDF91CF911F910F91FF90EF9038
:10D17000DF90CF90BF909F908F900895EF92FF9295
:10D180000F931F93CF93DF9300D01F92CDB7DEB7DD
:10D190008C017B01FB0184858830A8F089E294E052
:10D1A000F801918380831282138214821582C80150
:10D1B0000F900F900F900F90DF91CF911F910F91D3
:10D1C000FF90EF90089580E591E00E94209E24E07A
:10D1D00030E0AE014F5F5F4F6CE070E0F701848597
:10D1E0000E948227BE016F5F7F4FC8010E94CB82E1
:10D1F000DECFEF92FF920F931F93CF93DF93CDB7C4
:10D20000DEB764970FB6F894DEBF0FBECDBF0D87B3
:10D210001E872F87388B498B5A8B6B8B7C8B68E4EE
:10D2200075E185E19FE00E949582CE010D960E94F6
:10D230000E329E85892F8F70082F10E02D852223B6
:10D2400009F4A6C00115110509F474C0813009F470
:10D2500071C08130A0F18230C1F18E3009F07FC001
:10D2600092959F7069897A899C3011F070E060E036
:10D27000CE0101960E94B58065E376E0C7010E9469
:10D2800097D4892B09F03FC0BE016F5F7F4FCE015D
:10D2900007960E94AC80CE0107960E948B9FBC012E
:10D2A00086E19CE00E948782CE0107960E947980E9
:10D2B00001E010E0CE0101960E94798016C067E37C
:10D2C00075E185E19FE00E94958263E275E185E169
:10D2D0009FE00E94958285E19FE00E949E818E855D
:10D2E000807F01E010E009F400E0C80164960FB609
:10D2F000F894DEBF0FBECDBFDF91CF911F910F918C
:10D30000FF90EF90089565E476E0C7010E9497D4FE
:10D3100000E0892B71F6BE016F5F7F4FCE0107964B
:10D320000E94AC80CE0107960E948B9FBC0189EFC2
:10D330009AE0B8CF213021F1223039F166E175E170
:10D3400085E19FE00E9495826D8585E19FE00E94C6
:10D35000579585E19FE00E949E8101E010E066E024
:10D3600075E185E19FE00E949582B80185E19FE02B
:10D370000E945E9585E19FE00E949E8100E003C0CF
:10D380002093290201E010E0B0CF10922902FACFD9
:10D39000813009F05ECFD2CFAF92BF92CF92DF92B1
:10D3A000EF92FF920F931F93CF93DF93CDB7DEB72A
:10D3B000CA59D1090FB6F894DEBF0FBECDBF8E019A
:10D3C0000F5B1F4FD8011D921C92FE01ED5BFF4FBA
:10D3D0008EE1DF011D928A95E9F78091C10D909150
:10D3E000C20D892B09F49FC10E949F95882309F4DF
:10D3F0009AC1A091C10DB091C20D52961C921E927D
:10D40000519754961C921E92539784E890E01D9673
:10D410009C938E931C971E961C921E9780E090E31F
:10D4200050969C938E931F97ED91FC9111970088D5
:10D43000F189E02D60E270E0CD0119954FE150E0F7
:10D44000B8018091C10D9091C20D0E94F6957C01AA
:10D450008091C10D9091C20DDC01ED91FC91048889
:10D46000F589E02D1995E114F10409F45CC1F80186
:10D47000EE0DFF1D10828091CE0D1F928F93809133
:10D48000CD0D1F928F938091CC0D1F928F93809121
:10D49000CB0D1F928F938091CA0D1F928F93809115
:10D4A000C90D1F928F9384EC95E09F938F931F92E9
:10D4B00080E48F93FE0131966F01FF93EF930E94FA
:10D4C000DFD46CE370E184EE9DE00E949582B801A8
:10D4D00084EE9DE00E942F82B60184EE9DE00E94C2
:10D4E0002F8284EE9DE00E949E817E01F1E6EF0E88
:10D4F000F11CD70113961C921E92129788EE93E0AE
:10D50000A0E0B0E0F70184839583A683B78388E029
:10D51000848788EE93E09687858783EB93E09183F9
:10D520008083108A1786128B018B148A138A80E5F8
:10D5300090E0968B858B118E6BE67FE085E19FE016
:10D540000E94958263EC7DE0CE0185589F4F0E943A
:10D55000AC80BE0165587F4F85E19FE00E948782C5
:10D5600085E19FE00E949E81CE0185589F4F0E94D9
:10D57000798063EF75E0CE0183579F4F0E94B5809D
:10D5800063EF75E0CE0185589F4F0E94B580BE01C4
:10D5900065587F4FCE018B579F4F0E94AC8063EC44
:10D5A0007DE0CE018B579F4F0E941580BE016357CF
:10D5B0007F4F0E941580BC01CE018D569F4F0E9467
:10D5C000AC80CE018B579F4F0E947980CE01855849
:10D5D0009F4F0E947980CE0183579F4F0E94798090
:10D5E00085EF95E0CB57DF4F99838883C558D040AE
:10D5F000C757DF4F19821882C958D040C557DF4F2F
:10D6000019821882CB58D040CD56DF4F888199813E
:10D61000C359D040C957DF4F99838883C758D0403A
:10D6200066E370E185E19FE00E9495820E9470119F
:10D63000AB01BC012AE085E19FE00E94528185E1B7
:10D640009FE00E949E8164E670E080E090E00E948E
:10D650006BA28EE094E7D70150969C938E931F9710
:10D660006FEC7BE781ED9AE80E94E9C78C010FB669
:10D67000F894DEBF0FBECDBF892BA1F183E090E00F
:10D680000E94C9C3D8011D969C938E931C97FC01E0
:10D69000F182E0821282C7010E94B716882319F036
:10D6A000C7010E947F65D70153966D917C91549775
:10D6B0005596AD90BC906115710509F44BC0CE0133
:10D6C00085589F4F0E94CB82A501BE0165587F4FB0
:10D6D000C7010E94BA65181619060CF489C1C80161
:10D6E0000E94AA8A6DEC7FE085E19FE00E9495820E
:10D6F000EE24EA94FE2CCE018D569F4F0E94798035
:10D70000C701C656DF4F0FB6F894DEBF0FBECDBFC0
:10D71000DF91CF911F910F91FF90EF90DF90CF900D
:10D72000BF90AF90089540E250E06EE670E1C8010E
:10D730000E9438C760E570E184EE9DE00E9495820A
:10D74000B80184EE9DE00E942F8284EE9DE00E944D
:10D750009E8191CEF70161897289A501C7010E945E
:10D76000D916B9CF86EC9FE09F938F931F930F93A9
:10D770000E9470C8D70158961C921E925797D801E4
:10D780001C96ED91FC91A080B1800F900F900F90AE
:10D790000F9093E3C92ED12CD501ED91FC9100841B
:10D7A000F185E02DC501199541975CF4B1E0CB1AE4
:10D7B000D10839F064E170E080E090E00E946BA253
:10D7C000EBCF6E01E9E9CE0ED11CDF92CF9286E756
:10D7D0009FE09F938F931F930F930E948DC80F908C
:10D7E0000F900F900F900F900F900197D1F4D601EA
:10D7F0008D919C91F701908F878B67E576E0CE0144
:10D8000083579F4F0E94B58080E0C12CFAE0CF1271
:10D8100072C08A3009F073C0CE0183579F4F0E94B7
:10D820007980D7015796ED90FC90B8ECEB16F10497
:10D8300009F0BCC06AE270E184EE9DE00E9495822E
:10D8400064EF71E080E090E00E946BA2EF961FAE63
:10D850001EAEEF97C158DF4F19821882CF57D040C4
:10D860008FEF9FEFCF57DF4F99838883C158D04008
:10D870008CE093E0ED969FAF8EAFED97CD57DF4FE5
:10D8800019830883C358D040F8948091EC06909196
:10D89000ED06892B11F00E945A64CE0185589F4FE6
:10D8A0000E94029E9093ED068093EC067894C80146
:10D8B0000E94AA8A8091EC069091ED06892B09F0CE
:10D8C00063C067E576E0CE0183579F4F0E94B58025
:10D8D000CE0183579F4F0E94CBA8CE0183579F4F05
:10D8E0000E94798063E170E18EEE9DE00E94958256
:10D8F000F12CE12C00CF9DE0C91201C0C82EC80157
:10D900000E9434C8D82ED7011F96AD90BC90A114A8
:10D91000B10499F1BAE08B1779F0EDE08E1761F060
:10D92000FFEF8F1749F0682FCE0183579F4F0E945A
:10D930006B7F8C2DCD2C6ACFCF56DF4F888199819C
:10D94000C159D040892B91F0BE0163577F4FCE0162
:10D9500085589F4F0E94AC80CE0185589F4FF5019E
:10D960001995CE0185589F4F0E94798067E576E032
:10D97000CE0183579F4F0E944980FFEFDF12D9CF1E
:10D98000C8010E94AA8A48CF0E9438668091870801
:10D99000882329F00E94929867FF0E941B1B6CE06D
:10D9A00070E184EE9DE00E949582A5CEE0E3EE1644
:10D9B000E1E0FE0651F468EF7FE084EE9DE00E9416
:10D9C0009582C8010E94AA8A96CE60EE7FE08EEE14
:10D9D0009DE00E949582C8010E94AA8AB7018EEE3E
:10D9E0009DE00E945E958EEE9DE00E949E8183CE1A
:10D9F000D7015196BC9051975296AC90DF92CF923E
:10DA000089EC9FE09F938F931F930F930E9470C8A0
:10DA1000DF92CF9284EC9FE09F938F931F930F939D
:10DA20000E9470C8D8011C96ED91FC9181E0828320
:10DA3000DF92CF9281EC9FE09F938F931F930F9380
:10DA40000E9470C8D8011C96ED91FC911282AF9291
:10DA5000BF928BE89FE09F938F931F930F930E9439
:10DA600070C80FB6F894DEBF0FBECDBFB12C82E8F0
:10DA7000C82E8FE0D82E8B2D94E08902F00111245E
:10DA8000A5E8B0E0AC0FBD1FEA0FFB1F80819181BC
:10DA9000009709F467CE2281338121153105C1F346
:10DAA0003F932F939F938F93DF92CF921F930F9368
:10DAB0000E9470C8B3940FB6F894DEBF0FBECDBFFE
:10DAC000DACF0F931F93CF93DF93EB0102970CF400
:10DAD0009DC00A811B816DE57FE0C8010E94E3C6FD
:10DAE000892B51F481E00E94559988EC90E0DF91F8
:10DAF000CF911F910F91089569E57FE0C8010E94C1
:10DB0000E3C6892B11F480E0EECF69E37FE084EE79
:10DB10009DE00E9495820E94929863FB662760F9BF
:10DB200081E0682770E084EE9DE00E945E9584EEBF
:10DB30009DE00E949E818091C10D9091C20D892B24
:10DB400009F454C00A811B810E949F95882309F41F
:10DB50004DC0F80101900020E9F73197E01BF10B6F
:10DB6000B09708F043C0A091C10DB091C20D52967C
:10DB70001C921E92519754961C921E92539784E8C1
:10DB800090E01D969C938E931C971E961C921E9758
:10DB900080E090E350969C938E931F97ED91FC91BB
:10DBA00011970088F189E02D60E270E0CD011995B0
:10DBB000B8018091C10D9091C20D0E942F82809179
:10DBC000C10D9091C20DDC01ED91FC910190F081AD
:10DBD000E02D60E019958091C10D9091C20DDC019E
:10DBE000ED91FC910488F589E02D19956A817B817E
:10DBF00084EE9DE00E942F8262E37FE084EE9DE050
:10DC00000E94958284EE9DE00E949E81809188080A
:10DC10009091890802977CF10E94CC69883C91051B
:10DC200039F424E030E030938908209388085FCFEE
:10DC30008F3F9807C9F467E17FE085E19FE00E948C
:10DC4000958285E19FE00E949E811092850883E085
:10DC500090E0909389088093880882EB9DE00E9471
:10DC60007F6589EC90E043CF209187082111D9CFBF
:10DC70002FE030E0D8CF6AE07FE08EEE9DE00E949A
:10DC800095828EEE9DE00E949E8184EF91E02FCFE1
:10DC9000CF93DF93CDB7DEB72E970FB6F894DEBFE4
:10DCA0000FBECDBF8091860881116BC066E47EE017
:10DCB00084EE9DE00E94958284EE9DE00E949E810C
:10DCC0001092E10D1092E00D80E090E19093DC0D58
:10DCD0008093DB0D84E890E09093E30D8093E20D58
:10DCE00081E08093DD0D80E090E29093DF0D8093E2
:10DCF000DE0D8FEC9DE00E94A5258B37910509F084
:10DD0000C4C01C821B8282E293E09A8389838FECD9
:10DD10009DE09E838D838FEF9FEF98878F83809107
:10DD2000EC069091ED06892B11F00E945A64CE0109
:10DD300001960E94029E9093ED068093EC068FEC74
:10DD40009DE00E94CE138091EC069091ED06892B08
:10DD5000D9F46AE37EE08EEE9DE00E9495828EEE1D
:10DD60009DE00E949E8167E576E0CE0109960E94C3
:10DD7000B580CE0109960E94CBA8CE0109960E94DB
:10DD8000798090E080E014C067E27EE084EE9DE060
:10DD90000E94958284EE9DE00E949E810E943866DA
:10DDA0008091C10D9091C20D892B59F481E090E0D2
:10DDB0002E960FB6F894DEBF0FBECDBFDF91CF9188
:10DDC00008950E949F95882389F3A091C10DB09179
:10DDD000C20D52961C921E92519754961C921E92FE
:10DDE000539784E890E01D969C938E931C971E9603
:10DDF0001C921E9780E090E350969C938E931F9701
:10DE0000ED91FC9111970088F189E02D60E670E0BA
:10DE1000CD0119956091C10D7091C20D40E0CE0108
:10DE200009960E94F880BE01675F7F4F83EC9DE0FA
:10DE30000E947F7FCE0109960E9479808091C10D5A
:10DE40009091C20DDC01ED91FC910488F589E02DE3
:10DE5000199569E07EE085E19FE00E94958263EC80
:10DE60007DE0CE0109960E94AC80BE01675F7F4FC6
:10DE700085E19FE00E94878285E19FE00E949E816C
:10DE8000CE0109960E94798091CF8FEC9DE00E948F
:10DE9000E713892BA1F08FEC9DE00E94111467E538
:10DEA00076E0CE0101960E94B580CE0101960E94D7
:10DEB000CBA8CE0101960E9479800E943FA88FECEA
:10DEC0009DE00E94CE1366E17EE084EE9DE00E941C
:10DED000958284EE9DE00E949E8153CF0E94486E01
:10DEE000892B49F486EF9FEF9093890880938808E7
:10DEF00084EF91E0089588EC90E00895BF92CF926E
:10DF0000DF92EF92FF920F931F93CF93DF9300D096
:10DF100000D0CDB7DEB78C016B01FB018481958108
:10DF2000892BD9F1E080F1806FE370E0C7010E9496
:10DF30008CD4009791F19C012E193F09790137FD8E
:10DF40002CC067E576E0CE0101960E94B580F6010F
:10DF5000848195810097B9F08E159F0508F47C01A6
:10DF6000F60160817181FB01EE0DFF1DB080108212
:10DF7000CE0101960E945380F60180819181E80EC6
:10DF8000F91EF701B082BE016F5F7F4FC6010E948C
:10DF90007F7FCE0101960E94798063E076E0C60122
:10DFA0000E94FA7E882319F1F801128A118A80E012
:10DFB00090E19587848784E890E0948B838B81E05F
:10DFC000868780E090E2908B878781E090E02696BC
:10DFD0000FB6F894DEBF0FBECDBFDF91CF911F917A
:10DFE0000F91FF90EF90DF90CF90BF90089560E188
:10DFF00076E0C6010E94FA7E882369F0F801128A51
:10E00000118A148A138A84E890E09587848716869B
:10E0100080E090E3D8CF90E080E0D9CFDF92EF921C
:10E02000FF920F931F93CF93DF9300D000D0CDB713
:10E03000DEB78C017B0167EE74E1CE0101960E9490
:10E040007E80BE016F5F7F4FC7010E940F7FD82E79
:10E05000CE0101960E947980DD2019F1D801129637
:10E06000ED91FC9113970190F081E02D6081718119
:10E07000ED91FC910288F389E02D2CE136E04CE92A
:10E0800055E0C801199526960FB6F894DEBF0FBE6D
:10E09000CDBFDF91CF911F910F91FF90EF90DF9057
:10E0A00008956CEC74E1CE0101960E947E80BE0161
:10E0B0006F5F7F4FC7010E940F7FD82ECE01019660
:10E0C0000E947980DD20A1F0D8011296ED91FC919B
:10E0D00013970190F081E02D60817181ED91FC91A9
:10E0E0000288F389E02D2CE136E04FE855E0C9CFF6
:10E0F00061EB74E1CE0101960E947E80BE016F5FEC
:10E100007F4FC7010E940F7FF82ECE0101960E941B
:10E110007980FF2009F4B7CFD8011296ED91FC91D8
:10E1200013970190F081E02D60817181ED91FC9158
:10E130000288F389E02D2CE136E04EE756E0A1CFCE
:10E140006F927F928F929F92AF92BF92CF92DF9207
:10E15000EF92FF920F931F93CF93DF93CDB7DEB76C
:10E160002C970FB6F894DEBF0FBECDBF4C0186E1F1
:10E170009CE00E945A78892B39F180E00E94641754
:10E180006093B5077093B6078093B7079093B8076D
:10E1900086E19CE00E943878682E8DE290E09A83B8
:10E1A000898369824FE350E0BE016F5F7F4F8BE24E
:10E1B00097E00E94A7D48091B3079091B40701968D
:10E1C0009093B4078093B30789EF9AE00E945A783E
:10E1D000892B39F180E00E9464176093AF07709338
:10E1E000B0078093B1079093B20789EF9AE00E943D
:10E1F0003878782E8DE290E09A83898379824FE394
:10E2000050E0BE016F5F7F4F8DE697E00E94A7D47C
:10E210008091AD079091AE0701969093AE078093E1
:10E22000AD078091B5079091B607A091B707B0915F
:10E23000B807892B8A2B8B2B09F0C7C08AE268129A
:10E24000DEC01092B5071092B6071092B707109271
:10E25000B8071092B4071092B3076BE277E0CE01D3
:10E2600007960E94B58010922B07CE0107960E9458
:10E270000D7E8B859C85892B09F4DEC163E276E0F7
:10E28000CE0101960E94B580BE016F5F7F4FCE0127
:10E2900007960E94DF7E182FCE0101960E9479809A
:10E2A000112321F0809129028823A1F0BE01695F2A
:10E2B0007F4FCE0101960E94AC80CE0101960E9454
:10E2C0008B9FBC0189EF9AE00E948782CE01019664
:10E2D0000E947980BE01695F7F4FCE0101960E9446
:10E2E000AC80BE016F5F7F4FC4010E940E70CE01F3
:10E2F00001960E9479806CE276E0CE0101960E9440
:10E30000B580BE016F5F7F4FCE0107960E94DF7E12
:10E31000182FCE0101960E947980112309F44FC174
:10E32000BE01695F7F4F8EE49FE00E940F7F8111E5
:10E3300083C1BE01695F7F4F8EE49FE00E946280CF
:10E340004F815885D4011296ED91FC91139701905D
:10E35000F081E02D60817181ED91FC910288F3895B
:10E36000E02D22E336E0C401199580916B0790916E
:10E370006C07892B09F460C162E075E185E19FE0DB
:10E380000E94958210E000E0F0E1EF2EF12CB80140
:10E39000CE0107960E94CD7EFC018081882309F47E
:10E3A00047C18B859C850817190708F041C18091EA
:10E3B0006B0790916C078130910509F442C1029777
:10E3C00009F46AC10F5F1F4FE2CF0E949DA29B011B
:10E3D000AC016091B5077091B6078091B707909135
:10E3E000B807A12CB12C65011AE0E12EF12C00E058
:10E3F00010E00E94342A882309F420CF22CFADE018
:10E400006A1609F41ECF8091B3079091B407803447
:10E41000910508F016CF8091AF079091B007A091B9
:10E42000B107B091B207892B8A2B8B2B09F040C121
:10E43000BAE27B1257C11092AF071092B007109248
:10E44000B1071092B2071092AE071092AD076DE6B9
:10E4500077E0CE0107960E94B58010926D07CE013D
:10E4600007960E940D7E8B859C85892B09F49AC1A5
:10E4700063E276E0CE0101960E94B580BE016F5F37
:10E480007F4FCE0107960E94DF7E182FCE010196A6
:10E490000E947980112321F0809129028823A1F024
:10E4A000BE01695F7F4FCE0101960E94AC80CE0114
:10E4B00001960E948B9FBC0186E19CE00E948782AE
:10E4C000CE0101960E947980BE01695F7F4FCE0127
:10E4D00001960E94AC80BE016F5F7F4FC4010E9415
:10E4E0000E70CE0101960E9479806CE276E0CE013A
:10E4F00001960E94B580BE016F5F7F4FCE010796E7
:10E500000E94DF7E182FCE0101960E947980112390
:10E5100009F40BC1BE01695F7F4F8AE59FE00E944D
:10E520000F7F81113FC1BE01695F7F4F8AE59FE088
:10E530000E9462804F815885D4011296ED91FC9122
:10E5400013970190F081E02D60817181ED91FC9134
:10E550000288F389E02D22E436E0C4011995809108
:10E560006B0790916C07892B09F41CC164E075E17D
:10E5700085E19FE00E949582912C812C00E110E0C2
:10E58000B401CE0107960E94CD7EFC0180818823D4
:10E5900009F404C18B859C858816990608F0FEC095
:10E5A00080916B0790916C078130910509F4FFC051
:10E5B000029709F427C1BFEF8B1A9B0AE1CF67E3EB
:10E5C00076E0CE0101960E94B580BE016F5F7F4F5D
:10E5D000CE0107960E94DF7E182FCE0101960E9481
:10E5E0007980112309F4C1CEBE01695F7F4F84E5B4
:10E5F0009FE00E940F7F81111FC0BE01695F7F4FA6
:10E6000084E59FE00E9462804F815885D401129674
:10E61000ED91FC9113970190F081E02D6081718163
:10E62000ED91FC910288F389E02D2DE336E09BCE3D
:10E6300085E19FE00E949E81CE0107960E9479802D
:10E64000EACEB801CE0107960E94CD7EDC018C9106
:10E6500067E576E0803114F46FEE74E085E19FE0C9
:10E660000E942F82B801CE0107960E94CD7EFC0148
:10E670008081082E000C990BAA0BBB0B89839A830F
:10E68000AB83BC83FE82ED82BE016F5F7F4F85E16D
:10E690009FE00E94721A96CEB801CE0107960E94A2
:10E6A000CD7EDC016C9185E19FE00E94A2818ACE43
:10E6B0000E949DA29B01AC016091AF077091B007D1
:10E6C0008091B1079091B207A12CB12C65011AE09D
:10E6D000E12EF12C00E010E00E94342A882309F496
:10E6E000A7CEA9CEEDE07E1609F4A5CE8091AD07A8
:10E6F0009091AE078034910508F09DCE81E090E0C6
:10E700002C960FB6F894DEBF0FBECDBFDF91CF9130
:10E710001F910F91FF90EF90DF90CF90BF90AF903F
:10E720009F908F907F906F90089567E376E0CE0181
:10E7300001960E94B580BE016F5F7F4FCE010796A4
:10E740000E94DF7E182FCE0101960E94798011234E
:10E7500009F405CFBE01695F7F4F80E69FE00E940C
:10E760000F7F81111FC0BE01695F7F4F80E69FE070
:10E770000E9462804F815885D4011296ED91FC91E0
:10E7800013970190F081E02D60817181ED91FC91F2
:10E790000288F389E02D27E436E0DFCE85E19FE0B3
:10E7A0000E949E81CE0107960E947980A7CFB40176
:10E7B000CE0107960E94CD7EDC018C9167E576E064
:10E7C000803114F46FEE74E085E19FE00E942F82A7
:10E7D000B401CE0107960E94CD7EFC018081082EF7
:10E7E000000C990BAA0BBB0B89839A83AB83BC8368
:10E7F0001E830D83BE016F5F7F4F85E19FE00E9406
:10E80000721AD9CEB401CE0107960E94CD7EDC01EA
:10E810006C9185E19FE00E94A281CDCEFF920F9383
:10E820001F93CF93DF9300D000D0CDB7DEB78C011C
:10E83000BC01CE0101960E94AC80BE016F5F7F4F8C
:10E8400085E19FE00E94878285E19FE00E949E8192
:10E85000CE0101960E94798064E67FE0CE010196A8
:10E860000E947E80BE016F5F7F4FC8010E94DF7EE5
:10E87000F82ECE0101960E947980FF2069F0B80140
:10E88000CE0101960E94AC80CE0101960E94CBA8D9
:10E89000CE0101960E94798026960FB6F894DEBFCD
:10E8A0000FBECDBFDF91CF911F910F91FF900895C3
:10E8B0005F926F927F928F929F92AF92BF92CF9210
:10E8C000DF92EF92FF920F931F93CF93DF93CDB719
:10E8D000DEB7C956D1090FB6F894DEBF0FBECDBF63
:10E8E0004C018B01F42E642F85E19FE00E94579527
:10E8F0006DEC7AE085E19FE00E949582B801CE013F
:10E9000001965C010E94AC80B50185E19FE00E9408
:10E91000878285E19FE00E949E81C5010E947980E7
:10E9200092E0F91263C26BEC7AE0C5010E947E802E
:10E93000B501C8010E940F7FF82EC5010E947980A1
:10E94000FF2009F4C8C220E04DE251E0B40180E9A3
:10E950009DE00E94A487E0908108F090820864EC1A
:10E960007AE0CE018C599F4F0E947E806DEB7AE059
:10E97000CE01825A9F4F0E947E80CE018E5A9F4FB9
:10E980000E94D12868961FAD689767960FAD67976C
:10E990006696DFAC66976596CFAC659767E576E0DF
:10E9A000CE0181960E94B580BE016F5D7F4FC5018B
:10E9B0000E94AC806C2DC5010E94CA7F6CE476E099
:10E9C0000E94FB7F6D2D0E94CA7F6CE476E00E945E
:10E9D000FB7F602F0E94CA7F6CE476E00E94FB7F81
:10E9E000612F0E94CA7FBC01CE01885A9F4F0E94AE
:10E9F000AC80C5010E947980CE0181960E94798009
:10EA000068EB7AE0CE01845B9F4F0E947E8067E5D1
:10EA100076E0CE018A5B9F4F0E94B58001EC1DE03D
:10EA2000D80118966C9170E084E0759567958A9589
:10EA3000E1F7C5010E9473954D815E8169817A81FC
:10EA4000CE018A5B9F4F0E943F7FC5010E94798063
:10EA5000F80160856F7070E0C5010E9473954D816B
:10EA60005E8169817A81CE018A5B9F4F0E943F7FE0
:10EA7000C5010E9479800F5F1F4FFDE0073C1F0713
:10EA800079F662EB7AE0CE01805C9F4F0E947E8037
:10EA900061E97AE0CE0181960E947E80BE016F5DC1
:10EAA0007F4FCE01C8960E94AC80BE01605C7F4F54
:10EAB000CE01C8960E941580BE016A5B7F4F0E94FE
:10EAC0001580BE01645B7F4F0E941580BE01685AAD
:10EAD0007F4F0E941580BE01625A7F4F0E941580B1
:10EAE0008C014AE0B50180E590E00E947DC7F50108
:10EAF00001900020E9F73197AF014A195B09B50190
:10EB0000C8010E943F7F811103C0C8010E94B87FE5
:10EB1000BE016C597F4FC8010E941580B7010E9449
:10EB2000FB7FBC01C4010E948782C4010E949E81B8
:10EB3000CE01C8960E947980CE0181960E9479808C
:10EB4000CE01805C9F4F0E947980CE018A5B9F4FEF
:10EB50000E947980CE01845B9F4F0E947980CE0114
:10EB6000885A9F4F0E947980CE01825A9F4F0E94FF
:10EB70007980CE018C599F4F0E947980C4010E94F8
:10EB80009E8164E670E080E090E00E946BA2D40178
:10EB9000ED91FC910488F589E02DC401199501E0FF
:10EBA00010E080C022966EAD7FAD2297CE01819697
:10EBB0000E94639A892B09F448C118AE19AE1AAEA7
:10EBC0001BAE1CAE1DAE1EAE1FAE89AD8F7089AFE1
:10EBD00040E053E0BE016F5D7F4FCE01C8960E94BA
:10EBE000693300E020E033E040E250E0B501CE01BF
:10EBF000C8960E94E11FBC01C6010E94538008EC28
:10EC000010E125C1EE2009F4EFC046E050E070E0CD
:10EC100060E0C8010E946A7ED8016D917C91CE01AE
:10EC200081960E944954CE0181960E94901300E97A
:10EC300011E0882399F189A5873061F4CE0181968E
:10EC40000E94BD4F61E0892B09F462E0CE018196FC
:10EC50000E94751C18AE19AE1AAE1BAE1CAE1DAECE
:10EC60001EAE1FAE89AD8F7089AF40E053E0BE018C
:10EC70006F5D7F4FCE01C8960E94693300E020E0AF
:10EC800033E040E250E0B501CE01C8960E94E11F9A
:10EC9000BC01C6010E94538008EC10E1CE018196B0
:10ECA0000E94B713C801C759DF4F0FB6F894DEBFF3
:10ECB0000FBECDBFDF91CF911F910F91FF90EF90CD
:10ECC000DF90CF90BF90AF909F908F907F906F908C
:10ECD0005F900895F801608171810E94D5947C0154
:10ECE000892B09F040C104E911E0DCCFEE2009F4E2
:10ECF0007BC049E050E070E060E0C8010E946A7E9D
:10ED00004AE0B401C5010E94F88041E050E060E4AF
:10ED100074E0C8010E943F7F4D815E8169817A81E4
:10ED2000C8010E943F7F6DE67AE085E19FE00E9486
:10ED30009582B801CE0181960E94AC80BE016F5DC4
:10ED40007F4F85E19FE00E94878285E19FE00E94DE
:10ED50009E81CE0181960E94798065E67AE0CE019F
:10ED600081960E947E80F801848195812DA13EA12B
:10ED700082179307E1F4892BA1F1E080F18069A06B
:10ED80007AA0D7018D917D01882359F1082E000CBE
:10ED9000990B0E941CD46C01F30181913F01082E54
:10EDA000000C990B0E941CD4C816D90651F3CE0151
:10EDB00081960E947980552041F021E048EC50E096
:10EDC000B40180E99DE00E94A487D8018D919C91B7
:10EDD0000E94D287009711F484E991E08C01C5016B
:10EDE0003DC055245394E3CF01E97ECFB1E0FB123F
:10EDF00070C06AE87AE0C5010E947E80B501C80152
:10EE00000E94DF7E582EC5010E947980552049F16D
:10EE1000EE2051F346E050E070E060E0C8010E944F
:10EE20006A7E4AE0B401CE01805C9F4F0E94F88068
:10EE3000F80160817181CE0181960E944954CE0112
:10EE400081960E9490138111ADCE00E911E0CE01B0
:10EE500081960E94B713CE01805C9F4F0E947980FB
:10EE600021CF63E77AE0C5010E947E80B501C80129
:10EE70000E94DF7EF82EC5010E947980F11036CF06
:10EE800068E57AE0C5010E947E80B501C8010E9454
:10EE9000DF7E182FC5010E94798000E0112309F45C
:10EEA00001CF80E00E94559960E37AE084EE9DE016
:10EEB0000E94958284EE9DE00E949E8167E576E047
:10EEC000C5010E94B580C5010E94CBA8C5010E9462
:10EED000798000E065CE63E87AE0C5010E947E801B
:10EEE000B501C8010E94DF7EF82EC5010E9479801D
:10EEF000F11088CE6DE77AE0C5010E947E80B501F1
:10EF0000C8010E94DF7EF82EC5010E947980FF2093
:10EF100001F3EE2009F468CF45E050E070E060E0D6
:10EF2000C8010E946A7E6CE476E0C8010E94FA7E05
:10EF3000882339F0E0908A08F0908B08E114F104FE
:10EF400091F467E576E0C8010E94FA7E811107C05E
:10EF500080918A0890918B08009709F0BBCEE090D1
:10EF6000EC06F090ED0620E048EC50E2B40180E9B8
:10EF70009DE00E94A487C4010E949E811C821B8286
:10EF800082E293E09A8389839E828D828FEF9FEF46
:10EF900098878F83B701C5010E949988F2CD0895A3
:10EFA000FC01248135816217730748F480819181C7
:10EFB000009729F0860F971FFC018081089580E05B
:10EFC00008950895AF92BF92CF92DF92EF92FF9291
:10EFD0000F931F93CF93DF936C017B018B01040F81
:10EFE000151FEB015E01AE18BF08C017D10759F01D
:10EFF0006991D601ED91FC910190F081E02DC6015F
:10F000001995892B79F7C501DF91CF911F910F9148
:10F01000FF90EF90DF90CF90BF90AF900895FC01EC
:10F02000A089B1898C91A689B78982FD0FC09C9176
:10F03000818D8F5F8F77228D821749F0A18DAE0F62
:10F04000BF2FB11D5D969C93818F08958C9108957B
:10F05000FC01538D448D252F30E0842F90E0821BDE
:10F06000930B541718F081589F4F089501970895F6
:10F07000FC01918D828D981761F0A28DAE0FBF2F8C
:10F08000B11D5D968C91928D9F5F9F77928F90E0DE
:10F0900008958FEF9FEF0895FC01918D828D981751
:10F0A00031F0828DE80FF11D858D90E008958FEF8E
:10F0B0009FEF0895FC01918D228D892F90E080585B
:10F0C0009F4F821B91098F77992708958CED99E0C6
:10F0D0000E945A7821E0892B09F420E0822F0895BC
:10F0E00089EF9AE00E945A7821E0892B09F420E008
:10F0F000822F089586E19CE00E945A7821E0892BB6
:10F1000009F420E0822F089588EF9DE00E945A784C
:10F1100021E0892B09F420E0822F0895FC01A48DC1
:10F12000A80FB92FB11DA356BF4F2C91848D90E02D
:10F1300001968F779927848FA689B7892C93A08908
:10F14000B1898C9180648C93938D848D981306C0C3
:10F150000288F389E02D80818F7D80830895EF926E
:10F16000FF920F931F93CF93DF93EC0181E0888F81
:10F170009B8D8C8D981316C0E889F989808185FF55
:10F1800011C0EE89FF896083E889F98980818064F4
:10F19000808381E090E0DF91CF911F910F91FF90EC
:10F1A000EF900895F62E0B8D10E00F5F1F4F0F7735
:10F1B0001127E02E8C8D8E110CC00FB607FCFACFF4
:10F1C000E889F989808185FFF5CFCE010E948E788C
:10F1D000F1CFEB8DEC0FFD2FF11DE356FF4FF082C9
:10F1E0000B8FEA89FB8980818062D2CFCF93DF9336
:10F1F000EC01888D8823B9F0AA89BB89E889F9894F
:10F200008C9185FD03C0808186FD0DC00FB607FC83
:10F21000F7CF8C9185FFF2CF808185FFEDCFCE01B6
:10F220000E948E78E9CFDF91CF91089580E090E041
:10F23000892B29F00E94847881110E94000080E0CF
:10F2400090E0892B29F00E947A7881110E940000B9
:10F2500080E090E0892B29F00E94707881110E9453
:10F26000000080E090E0892B29F00E9466788111EF
:10F270000C94000008950F931F93FC016285738521
:10F28000848595850281138124813581601B710BF2
:10F29000820B930B0685178520893189601B710BC2
:10F2A000820B930B1F910F910895DC01ED91FC915E
:10F2B0000190F081E02D19948FEF9FEF0895FC01EC
:10F2C00062897389848995890895EF920F931F93BA
:10F2D000CF93DF93FC01248D222341F0213051F1A3
:10F2E000DF91CF911F910F91EF900895228933897B
:10F2F0004489558986899789A08DB18D821B930B8E
:10F30000A40BB50B892F9A2FAB2FBB278C010F5F56
:10F310001F4F6281738184819581CFB7F894DCB7E8
:10F32000E1E0ECBFEE24E394E2E0FEEF1995DCBFF0
:10F33000CFBFD6CFF0E0E0E0DF91CF911F910F91EA
:10F34000EF901994FC01138E128E41110CC082892A
:10F350009389A489B589868B978BA08FB18F148EE2
:10F3600081E090E0089590E080E00895CF92DF92F0
:10F37000EF92FF92CF93DF93DC01CB01642FCFB7E5
:10F38000F8946D01EE24FF24CBBEDCB741E04CBF06
:10F39000A901E1E0FEEF1995DCBFCFBFDF91CF916E
:10F3A000FF90EF90DF90CF900895CF93DF93FC0113
:10F3B000248D211110C0EC01828D938D892B49F091
:10F3C00066897789808D918D30E020E045E00E944C
:10F3D000B6791B8E1A8EDF91CF9108951F93CF932C
:10F3E000DF93FC01248D211145C0162FEC01828D85
:10F3F000938D892B49F466897789808D918D30E0D2
:10F4000020E043E00E94B6794A8D5B8DCA0181708D
:10F410009927FE01E80FF91F158F892B69F02D8DB3
:10F420003E8D6E897F89888D998D640F751F811D32
:10F43000911D41E00E94B6798A8D9B8D01969B8F2C
:10F440008A8F81159140B1F46E897F89888D998D5D
:10F4500030E020E045E00E94B6791B8E1A8E8E893E
:10F460009F89A88DB98D9F5FAF4FBF4F8E8B9F8BAC
:10F47000A88FB98F81E090E0DF91CF911F9108951F
:10F48000DC01ED91FC910280F381E02D40E01994C4
:10F49000FB0124813581428153812417350750F4C3
:10F4A000A081B181A20FB31F8C93848195810196B5
:10F4B0009583848380E00895CF93DF93EC01E88106
:10F4C000F9810284F385E02DCE0119950196B9F7F3
:10F4D000DF91CF910895CF92DF92EF92FF920F9339
:10F4E0001F93CF93DF937C016A018B01D0E0C0E0D2
:10F4F000CC15DD0581F0D701ED91FC910284F385F7
:10F50000E02DC70119958F3F980729F0F8018193E5
:10F510008F012196EDCFCE01DF91CF911F910F91F9
:10F52000FF90EF90DF90CF900895CF93C62FDC012E
:10F53000ED91FC910088F189E02D1995DC01ED91A8
:10F54000FC910190F081E02D6C2FCF911994062E43
:10F55000000C770BFC01778366830895CF93DF93CC
:10F56000EC018E819F81019611F5E881F981008877
:10F57000F189E02DCE011995DC01ED91FC9100841B
:10F58000F185E02D1995892BB1F0E881F98102848C
:10F59000F385E02DCE0119958132910534F3E88190
:10F5A000F9810684F785E02D682FCE01199581E059
:10F5B000DF91CF91089580E0FBCFFC0120812EBD2B
:10F5C0009B012150310941F051810DB407FEFDCF5F
:10F5D0004EB55EBD4193F5CF61507109860F971FFF
:10F5E0000DB407FEFDCF2EB5FC0120830895E091F8
:10F5F0008D08F0918E08808190918C08892B8083F2
:10F600000895E0918D08F0918E08908180918C088A
:10F6100080958923808308958EBD00000DB407FE78
:10F62000FDCF8EB5089590E02091C909233339F4B8
:10F630000C96982F990F990F990F80E0089548968E
:10F64000F8CFEF92FF920F931F93CF93DF93EC01CC
:10F650008B017A010E949DA2688B798B8A8B9B8B90
:10F660008C819D81DC01ED91FC910280F381E02D84
:10F67000A701B801DF91CF911F910F91FF90EF90FB
:10F6800019941F93CF93DF93EC01162F0E949DA234
:10F69000688B798B8A8B9B8B8C819D81DC01ED91B2
:10F6A000FC910190F081E02D612FDF91CF911F91AE
:10F6B0001994CF92DF92EF92FF92CF93DF93EC01F8
:10F6C0008E819F818F3F980759F02FEF3FEF3F8347
:10F6D0002E83DF91CF91FF90EF90DF90CF90089530
:10F6E0000E949DA26B017C01A4EFCA0EA1E0DA1E6C
:10F6F000E11CF11CE881F9810088F189E02DCE013F
:10F700001995DC01ED91FC910084F185E02D1995AE
:10F71000892B39F40E949DA26C157D058E059F05ED
:10F7200048F3E881F9810088F189E02DCE0119952F
:10F73000DC01ED91FC910284F385E02DDF91CF9106
:10F74000FF90EF90DF90CF9019940E9417D40F9301
:10F750001F93CF93DF93EC0188819981009759F033
:10F760002A813B812617370730F081E0DF91CF9166
:10F770001F910F9108958B016F5F7F4F0E9436D3C9
:10F78000009759F0998388831B830A832C813D81DC
:10F79000232B59F7FC011082E8CF80E0E7CFEF92EE
:10F7A000FF920F931F93CF93DF93009751F4CFEF06
:10F7B000DFEFCE01DF91CF911F910F91FF90EF907E
:10F7C0000895DC011C96ED90FC90F70100811181F9
:10F7D000D801ED91FC910688F789E02DC8011995B3
:10F7E000882329F3D801ED91FC910084F185E02D67
:10F7F000C8011995D801ED91FC91892B61F3028420
:10F80000F385E02DC8011995EC01019681F2F8010C
:10F81000818D882329F06C2F88EF9DE00E945795F9
:10F82000D70112968C91882321F2C532D10509F6B1
:10F83000D801ED91FC910084F185E02DC801199566
:10F8400002975CF0D801ED91FC910688F789E02DD4
:10F85000C80119958111ECCFAACFD1E0C0E0D80141
:10F86000ED91FC910284F385E02DC80119958F3F3D
:10F87000980709F49CCF9C01215431092A313105A4
:10F8800070F48D2F8295807F829FC00D1124D1113D
:10F8900004C00C2E000CDD0B8CCFD0E0E0CF9C011F
:10F8A000215631092A31310560F3C0978A3091051C
:10F8B00070F79D2F9295907F989FC00D1124E7CFF0
:10F8C000CF92DF92EF92FF920F931F93CF93DF932C
:10F8D0006C018B0186E090E00E94C9C3EC0190931B
:10F8E0000E0980930D09F60101900020E9F7CF0180
:10F8F0008C199D090E94C9C37C01B6010E94A0D445
:10F90000F60101900020E9F73197EC19FD09EE0DA1
:10F91000FF1D1082F982E8821B830A8380911009FF
:10F92000909111099D838C83D0931109C093100984
:10F93000DF91CF911F910F91FF90EF90DF90CF90CB
:10F940000895FC01868197818F3F980729F02FEF5A
:10F950003FEF378326830895808591850C9434C8C2
:10F960007F928F929F92AF92BF92CF92DF92EF924F
:10F97000FF920F931F93CF93DF93CDB7DEB7A69778
:10F980000FB6F894DEBF0FBECDBF8C01762E942E3D
:10F99000852E20E2A22ECE0101967C01DC01EA2D0B
:10F9A0001D92EA95E9F76801F3E4CF0ED11C89E2D4
:10F9B00094E09AA389A38FEF8BA38CA38DA38EA32E
:10F9C00043E450E0BE016F5D7F4FC6010E941428E2
:10F9D000019609F4BFC081E089838A8386E0B82E4E
:10F9E000BB821C82D80114966D917D918D919C9162
:10F9F00017970E943ED06D837E838F839887898678
:10FA00009A8680E890E09C878B874CE150E0B701B4
:10FA1000C6010E94A927FE0137968AE1DF011D92E7
:10FA20008A95E9F74801B8E08B0E911CF401D701E3
:10FA300001900D92BA94E1F740E150E0B701C601A0
:10FA40000E94A927F7011192AA94E9F796E0A92E3E
:10FA5000B12C40E250E0B701C6010E94A927F1E0B5
:10FA6000AF1AB108B1F783E6898392E89A8393E5E8
:10FA70009B838C8385E38D8381E08E837F829DE3EE
:10FA8000988797E099878A8786E0F401DE011B96C4
:10FA900001900D928A95E1F78CE0898B8A8B6EE458
:10FAA00076E0CE0143960E94A0D4D8011B966C91BB
:10FAB000CE0149960E94669EF8016485CE014B9660
:10FAC0000E94669ED8011D966C91CE014D960E94B3
:10FAD000669E4EE150E0B701C6010E94A927B3E03F
:10FAE0007B121EC082E3898384E08A83F8019685B5
:10FAF0009B8397859C8390899D8391899E8396E3C0
:10FB00009F838887828D8987838D8A87848D8B8761
:10FB1000858D8C874CE050E0B701C6010E94A92773
:10FB200087E3898386E08A8391E09B8393E09C83CB
:10FB30008D838FE08E838AE38F838BE388878FEFBB
:10FB4000898749E050E0B701C6010E94A927C60194
:10FB50000E94E327A6960FB6F894DEBF0FBECDBF76
:10FB6000DF91CF911F910F91FF90EF90DF90CF9099
:10FB7000BF90AF909F908F907F90089590E080E02D
:10FB80000C948126CF93DF93C4E1D0E00E94BE7D28
:10FB9000882361F061E070E080E090E00E946BA259
:10FBA0002197A1F780E0DF91CF91089581E0FBCF0D
:10FBB000FF920F931F93CF93DF931F921F92CDB7A6
:10FBC000DEB7F82E22E030E0AE014F5F5F4F66E215
:10FBD00070E00E94822709811A81102701271027CF
:10FBE00022E030E0AE014F5F5F4F66E270E08F2DA4
:10FBF0000E94822789819A81982789279827081748
:10FC0000190749F4C8010F900F90DF91CF911F9110
:10FC10000F91FF9008958C01E3CFAF92BF92CF92E6
:10FC2000DF92EF92FF920F931F93CF93DF93DC014C
:10FC3000CD90DC901197C114D10439F01496CD9178
:10FC4000DC918C017601209761F4DF91CF911F91B7
:10FC50000F91FF90EF90DF90CF90BF90AF900895FD
:10FC600075015701BFEFAB1ABB0AF7018081082E5F
:10FC7000000C990B0E94DAC6892B91F72197CC0DC5
:10FC8000DD1D8881082E000C990B0E94DAC6892B95
:10FC900029F0CE15DF0510F02197F3CFAE014F5FAD
:10FCA0005F4F4E195F09D80115965C934E931497D8
:10FCB000CE14DF0420F4B701C6010E9453D4D8014A
:10FCC000ED91FC91119714968D919C91E80FF91F7D
:10FCD0001082BBCFCF93DF93DC011496ED91FC91A2
:10FCE0006E177F0728F54115510511F19F01261B5D
:10FCF000370B4217530708F49A01DB01EC018881A6
:10FD00009981E21BF30BFD83EC83AF01461B570B7C
:10FD1000260F371FBC01620F731F8A0F9B1F0E94A3
:10FD2000C5D4E881F9818C819D81E80FF91F10828B
:10FD3000DF91CF910895DF92EF92FF920F931F937F
:10FD4000CF93DF93FC01E480F580E114F10451F4DA
:10FD50008FEF9FEFDF91CF911F910F91FF90EF9069
:10FD6000DF900895EC010190F081E02DEE0DFF1D74
:10FD7000D080108208811981062E000C770BC801F3
:10FD80000E94D4D40E0D1F1DF801D082009701F3FC
:10FD900028813981821B930BDDCFFC0124813581C1
:10FDA0006217730720F480819181009729F41092E3
:10FDB0000F098FE099E00895860F971F0895FB01C2
:10FDC00044815581FC01248135812417350778F061
:10FDD00080819181009759F0FB01608171816115EB
:10FDE000710529F00E94B7D421E0892B09F020E0A9
:10FDF000822F0895FC0124813581232B39F421E0E1
:10FE0000FB018081882349F020E007C08081918137
:10FE10000E9497D421E0892BB9F7822F0895FC0125
:10FE200024813581FB014481558124173507E1F494
:10FE3000FC0180819181FB01608171810097D1F08B
:10FE400061157105A1F4232BC1F0FC01808190E0C4
:10FE500008C0232B91F0FB01808190E09195819562
:10FE6000910921E0892B09F020E0822F08950E945A
:10FE700097D4F7CF6115710561F721E0F6CFEF92C6
:10FE8000FF920F931F93CF93DF936115710541F498
:10FE900080E0DF91CF911F910F91FF90EF90089537
:10FEA00041155105B1F07B01EC010C811D81040F5E
:10FEB000151FB8010E94A77B882351F3288139813F
:10FEC0008C819D81B701820F931F0E94A0D41D8356
:10FED0000C8381E0DECFCF93DF931F921F92CDB7CB
:10FEE000DEB769831A8241E050E0BE016F5F7F4F49
:10FEF0000E943F7F0F900F90DF91CF9108950F9355
:10FF00001F93CF93DF938C01EB01FC0180819181E2
:10FF10000097E1F06881798161157105A9F042814E
:10FF200053812C813D814217530770F00E94A0D469
:10FF30008C819D81F801958384831D821C82DF91D1
:10FF4000CF911F910F9108950E9465C48881998176
:10FF5000F801918380838A819B81938382838C8142
:10FF60009D8195838483198218821B821A82E5CF32
:10FF7000CF93DF93EC0188819981009711F00E9463
:10FF800065C4198218821D821C821B821A82DF912D
:10FF9000CF910895EF92FF920F931F93CF93DF932A
:10FFA00000D01F92CDB7DEB77C01862F4AE08E01CC
:10FFB0000F5F1F4FB80190E00E947DC7F8010190CC
:10FFC0000020E9F73197AF01401B510BB801C70181
:10FFD0000E943F7F811103C0C7010E94B87FC70103
:10FFE0000F900F900F900F90DF91CF911F910F9175
:10FFF000FF90EF900895CF93DF93EC0161157105A9
:020000021000EC
:1000000039F4CE010E94B87FCE01DF91CF910895DF
:10001000FB0101900020E9F73197AF01461B570B18
:100020000E943F7F882369F3EFCFCF93DF93EC01EA
:10003000FB0144815581608171810E943F7F811164
:1000400003C0CE010E94B87FCE01DF91CF91089509
:10005000EF92FF920F931F93CF93DF93EC017B01FD
:100060008A01BA010E94A77B81110BC0CE010E94B8
:10007000B87FCE01DF91CF911F910F91FF90EF904C
:1000800008951D830C83B701888199810E94A0D4B3
:10009000F0CFFB0101900020E9F73197AF01461B3B
:1000A000570B0C942880CF93DF93EC0161157105F9
:1000B00031F00E944980CE01DF91CF9108950E94D6
:1000C000B87FF9CFCF93DF93EC01FB018617970739
:1000D00049F0608171816115710541F0448155815C
:1000E0000E942880CE01DF91CF9108950E94B87FB1
:1000F000F9CFFC01808191810C9465C4EF92FF924D
:100100000F931F93CF93DF93EC018B011982188219
:100110001B821A821D821C82CB010E9411C77C01A6
:10012000BC01CE010E94A77B811109C0CE01DF91E5
:10013000CF911F910F91FF90EF900C94B87FFD82AB
:10014000EC82B80188819981DF91CF911F910F9145
:10015000FF90EF900C940AC7FC0111821082138269
:100160001282158214820C946280FC01118210822A
:1001700013821282158214826115710551F0FB0100
:1001800001900020E9F73197AF01461B570B0C9403
:10019000288008950F931F93CF93DF93EC010E9463
:1001A0009DA2688779878A879B87E881F981028485
:1001B000F385E02DCE01199597FF15C00E949DA2F1
:1001C000088519852A853B85601B710B820B930B73
:1001D0000C811D812E813F81601771078207930773
:1001E00020F38FEF9FEFDF91CF911F910F91089533
:1001F000EF92FF920F931F93CF93DF93EC017B015C
:10020000042F67E576E00E94B580C7010E94CA808E
:10021000002E000C110B97FD0BC00817190741F0B9
:10022000682FCE010E946B7FC7010E94CA80F3CF66
:10023000CE01DF91CF911F910F91FF90EF90089524
:10024000CF92DF92EF92FF920F931F93CF93DF93A2
:100250006C017A018B01D0E0C0E0C6010E94CA8027
:1002600097FD07C0F80181938F012196EC16FD06DA
:10027000A1F7CE01DF91CF911F910F91FF90EF90E9
:10028000DF90CF900895FB0101900020E9F73197AE
:10029000AF01461B570BDC01ED91FC910280F3810D
:1002A000E02D19948F929F92AF92BF92EF92FF929E
:1002B0000F931F93CF93DF93CDB7DEB7A1970FB600
:1002C000F894DEBF0FBECDBF7C01FA01CB0119A2AD
:1002D000223008F42AE08E010F5D1F4F822E912CF0
:1002E000B12CA12CBF01A50194010E94ABCFF90153
:1002F000CA016A300CF5605DD8016E938D01232B25
:10030000242B252B79F790E080E0109721F0BD0198
:10031000C7010E944381A1960FB6F894DEBF0FBEBD
:10032000CDBFDF91CF911F910F91FF90EF90BF90C4
:10033000AF909F908F900895695CDECF65E576E081
:100340000C944381DC01ED91FC910190F081E02D52
:100350001994CF92DF92EF92FF920F931F93CF9356
:10036000DF932115310581F4DC01ED91FC910190C1
:10037000F081E02D642FDF91CF911F910F91FF90BD
:10038000EF90DF90CF9019942A30310501F52AE0E3
:1003900077FF1DC06A017B01EC016DE20E94A28122
:1003A0008C0144275527BA014C195D096E097F0954
:1003B0002AE0CE010E945281800F911FDF91CF91E0
:1003C0001F910F91FF90EF90DF90CF900895DF91F4
:1003D000CF911F910F91FF90EF90DF90CF900C94F1
:1003E00052818F929F92AF92BF92CF92DF92EF9203
:1003F000FF920F931F93CF93DF937C018B014C01EE
:1004000082E0880E911C5701E5E0AE0EB11CD0E0F1
:10041000C0E0F40161914F01C8010E9457956C0141
:100420006EE2C8010E94A2818C0D9D1DC80FD91FCC
:100430008A149B0471F7F7016581C8010E945795E2
:100440008C0F9D1FDF91CF911F910F91FF90EF9027
:10045000DF90CF90BF90AF909F908F9008956115DF
:10046000710511F00C94438190E080E008950F93A2
:100470001F93CF93DF93EC018B0163EF75E00E9434
:100480002F8201151105C1F1F80161918F016623D9
:1004900099F1603240F0623231F06C3521F0CE01DA
:1004A0000E94A281F1CF6CE5CE010E94A281F801E9
:1004B000319780818C30D1F044F48930D9F08A3082
:1004C000B9F0883009F762E6EACF823259F024F4B5
:1004D00062E78D3021F3D8CF8F3231F06CE58C3567
:1004E000F1F2D2CF62E2DBCF6FE2D9CF66E6D7CFAF
:1004F0006EE6D5CF64E7D3CF62E2CE010E94A2813F
:1005000090E080E0DF91CF911F910F910895DB0182
:1005100014964D915C9115976D917C91DC01ED9154
:10052000FC910280F381E02D1994EF92FF920F93DA
:100530001F93CF93DF938C017B01D0E0C0E0F701E4
:10054000EC0FFD1F6491662361F0D801ED91FC91E1
:100550000190F081E02DC8011995892B11F02196A9
:10056000EECFCE01DF91CF911F910F91FF90EF90D1
:1005700008950F931F93CF93DF93EC010E94958210
:100580008C01CE010E949E81800F911FDF91CF913F
:100590001F910F910895DC0189E294E08D939D9362
:1005A00084E0FB0101900D928A95E1F708953F9256
:1005B0004F925F926F927F928F929F92AF92BF9273
:1005C000CF92DF92EF92FF920F931F93CF93DF931F
:1005D000CDB7DEB7EA970FB6F894DEBF0FBECDBF3A
:1005E0007C012A013B0169010E949DA24B015C0133
:1005F00087010D5B1F4FC8010E948315181619064D
:10060000ACF00E949DA2681979098A099B094616D7
:1006100057066806790608F468C10E946D6561E0B6
:1006200070E080E090E00E946BA2E5CF42E250E0F3
:10063000BE016F5F7F4FC8010E940E158981823015
:10064000D1F0312C832DEA960FB6F894DEBF0FBEA1
:10065000CDBFDF91CF911F910F91FF90EF90DF9071
:10066000CF90BF90AF909F908F907F906F905F9052
:100670004F903F900895F8018489958983349105BE
:1006800001F76D817E818F8198850E943ED04B015C
:100690005C01F60180829182A282B38246E050E042
:1006A000B701685F7F4FCE014D960E9446D4892BDB
:1006B00041F6F70180819181A281B3818816990664
:1006C000AA06BB0608F4BDCF84819581A681B781B7
:1006D00088159905AA05BB0508F4B3CF89899A89BD
:1006E000AB89BC8986879787A08BB18B4EEC50E095
:1006F00070E060E0C8010E940E15312CC70182969F
:1007000098AB8FA7F701B696FAABE9AB08969CAB0E
:100710008BAB67019AE1C90ED11CBD96FEABEDAB68
:10072000C701429698AF8FABFD97FAAFE9AF47018B
:10073000FEE18F0E911CF801818D928D181619061D
:100740000CF080CFC8010E942D158333910509F468
:10075000B2C014F58130910509F464C044F4892BCA
:1007600051F3C8010E942D15AC01552775C0833087
:10077000910509F462C00697A1F7C8010E942D15E2
:10078000B82E44E050E0B401C8010E940E15EB2DD4
:10079000E450FF0BAF0160C08A33910509F45FC0DC
:1007A00084F585339105B1F1C697D9F6C8010E9449
:1007B0002D155C01B601CE0189960E94CB828BA5D6
:1007C0009CA5ADA5BEA5892B8A2B8B2BB1F0EDA9DD
:1007D000FEA94080518062807380B601CE0183966D
:1007E0000E94CB828DA19EA1AFA1B8A5A5014816FC
:1007F00059066A067B0609F0B8CF44E050E0B6011E
:1008000018C08B33910509F440C08F3F910509F45E
:1008100092CFA7CFC8010E942D15C8010E942D15A7
:10082000382E89CFC8010E942D1544E050E06FA9F1
:1008300078ADC8010E940E157ECFC8010E942D150B
:10084000B82E44E050E069AD7AADC8010E940E15A3
:100850008B2D8450990BAC0170E060E0EACFC801A9
:100860000E942D1544E050E069A97AA9C8010E94B0
:100870000E15F70166A177A180A591A50E943ED033
:1008800066A377A380A791A756CFC8010E942D1514
:1008900044E050E06BA97CA9C8010E940E15F70145
:1008A00062A573A584A595A50E943ED062A773A7F3
:1008B00084A795A740CFC8010E942D1544E050E0C1
:1008C0006FA578A9C8010E940E15F70162A173A156
:1008D00084A195A10E943ED062A373A384A395A393
:1008E00066A777A780AB91AB26CF33243A94AACEE4
:1008F0002F923F924F925F926F927F928F929F9230
:10090000AF92BF92CF92DF92EF92FF920F931F931D
:10091000CF93DF9300D000D0CDB7DEB78C010E941B
:100920003AC52FEC37E040E050E00E94CDCFDC012B
:10093000CB010196A11DB11DF80184839583A68387
:10094000B78380839183A283B3835801F3E4AF0E0E
:10095000B11CC5010E94D81464E470E0C5010E9476
:100960005216882309F445C10E949DA22B013C0127
:10097000480182E4880E911C48EEC42E43E0D42E38
:10098000E12CF12C52E0252E1E821D82D4018C9187
:100990008330B1F1811166C0F80184819581A6810F
:1009A000B7810196A11DB11D84839583A683B7836A
:1009B0000E949DA26419750986099709A7019601ED
:1009C0000E94ABCFA90161E0C8010E94B07C81E028
:1009D000D4018C938D819E810197C1F20E949DA2CA
:1009E0006419750986099709D801D6962D913D910C
:1009F0004D915C91D997261737074807590720F67C
:100A0000C5010E94D814F80184819581A681B7811F
:100A10000196A11DB11D84839583A683B7830E948F
:100A20009DA2F801FE9660837183828393838D81FA
:100A30009E8126960FB6F894DEBF0FBECDBFDF9124
:100A4000CF911F910F91FF90EF90DF90CF90BF90CB
:100A5000AF909F908F907F906F905F904F903F905E
:100A60002F9008958430F1F4F80184819581A68156
:100A7000B7810196A11DB11D84839583A683B78399
:100A80000E949DA26419750986099709A70196011C
:100A90000E94ABCFA90163E0C8010E94B07CD401E1
:100AA0002C9298CF813051F5F80142AD53AD64AD31
:100AB00075AD9E012F5F3F4FC8010E94D782382E2F
:100AC000F2E08F1390C089819A81AB81BC81F801DB
:100AD00084839583A683B7830E949DA264197509B8
:100AE00086099709A70196010E94ABCFA90163E08F
:100AF000C8010E94B07CD4013C926CCF823009F0D6
:100B000069CFF80142AD53AD64AD75AD9E012F5F65
:100B10003F4FC8010E94D782382EF5E08F135DC089
:100B2000E3E0D401EC93F80182A193A1A4A1B5A1C3
:100B3000892B8A2B8B2B41F484E893E0A0E0B0E072
:100B400082A393A3A4A3B5A3F80186A197A1A0A50E
:100B5000B1A5892B8A2B8B2B61F482A193A1A4A12F
:100B6000B5A1B695A7959795879586A397A3A0A7B6
:100B7000B1A7F80182A593A5A4A5B5A5892B8A2BB9
:100B80008B2BA9F482A193A1A4A1B5A1AC01BD01B5
:100B900023E076956795579547952A95D1F7841B5D
:100BA000950BA60BB70B82A793A7A4A7B5A7F8012F
:100BB00086A197A1A0A5B1A586A797A7A0ABB1AB29
:100BC00082A593A5A4A5B5A582AB93ABA4ABB5AB09
:100BD00081E090E09E838D83FDCE96E0891303C073
:100BE000D4011C92F7CEBFEF3B12F4CEF401108279
:100BF000F1CE1E821D821BCF1F920F920FB60F9255
:100C000011240BB60F922F933F934F935F936F93E3
:100C10007F938F939F93AF93BF93EF93FF938CED4D
:100C200099E00E948E78FF91EF91BF91AF919F91D3
:100C30008F917F916F915F914F913F912F910F9085
:100C40000BBE0F900FBE0F901F9018951F920F9222
:100C50000FB60F9211240BB60F922F933F934F9321
:100C60005F936F937F938F939F93AF93BF93EF9314
:100C7000FF938CED99E00E940F78FF91EF91BF9167
:100C8000AF919F918F917F916F915F914F913F9124
:100C90002F910F900BBE0F900FBE0F901F901895C5
:100CA0001F920F920FB60F9211240BB60F922F9333
:100CB0003F934F935F936F937F938F939F93AF93E4
:100CC000BF93EF93FF9389EF9AE00E948E78FF9194
:100CD000EF91BF91AF919F918F917F916F915F91B4
:100CE0004F913F912F910F900BBE0F900FBE0F9021
:100CF0001F9018951F920F920FB60F9211240BB6EA
:100D00000F922F933F934F935F936F937F938F93A4
:100D10009F93AF93BF93EF93FF9389EF9AE00E9465
:100D20000F78FF91EF91BF91AF919F918F917F913C
:100D30006F915F914F913F912F910F900BBE0F904C
:100D40000FBE0F901F9018951F920F920FB60F9223
:100D500011240BB60F922F933F934F935F936F9392
:100D60007F938F939F93AF93BF93EF93FF9386E10E
:100D70009CE00E948E78FF91EF91BF91AF919F917F
:100D80008F917F916F915F914F913F912F910F9034
:100D90000BBE0F900FBE0F901F9018951F920F92D1
:100DA0000FB60F9211240BB60F922F933F934F93D0
:100DB0005F936F937F938F939F93AF93BF93EF93C3
:100DC000FF9386E19CE00E940F78FF91EF91BF9125
:100DD000AF919F918F917F916F915F914F913F91D3
:100DE0002F910F900BBE0F900FBE0F901F90189574
:100DF0001F920F920FB60F9211240BB60F922F93E2
:100E00003F934F935F936F937F938F939F93AF9392
:100E1000BF93EF93FF9388EF9DE00E948E78FF9140
:100E2000EF91BF91AF919F918F917F916F915F9162
:100E30004F913F912F910F900BBE0F900FBE0F90CF
:100E40001F9018951F920F920FB60F9211240BB698
:100E50000F922F933F934F935F936F937F938F9353
:100E60009F93AF93BF93EF93FF9388EF9DE00E9412
:100E70000F78FF91EF91BF91AF919F918F917F91EB
:100E80006F915F914F913F912F910F900BBE0F90FB
:100E90000FBE0F901F901895CF92DF92EF92FF92A6
:100EA0001F93CF93DF93EC016A017B01122FE88936
:100EB000F98982E08083C11481EED806E104F1044F
:100EC000A1F060E079E08DE390E0A70196010E9437
:100ED000ABCF2150310941095109569547953795B6
:100EE0002795211580E1380798F0E889F989108263
:100EF00060E874E88EE190E0A70196010E94ABCF14
:100F00002150310941095109569547953795279543
:100F1000EC85FD853083EE85FF852083188EEC8976
:100F2000FD891083EA89FB89808188698083EA8949
:100F3000FB8980818F7D8083DF91CF911F91FF900E
:100F4000EF90DF90CF900895DF92EF92FF920F9392
:100F50001F93CF93DF9300D000D0CDB7DEB78B01C6
:100F60007A01D22E67E576E0CE0101960E94B58027
:100F70009E012F5F3F4F4D2DB701C8010E94F5A97B
:100F8000CE0101960E94798026960FB6F894DEBFB6
:100F90000FBECDBFDF91CF911F910F91FF90EF90CA
:100FA000DF900895CF92DF92EF92FF920F931F93FD
:100FB000CF93DF93CDB7DEB7EC970FB6F894DEBFD3
:100FC0000FBECDBFDC012C91222309F469C060E47F
:100FD00074E00E9447C79A8389837E01B3E0EB0ED9
:100FE000F11C01E010E060E474E090E080E00E9419
:100FF00047C7D02EC12EF701819391937F010E3107
:10100000110521F00F5F1F4F892B69F700910D0922
:1010100010910E09E980FA800115110589F1D801B6
:101020006D917C91C7010E9497D4892B29F5D80135
:101030001296ED91FC91BE016F5F7F4F8D2D9C2D1F
:1010400019958C0188EF9DE00E949E816FEE76E1FC
:1010500088EF9DE00E949582C801EC960FB6F89447
:10106000DEBF0FBECDBFDF91CF911F910F91FF90DB
:10107000EF90DF90CF900895F80104811581CCCFD7
:1010800063EF76E188EF9DE00E94B98288EF9DE0F2
:101090000E949E816FEE76E188EF9DE00E9495822E
:1010A00010E000E0D9CFCF9388EF9DE00E945A78FE
:1010B000892BE9F188EF9DE00E943878C82F8A30AB
:1010C00089F08D3079F0883001F568E088EF9DE097
:1010D0000E94A28180911209882331F3815080936C
:1010E0001209E2CFE0911209F0E0EF52F74F1082BF
:1010F00065E576E088EF9DE00E942F8281ED98E023
:101100000E94D28710921209CFCF682F88EF9DE0FE
:101110000E94A281E0911209EB3330F681E08E0F3C
:1011200080931209F0E0EF52F74FC083BDCFCF910B
:1011300008958F929F92AF92BF92CF92DF92EF92DB
:10114000FF920F931F93CF93DF936115710509F4FD
:1011500097C0DB011896EC911897E295E07FE59532
:10116000E595E595E595E73008F08AC0EC010E2E8F
:10117000000CFF0B8827E054F7478F4F0C9436D0B4
:10118000C788D888E188F888438955898E8968E5B9
:1011900076E0CE01DF91CF911F910F91FF90EF90FC
:1011A000DF90CF90BF90AF909F908F900C94438131
:1011B00019968C9162E676E0882359F36DE576E026
:1011C000E8CF19964D915D916D917C911C972AE025
:1011D00030E0CE01DF91CF911F910F91FF90EF9002
:1011E000DF90CF90BF90AF909F908F900C94A9818B
:1011F0001996CD90DD90ED90FC901C9720E030E0AA
:10120000A901C701B6010E9461CE87FF09C066EE41
:1012100074E0CE010E942F82F7FAF094F7F8F09470
:10122000C701B6010E943AD14B015C012AE0BC0122
:10123000A401CE010E9452816CE476E0CE010E94AE
:101240002F82C501B4010E9466CE9B01AC01C7018B
:10125000B6010E9454D02DEC3CEC4CE45DE30E94BE
:1012600055D020E030E040E251E40E94C7CE0E9419
:101270003AD1AB0170E060E02AE0CE010E945281D9
:1012800090E080E01DC019966D917C91CE01DF91B8
:10129000CF911F910F91FF90EF90DF90CF90BF9073
:1012A000AF909F908F900C94378216960D911C9161
:1012B0006BE5CE010E94A281019679F48FEF9FEF3A
:1012C000DF91CF911F910F91FF90EF90DF90CF9022
:1012D000BF90AF909F908F9008950115110579F000
:1012E000B801CE010E949988019641F3D801129667
:1012F0000D911C910115110511F06CE2DACF6DE52D
:10130000CE010E94A28121E030E0019611F030E090
:1013100020E088279927821B930BD2CF16960D9138
:101320001C916BE7CE010E94A281019639F2011552
:10133000110529F1D8016D917C91CE010E9437826F
:10134000019609F4BBCF6AE3CE010E94A281019607
:1013500009F4B4CFB801CE010E949988019609F42E
:10136000ADCFD80112960D911C910115110539F0E0
:101370006CE2CE010E94A2810196C9F69FCF6DE773
:10138000BFCFCF93DF93EC01E881F9810284F3852D
:10139000E02DCE0119958F3F980769F0E881F9811A
:1013A000813291059CF30684F785E02D682FCE01EC
:1013B000199590E080E0DF91CF910895CF92DF9270
:1013C000EF92FF920F931F93CF93DF937C016B01FA
:1013D000DC01ED91FC910284F385E02D1995829753
:1013E00061F0CFEFDFEFCE01DF91CF911F910F9131
:1013F000FF90EF90DF90CF900895F6018085807F79
:101400008460808786E090E00E94C9C38C010097C9
:1014100041F3E1E9F8E0DC01ED93FC9380E4DF01C6
:101420001D928A95E9F780E490E0F8019383828326
:1014300015821482D701ED91FC910284F385E02D91
:10144000C7011995EC010196C9F0C232D10509F422
:101450004DC0C032D1050CF449C0B8018C2FCC3539
:10146000D10549F5D701ED91FC910284F385E02D7A
:10147000C7011995EC018F3F980721F4C8010E941C
:1014800065C4B1CF8236910541F15CF48F3291058C
:1014900009F18C359105D9F0829761F6B80182E2A5
:1014A0000AC08E369105E1F04CF4B8018CE0C636E6
:1014B000D10509F0BFCF0E94487ABCCF8237910591
:1014C00091F0B80189E0C437D105A9F3B3CFB801D1
:1014D0008CE5F1CFB8018FE2EECFB80188E0EBCF19
:1014E000B8018AE0E8CFB8018DE0E5CFF80184814A
:1014F0009581009749F00190F081E02DE80FF91FE8
:1015000031978081882321F0B80180E00E94487AD9
:10151000D80114968D919C910E94C9C3EC0100974B
:1015200039F061E978E00E94A0D4C8010E9465C446
:10153000F601D287C187D0E0C0E055CF8DE090E0C2
:101540000E94C9C3009729F02DE0FC0111922A9551
:10155000E9F708950F931F93CF93DF930097E1F07E
:10156000EC010C851D850115110579F0D8018D91CF
:101570009C91009739F0DC01ED91FC910488F5898C
:10158000E02D1995C8010E9465C4CE01DF91CF916D
:101590001F910F910C94BFC7DF91CF911F910F91B5
:1015A0000895AF92BF92CF92DF92EF92FF920F9386
:1015B0001F93CF93DF9300D01F92CDB7DEB7611595
:1015C0007105B1F06B01182FDB011C96AD90BC903A
:1015D000F501E080F180D701ED91FC910688F78953
:1015E000E02DC7011995811106C0C6010E94AA8A83
:1015F0008FEF9FEF13C0F5019281911124C0D701A5
:10160000ED91FC910190F081E02D612FC7011995BA
:10161000F701818D811111C090E080E00F900F9053
:101620000F900F90DF91CF911F910F91FF90EF904E
:10163000DF90CF90BF90AF900895612F88EF9DE02D
:101640000E94A281E9CF812F8F7D81548A31B8F227
:1016500080ED810F8A3098F283ED810F823078F22D
:101660001F3569F21E3759F21132B1F086EC810F45
:10167000823090F08AED810F873070F01D3361F079
:10168000812F8F7E8F3241F08DED810F823020F0DF
:101690001B3511F01D3511F491FFB1CF19821A825B
:1016A0001B821C82812F012E000C990B9F931F938C
:1016B00088E696E09F938F938E010F5F1F4F1F93D5
:1016C0000F930E941CD56E01F4E0CF0ED11C0F9039
:1016D0000F900F900F900F900F90D8016D918D018A
:1016E000D701ED91FC910190F081E02DC701199592
:1016F000F701818D882339F0F8013197608188EFF7
:101700009DE00E94A2810C151D0539F785CFCF936E
:10171000C82F462F61E070E00E94642661E070E00F
:101720008C2F0E9492268111F9CFCF910895AF920C
:10173000BF92CF92DF92EF92FF920F931F93CF93BE
:10174000DF9300D01F92CDB7DEB78C016B017A0119
:101750008091C9098333E9F45B016801C40ED51E89
:10176000C016D106A9F10E94017B8FE00E940C7B7C
:10177000812F0E940C7B802F0E940C7B0F5F1F4FDC
:1017800080E00E940C7BF50181935F010E94F77A53
:10179000E7CF843369F50E94017B19830A838F2D7B
:1017A0008F778B83EC8264E070E0CE0101960E941B
:1017B000DD7AA70170E060E0C6010E94A4CDE114CB
:1017C000F10421F0B701C6010E94DD7A0E94F77A88
:1017D000C7010F900F900F900F90DF91CF911F9145
:1017E0000F91FF90EF90DF90CF90BF90AF90089552
:1017F0000E94017B0F3F110509F030F419820A8322
:101800001B8263E070E0D1CF17FD0BC019820A8301
:1018100033E0169507953A95E1F7007E08600B8353
:10182000F0CFC80126E0969587952A95E1F7807E4E
:1018300019830A830115104C18F480618B83E1CF62
:101840008861FCCFAF92BF92CF92DF92EF92FF926E
:101850000F931F93CF93DF9300D000D01F921F925E
:10186000CDB7DEB78C017B016A018091C909833352
:10187000E1F45801A40EB51EA016B10609F46FC01C
:101880000E94017B80EF0E940C7B812F0E940C7BC9
:10189000802F0E940C7B0F5F1F4FF70181917F010A
:1018A0000E940C7B0E94F77AE7CF5B01A40EB51E65
:1018B0008433C1F40E94017B19830A838D2D8068D3
:1018C0008B83CC8264E070E0CE0101960E94DD7AC9
:1018D000AE14BF0409F441C0F70181917F010E9459
:1018E0000C7BF6CF0E94017B0F3F110509F028F415
:1018F00019820A8384E08B830CC017FD17C01982FC
:101900000A8333E0169507953A95E1F7007E0C605F
:101910000B8386E0C816D104A0F5F701DE0114960A
:10192000EA15FB0599F081918D93FACFC80126E065
:10193000969587952A95E1F7807E19830A8301158C
:10194000104C10F48461D7CF8C61D5CFB6016D5F98
:101950007F4FCE0101960E94DD7A0E94F77AC60180
:1019600028960FB6F894DEBF0FBECDBFDF91CF91A2
:101970001F910F91FF90EF90DF90CF90BF90AF90AD
:10198000089563E070E0CE0101960E94DD7AF701D0
:1019900081917F010E940C7BAE14BF04C1F7DDCFA3
:1019A000CF93DF931F92CDB7DEB7898341E050E03C
:1019B000BE016F5F7F4F90E080E00E94228C0F900D
:1019C000DF91CF9108951F93CF93DF931F921F92C2
:1019D000CDB7DEB780919008811100C160E372E05D
:1019E00080E090E00E946BA21FB7F89480918F086E
:1019F000811127C0E3EAFBE18491E9EFFBE19491D7
:101A0000E82FF0E0EE0FFF1FE65CF44EA591B491D5
:101A1000EC91E92321F461E085E30E94E5A061E017
:101A200085E30E9413A18CB580618CBD8CB5806468
:101A30008CBD61E084E30E9413A161E083E30E9416
:101A400013A180918F088F5F80938F081FBFE8E7F5
:101A5000FBE1E491F0E0EE0FFF1FEC5AF44E8591AC
:101A6000949190938E0880938D08EEECFBE1E491C5
:101A7000E0938C0861E08AE00E9413A10E94F77A4B
:101A800080E591E00E94209E84E38093C90980E86C
:101A90000E94D08C0E94C27D8823A1F188E00E9420
:101AA000D08C0E94BE7D883069F580E10E94D08C88
:101AB0000E94BE7D803131F580E00E94D08C0E9472
:101AC000BE7D182F81111EC08FE190E00E948126FB
:101AD0008330C1F480E48093800842E06EE170E0DE
:101AE000812F0E94642642E06FE170E0812F0E9406
:101AF00064261F5F183089F70E94A82781E0809331
:101B0000900866C087E38093C90980E80E94D08C62
:101B10000E94C27D8823F9F088E00E94D08C0E9448
:101B2000BE7D8830C1F480E10E94D08C0E94BE7DD1
:101B3000182F803181F480E00E94D08C0E94BE7DFD
:101B4000811109C089E390E00E948126843019F454
:101B500010938008D1CF83E38093C90980E80E9465
:101B6000D08C0E94C27D882371F180E10E94D08CCC
:101B70000E94BE7D803139F582E10E94D08C0E94A6
:101B8000BE7D823101F580E00E94D08C0E94BE7D36
:101B9000811119C084E08093800815E51A8341E023
:101BA00050E0BE016E5F7F4F8BE190E00E94228C7F
:101BB000198341E050E0BE016F5F7F4F8AE190E002
:101BC0000E94228C99CF1092C9090E94A82780E018
:101BD0000F900F90DF91CF911F91089581E0F8CF82
:101BE0006F927F929F92AF92BF92CF92DF92EF92CD
:101BF000FF920F931F93CF93DF931F921F92CDB746
:101C0000DEB7982E8B013A01690122E030E0AE0187
